:100000000C94F9080C9448090C9448090C9448097C
:100010000C9448090C9448090C9448090C9448091C
:100020000C9448090C94591C0C9448090C944809E8
:100030000C946A360C9448090C9448090C944809AD
:100040000C9448090C9448090C947C180C944809A9
:100050000C94AA0E0C9448090C94740E0C94480944
:100060000C94491F0C9448090C94F0310C944809E5
:100070000C947A8F0C9448090C94A9860C94480926
:100080000C9448090C9448090C944809701F751F7A
:100090007A1F831F9A1FB11FC11FD11F0C20F5218A
:1000A000B11FB720C820F720152132218C21E7216C
:1000B0000224CF245E25DE251626B926C0282A294B
:1000C000A429ED29372A652A922AF52A3F2B892B64
:1000D000822C0F3243328632F6320E334F330634DF
:1000E000CD34CD34CD34CD34CD34CD34CD34CD3408
:1000F000CD34CD34CD34823484348934A134A33426
:10010000086AC76A4C6B7B6AA26BD26B3C6AAA6AAC
:10011000AC774A78CF7831798579EE794E816F7AEC
:10012000A17AA17AA17AA17AA17AA17AA17AA17AF7
:10013000A17ACF7A4A7BDF7B047C477C9F7C2A7D37
:10014000137E7A7E7A7E7A7E7A7E7A7E7A7E7A7E56
:100150007A7E7A7EB27ED07EF57E517F8D7FFC7F67
:100160002980C9804E81298129812981298129817C
:10017000298129812981CD8DD08DD08DD08DD98DAA
:10018000DC8DDF8DF18DEE8D0A0D3D3D3D3D3D3D1C
:100190003D3D3D3D3D3D3D3D3D3D3D3D3D3D3D3D8F
:1001A0003D3D3D3D3D3D3D3D3D3D3D3D3D000A0D1F
:1001B000426174743A002025642043656C6C73209E
:1001C00000204C6F77207761726E696E673A202548
:1001D000642E2564000A0D466F756E6420424C2D16
:1001E0004374726C3A20002564000A0D0A0D212127
:1001F000204D495353494E4720424C2D4354524CB5
:100200003A202564202121000A0D43616C69627245
:100210006174696E6720707265737375726520739F
:10022000656E736F722E2E004F4B0A0D000A0D463D
:100230006C696768742D74696D65202575206D691A
:100240006E20546F74616C3A2575206D696E0041A3
:100250006E676C654E69636B202020202020204152
:100260006E676C65526F6C6C20202020202020412E
:1002700063634E69636B20202020202020202041D2
:100280006363526F6C6C2020202020202020205996
:1002900061774779726F202020202020202020487D
:1002A00065696768742056616C756520202020415F
:1002B00063635A2020202020202020202020205648
:1002C0006F6C74616765205B302E31565D20204D68
:1002D0006F746F7220312020202020202020204D9C
:1002E0006F746F7220322020202020202020204D8B
:1002F0006F746F7220332020202020202020204D7A
:100300006F746F7220342020202020202020204D68
:100310006F746F7220352020202020202020204D57
:100320006F746F7220362020202020202020204D46
:100330006F746F7220372020202020202020204D35
:100340006F746F722038202020202020202020521F
:1003500065636569766572204C6576656C2020471B
:1003600079726F20436F6D7061737320202020437A
:10037000757272656E74205B302E31415D202043B2
:1003800061706163697479205B6D41685D20205301
:100390006572766F202020202020202020202043FE
:1003A0006F6D706173732056616C756520202049F4
:1003B00032432D4572726F7220202020202020327F
:1003C00033202020202020202020202020202047F3
:1003D00050535F4E69636B2020202020202020474F
:1003E00050535F526F6C6C20202020202020203240
:1003F00036202020202020202020202020202032D5
:1004000037202020202020202020202020202032C3
:1004100038202020202020202020202020202032B2
:1004200039202020202020202020202020202033A0
:100430003020202020202020202020202020203399
:10044000312020202020202020202020202020219A
:10045000212120494E434F4D50415449424C4520A3
:10046000212121002A002E000A0D20444143206F43
:100470007220493243204552524F52212043686531
:10048000636B204932432C2033567265662C20441E
:10049000414320616E6420424C2D4374726C005BBA
:1004A00025695D005B25695D002B204D696B726FCE
:1004B0004B6F70746572202B0048573A5625642E96
:1004C00025642053573A25642E256425632056342D
:1004D0000053657474696E673A2564202573004D76
:1004E00069786572204572726F72210045525225FB
:1004F00032643A00486172647761726520457272B5
:100500006F7220313A2564202121004D697373698F
:100510006E6720424C2D4374726C3A256421210091
:10052000493243204552524F5221212100486569EA
:100530006768743A202025356900536574706F69C7
:100540006E743A2535690050726573737572653A39
:10055000253569004F66667365743A202025356934
:100560000048656967687420636F6E74726F6C0011
:1005700044495341424C4544006163742E206265F6
:100580006172696E67004E69636B3A2020202020FB
:100590002025356900526F6C6C3A202020202020E5
:1005A00025356900436F6D706173733A20202025F3
:1005B0003569004B25693A25346920204B25693A75
:1005C00025346920004E693A2534692020526F3A5B
:1005D000253469200047733A253469202047693A59
:1005E000253469200050313A253469202050323AB0
:1005F000253469200050333A253469202050343A9C
:1006000025346920004779726F202D2053656E7361
:100610006F72004E69636B25346920282533692E7B
:1006200025692900526F6C6C2534692028253369AF
:100630002E256929004769657225346920282533EC
:100640006929004E69636B202534692028253369A8
:100650002E25782900526F6C6C20253469202825BE
:1006600033692E25782900596177202025346920A7
:100670002825336929004E69636B202534692028B9
:1006800025336929282533692900526F6C6C202590
:1006900034692028253369292825336929005961BF
:1006A00077202025346920282533692928253369B6
:1006B0002900414343202D2053656E736F72004E15
:1006C00069636B2025346920282533692900526F1E
:1006D0006C6C20253469202825336929005A202094
:1006E000202025346920282533692900566F6C7431
:1006F0006167653A2020202533692E25316956002F
:1007000043757272656E743A2020202533692E2558
:1007100031694100506F7765723A202020202025F2
:10072000346957004469736368617267653A2025CC
:1007300035696D416800526563656976657200527E
:10074000432D525353493A2020202025346900522A
:10075000432D5175616C6974793A202534690052D2
:10076000432D4368616E6E656C733A2534690043AE
:100770006F6D70617373004D61676E65743A202010
:1007800020253569004779726F3A202020202025E6
:10079000356900536574706F696E743A2025356948
:1007A00000506F746925693A202025336900506F25
:1007B000746925693A202025336900536572766F84
:1007C000202000536574706F696E74202025336992
:1007D00000506F736974696F6E3A20253369005257
:1007E000616E67653A2533692D25336900424C2DCA
:1007F0004374726C204572726F72732000253364EB
:100800002025336420253364202533642000424CA6
:100810002054656D7065726174757265002533646E
:100820002025336420253364202533642000424C86
:100830002D4374726C20666F756E642000202563F2
:1008400020202025632020202563202020256320D0
:1008500000202563202020256320202025632020E0
:1008600020256320002025632020202D2020202DFE
:100870002020202D2000313000313100313200465F
:100880006C696768742D54696D65202000546F741D
:10089000616C3A2535756D696E004163743A2020AC
:1008A0002535756D696E0028726573657429000AB7
:1008B0000D47656E65726174696E67206465666177
:1008C000756C7420506172616D657465722053653A
:1008D00074202564000A0D5573696E67205061729B
:1008E000616D6574657220536574202564000A0D7E
:1008F00047656E65726174696E67206465666175CF
:100900006C74204D69786572205461626C65000AD0
:100910000D4D697865722D436F6E6669673A2027C1
:1009200025732720282575204D6F746F7273290059
:100930000A0D414343206E6F742063616C696272DB
:1009400061746564210D0A0000008F001E01AD0175
:100950003B02CA025803E603740402058F051B0616
:10096000A7063307BE074808D2085B09E3096B0AEC
:10097000F20A780BFD0B810C040D860D070E870E15
:10098000060F840F00107B10F5106E11E5115B123D
:10099000CF124213B31323149214FE146A15D31505
:1009A0003B16A11605176717C81727188318DE18F6
:1009B00037198E19E319361A871AD61A231B6E1B9C
:1009C000B61BFD1B411C831CC31C001D3C1D751D5B
:1009D000AB1DE01D121E421E6F1E9A1EC31EE91E95
:1009E0000D1F2E1F4D1F691F841F9B1FB01FC31F8C
:1009F000D31FE11FEC1FF51FFB1FFF1F002000008E
:100A000005000500040106010800060102000400BB
:100A100004000700070007000700070007000700A1
:100A200003010301050017010F01060009010A0176
:100A300019010501050119011A010F0100004E6F8E
:100A4000204572726F722020202020202020004E2E
:100A50006F7420636F6D70617469626C6520200033
:100A60004D4B334D6167206E6F7420636F6D706105
:100A7000004E6F20464320636F6D6D756E69636134
:100A80007400436F6D7061737320636F6D6D756E6D
:100A900069630047505320636F6D6D756E696361C4
:100AA00074696F00636F6D706173732076616C752C
:100AB00065202020005243205369676E616C206CD2
:100AC0006F73742020004643207370692072782071
:100AD0006572726F7220004E6F204E4320636F6DFF
:100AE0006D756E69636174004643204E69636B20C7
:100AF0004779726F2020202000464320526F6C6C93
:100B0000204779726F2020202000464320596177CA
:100B1000204779726F2020202020004643204E6914
:100B2000636B204143432020202020004643205275
:100B30006F6C6C204143432020202020004643203E
:100B40005A2D414343202020202020202000507295
:100B50006573737572652073656E736F72200049DB
:100B600032432046432D3E424C2D4374726C20008C
:100B7000426C204D697373696E672020202020200D
:100B8000004D69786572204572726F7220202020B6
:100B900020004361726566726565204572726F72EE
:100BA00020200047505320466978206C6F737420D2
:100BB000202020004D61676E6574204572726F724F
:100BC00020202020004D6F746F7220726573746155
:100BD000727420202000424C204C696D697461744D
:100BE000696F6E202020004750532052616E676568
:100BF00020202020202020004E6F2053442D4361D0
:100C000072642020202020200053442D4C6F676701
:100C1000696E67206572726F7200466C79696E67E3
:100C20002072616E676521202020004D617820418F
:100C30006C74697475646521202020004E6F204714
:100C400050532066697820202020202000636F6D9B
:100C500070617373206E6F742063616C2E002021AD
:100C600021204C69506F20766F6C7461676520217C
:100C70002120200020202020204D696B726F4B6FB7
:100C80007074657220202020200020202020202049
:100C90002020202020202020202020202020200074
:100CA00020202532692E253169562020002020255C
:100CB00032692E25316956202000414C543A2534A2
:100CC000696D20256300414C543A2534696D20201C
:100CD00000414C543A2D2D2D2D2000202025326925
:100CE0003A2530326920200020202532693A25300B
:100CF00032692020004449523A202533642563009C
:100D000043002000202025356920200020202535A3
:100D100069202000493A2532692E25316941200099
:100D20003A003A003A002D2D2D2D2D2D2D2D2D2B55
:100D30002D2D2D2D2D2D2D2D2D2D2D002D2D2D2D10
:100D40002D2D2D2D2D2D2D2D2D2D2D2D2D2D2D2DD3
:100D50002D003A005341543A25326420004449534F
:100D6000543A2533646D00442000334400212100AF
:100D70004D41473A25337525252000484D3A253306
:100D800064256320256300696E636C3A253264250F
:100D900063282532692900202020202532756D2FF7
:100DA000733A2020484D3A2533642563202563009B
:100DB0004552523A202532642021004552523A20B1
:100DC000002121204C69506F20766F6C746167653B
:100DD00020212100207777772E4D696B726F4B6F42
:100DE000707465722E6465202000202532693A25D2
:100DF00030326920202532692E253169562025346C
:100E0000696D416800202532693A25303269202019
:100E10002532692E25316956202534696D416800D7
:100E20004449523A253364256300414C543A2534F1
:100E3000696D00414C543A2534696D00414C543A77
:100E40002D2D2D2D2000256300484D3A2533642596
:100E5000632020444953543A2533646D20256300B0
:100E60005057523A2532692E25316941202825698B
:100E7000572920004346002020004750533A25328E
:100E8000756D2F73205341543A2564200020203380
:100E90004420004E4F4649580044475053200020FC
:100EA00020204E6F204E6176694374726C202020A2
:100EB00020202020002532692E2569202532692E28
:100EC0002569202532692E2569202532692E25695C
:100ED00041002533692025336920253369202533D6
:100EE00069256343002532692E2569202532692E44
:100EF000256941002532692E2569202532692E2574
:100F000069202532692E2569202532692E256941FF
:100F100000253369202533692563432020202020C4
:100F200020202000253369202533692025336920BE
:100F3000253369256343004552523A202532642007
:100F400021004552523A20002121204C69506F2047
:100F5000766F6C7461676520212100207777772E8A
:100F60004D696B726F4B6F707465722E64652020D3
:100F70000053657474696E673A25752025732000E7
:100F80004D696E3A2532692E253169562025732028
:100F900000414C543A00504F54493A2533752000D3
:100FA000284F4E29202000284F46462920004C4932
:100FB0004D495400564152494F0044495341424C17
:100FC00045440043463A0044495341424C4544009D
:100FD00020284F4E29200020284F46462900205423
:100FE00045414348004750533A0044495341424C1D
:100FF0004544002846524545290028484F4D45297B
:10100000002841494429200028484F4C4429002009
:1010100046533A257573656B2000484F4D45204176
:101020004C543A0025756D00484F4C4420004E69E1
:101030003A25346920526F3A25346920433A2533E2
:10104000690047733A2534692059613A253469208B
:101050000050313A2534692050323A253469203322
:101060003A2533690050343A2534692050353A2501
:10107000346920363A25336900434F55504C494E68
:1010800047204F46462120004C4F4F50494E4721A4
:1010900020004848212000434F4D50415353204FDA
:1010A0004646212000004F50515253545356574842
:1010B000005859005A5545464748410049424A4A56
:1010C0000000000000000000000000444C4D000043
:1010D0000000004E0000004B00430A0D7777772E8A
:1010E0004D696B726F4B6F707465722E646520284A
:1010F000632920486953797374656D7320476D6265
:1011000048000A0D74686520757365206F66207449
:1011100068697320736F66747761726520697320E4
:101120006F6E6C79207065726D6974746564200AE5
:101130000D6F6E206F726967696E616C204D696B0F
:10114000726F4B6F707465722D4861726477617253
:1011500065005573657200486F5454205634004141
:1011600043542044534C004A657469005370656BC6
:101170007472756D0050504D000A0D5265636569BB
:101180007665723A2000532E42757300756E6B6E51
:101190006F776E2E205573696E672050504D2E2E3E
:1011A0002E006E6F7420737570706F72746564209A
:1011B000627920686172647761726521000A0D4668
:1011C0006C69676874436F6E74726F6C0A0D486166
:1011D0007264776172653A25642E25640A0D536F37
:1011E0006674776172653A5625642E2564256320FE
:1011F000000011241FBECFEFD0E4DEBFCDBF12E050
:10120000A0E0B1E0E4ECF4E201E00BBF02C0079023
:101210000D92A43DB107D9F71BE0A4EDB2E001C0E7
:101220001D92AC3DB107E1F77AEAE2E0F0E081E23D
:1012300080935700D4907E010894E11CF11C20EFAC
:1012400037EF41E050E087016FE0DA01C9012F5F1D
:101250003F4F4F4F5F4FABBFFC018791F801819328
:101260008F01615067FFF1CFF7016EE08191782720
:101270007095615067FFFACF8889781729F0F7E9F0
:10128000DF1611F40000FECF0E941B0A0C9461923D
:101290000C94000088E891E09F938F9380E695E19D
:1012A0009F938F93E0913B05F0913C0509950F903A
:1012B0000F900F900F90089580918407E82FFF27DB
:1012C000EE0FFF1FE954F74F808191818D5E9F4F94
:1012D00014F010920201808191818A5B9F4FCCF4BF
:1012E000809102018823A9F481E08093020180911A
:1012F0006F058F5F80936F05853038F088EE93E03F
:10130000909309038093080304C066E970E00E948B
:10131000183A80916F0599279093070780930607E5
:1013200008951F93CF93DF93182F882389F08EEAB7
:1013300091E09F938F9380E695E19F938F93E09147
:101340003B05F0913C0509950F900F900F900F9081
:101350008091A707823308F044C084EF91E00E9497
:101360006F19EC01112329F0CE010E94781988230E
:10137000D9F3C2E0D0E026E530E080911F019091E2
:1013800020018217930730F02196255D3F4FC7302B
:10139000D10598F38091A7079927C89F9001C99F0D
:1013A000300DD89F300D1124209300011123D9F066
:1013B00068EC70E08C2F0E94183ADF93CF9386EB95
:1013C00091E09F938F9380E695E19F938F93E091B7
:1013D0003B05F0913C0509958DB79EB706968DBFEC
:1013E00002C080930001112311F1809100016AE095
:1013F0000E94B491892F99279F938F938091000128
:101400000E94B49199279F938F9381EC91E09F93D1
:101410008F9380E695E19F938F93E0913B05F09148
:101420003C0509952DB73EB7285F3F4F2DBFDF9193
:10143000CF911F910895CFEFD0E4DEBFCDBF8824B8
:10144000992414B815B8B7EEEB2EB3E0FB2E2EECB2
:101450003FEFE20EF31EF7FEFACF199B02C085E1C3
:1014600001C086E18093010181E887B93E9A8FEF40
:1014700088B98BE184B981E085B98EE38AB987E4C4
:101480008BB9469A84B7877F84BF8091600088615A
:10149000809360001092600084EC99E090930903BF
:1014A0008093080310921404109213041092BC0845
:1014B0001092BB0810921604109215041092180492
:1014C0001092170420910101243128F084EC94E05B
:1014D000A0E0B0E004C08BE095E0A0E0B0E0809335
:1014E0003C0190933D01A0933E01B0933F012A300F
:1014F00011F0243110F0289801C0289A2C3010F0F7
:10150000263111F4299A01C029980E94D8190E9405
:10151000A9190E9468150E9441360E94DA1D81E0D7
:101520000E94A4310E949A680E9451720E94458EC6
:10153000809101018C3010F0863111F4299A01C09C
:10154000299878940E94C33080914D0382608093E3
:101550004D03109250030E94644584EF91E00E9475
:101560006F197C0180914D0380FD05C0C7010E9469
:1015700078198823B9F385ED91E09F938F93A0E6C6
:10158000AA2EA5E1BA2EBF92AF92E0913B05F09151
:101590003C05099580EA9FE00E946F197C01C0E03C
:1015A000D0E00F900F900F900F9009E518E0FDE04C
:1015B000CF2EF8E0DF2E0E94644580914D0380FD20
:1015C00005C0C7010E9478198823B9F3F60180810C
:1015D0001816ACF40BC00E94644580914D0380FD49
:1015E00005C0C7010E9478198823B9F3C7010E947A
:1015F0007819882321F4F8018081882364F7F801A1
:10160000808187FF19C02196DF93CF93219787EEC2
:1016100091E09F938F93BF92AF92E0913B05F09141
:101620003C0509958091D5028F5F8093D5022DB737
:101630003EB72A5F3F4F2DBF219684E090E0C80E51
:10164000D91E085F1F4FCC30D10508F4B4CFC0E0DD
:10165000D0E006E518E0EDE0EE2EE8E0FE2EF80121
:10166000838187FD1DC0F70180811816CCF4219677
:10167000DF93CF9321978AEE91E09F938F9380E63B
:1016800095E19F938F93E0913B05F0913C0509957F
:1016900082E0809306032DB73EB72A5F3F4F2DBFF0
:1016A000F801838180788383219624E030E0E20E84
:1016B000F31E085F1F4FCC30D10588F20E944A0903
:1016C000909182078091D502981728F48091550552
:1016D00080618093550588E092E09F938F93C0E6E8
:1016E000D5E1DF93CF93E0913B05F0913C0509955F
:1016F00088EE93E00E946F197C010E94E01D0F901C
:101700000F900F900F90C7010E9478198823D9F38A
:1017100088E292E09F938F93DF93CF93E0913B0514
:10172000F0913C05099580E00E94FC3A809101010E
:101730000F900F900F900F908A3011F0843110F0BD
:10174000289801C0289A80ED97E090930903809330
:10175000080385E5809371058EE090E00E94E72EF6
:101760009927182F00278FE090E00E94E72E080F9E
:10177000111D1093DB020093DA028AE090E00E94D0
:10178000E72E9927182F00278BE090E00E94E72E84
:10179000080F111D1093D9020093D8020F5F1F4F3D
:1017A00039F08091DA029091DB028F5F9F4F41F414
:1017B0001092DB021092DA021092D9021092D80233
:1017C0008091D8029091D9029F938F938091DA02F1
:1017D0009091DB029F938F938DE292E09F938F9382
:1017E000DF93CF93E0913B05F0913C0509950E9472
:1017F000742388E893E19093370180933601C1E028
:10180000C09370058C2F0E9491098091AA070E94B5
:10181000918D0E944A0980ED97E00E946F197C012A
:101820008AEF90E00E946F1983E08093DE061092A9
:10183000D4028091F1072DB73EB7285F3F4F2DBFEF
:1018400084FF02C0C093DC028091DE02882311F085
:101850004798FECF80910C03882309F43DC2809104
:101860001101882309F438C210920C0380916F058E
:10187000882319F00E945C0902C00E94A3480E94BC
:101880006445209101012A3011F0243110F028988C
:1018900001C0289A80910704882331F080910704C1
:1018A0008150809307040EC080916F008062809306
:1018B0006F001092B8081092B708809155058860A3
:1018C000809355058091360190913701019790934F
:1018D0003701809336018091360190913701892B31
:1018E00021F080914E038823C9F1809136019091B7
:1018F0003701892BD9F40E94CE3185E090E0909396
:10190000370180933601809118079091190701964D
:1019100090931907809318078091550581608093F3
:1019200055058091DF0682608093DF068091090172
:1019300090910A018F5F9F4FC1F480910604882324
:10194000A1F088EA91E6909309038093080380E868
:1019500090E090930A018093090107C02A3011F0AA
:10196000243110F0289801C0289A0E94FD8E8091A1
:101970000C03882309F0B0C180911C05882319F05D
:101980000E94D281A9C180910F01882311F00E9489
:10199000311A0E94AC150E94FA10C7010E947819F2
:1019A000882309F495C184E190E0E80EF91E0E94B5
:1019B000EF198091AA07863019F40E94707704C04D
:1019C000843011F40E94A28280914E03882349F052
:1019D000809155058260809355058091DF06826075
:1019E0000FC08091080390910903892B59F48091CD
:1019F000360190913701079728F08091DF068D7F9F
:101A00008093DF068091DC02882361F080910704D7
:101A1000873940F01092DC0288E893E19093090343
:101A20008093080380910401882321F081508093E2
:101A300004012EC080937B051092DB031092DA0321
:101A40001092D9031092D8031092D7031092D603A4
:101A5000809107048823E1F48091090190910A01A3
:101A60008F5F9F4FA9F42091DC02223089F088E932
:101A70009AE3909309038093080380E09CE090939D
:101A80000A0180930901222319F082E08093DC028D
:101A900080919701893C48F0815080939701809113
:101AA00055058B7F809355053FC080919809882309
:101AB000F9F08091550584608093550589E0809305
:101AC000E2048091090190910A018F5F9F4F81F498
:101AD00080910604882361F088E99AE390930903D2
:101AE0008093080380E098EA90930A0180930901AB
:101AF0001092D4041092D3041092D2041092D10404
:101B00001092D00410928B091092CA091092C90940
:101B10001092CC091092CB098FEF9FEF9093C809D8
:101B20008093C7091092970180910001282F3327D5
:101B300080911F019091200182179307CCF480912E
:101B4000CF0380628093CF038091090190910A01B5
:101B50008F5F9F4FC1F480E797E1909309038093D3
:101B6000080380E093E090930A01809309010BC081
:101B70008091080390910903892B29F48091CF0368
:101B80008F7D8093CF030E94916D84E08093070343
:101B90008091DD028F5F8093DD02813309F04FC0B9
:101BA0001092DD028091CF0381FF0AC08091D6029E
:101BB0009091D70201969093D7028093D6023FC0AE
:101BC0005AEA852E55E0952E809127079091280797
:101BD0009C01442737FD4095542F80911701909127
:101BE0001801A0911901B0911A01281739074A0765
:101BF0005B0734F4809127079091280701961BC05A
:101C000080912707909128079C01442737FD409534
:101C1000542F8091170190911801A0911901B09152
:101C20001A0182179307A407B5074CF48091270780
:101C3000909128070197909328078093270708948D
:101C4000811C911C32E783163BE0930609F040C0EB
:101C5000882499242091DA023091DB022F5F3F4FD4
:101C60003093DB022093DA028091D8029091D9025E
:101C700001969093D9028093D802832F9927682FD9
:101C80008EE090E00E94EF2E8091DA029091DB02CC
:101C90009070682F8FE090E00E94EF2E8091D80224
:101CA0009091D902892F9927682F8AE090E00E94AD
:101CB000EF2E8091D8029091D9029070682F8BE01E
:101CC00090E00E94EF2E84E190E00E946F197C0169
:101CD0000E94E16D0E94687280910703882309F0D9
:101CE000B3CD0E94BB68B0CD1F920F920FB60F927A
:101CF00011248F939F93EF93FF9380910601882384
:101D0000E1F48091F8029091F90201969093F90222
:101D10008093F802FC01E15DF94FE081ED3019F0AC
:101D20008F3A910539F41092F9021092F80281E08D
:101D300080930601E093C60004C01092F90210924D
:101D4000F802FF91EF919F918F910F900FBE0F902E
:101D50001F9018951F920F920FB60F9211242F9378
:101D60003F934F935F936F937F938F939F93AF9323
:101D7000BF93CF93EF93FF9390E08091DE02813089
:101D800029F48091C6008093CE00CCC08091DE0201
:101D9000823029F48091C60080937E05C3C0809173
:101DA000C6008093F0025091FE025F3A10F09093CB
:101DB000FF028091F0028D3009F065C08091FF0232
:101DC000823009F060C09093FF02852F99278258D6
:101DD0009A4FFC01329740812091FA023091FB0228
:101DE000241B3109DC0111978C91281B3109C90191
:101DF0009F709093FB028093FA0246E09695879538
:101E00004A95E1F7982F935C9093FC022F73307002
:101E1000235C2093FD028081981729F48C91281768
:101E200011F491E006C090E08091ED028F5F809305
:101E3000ED02C091EF02CC2309F074C0992309F49C
:101E400071C081E08093EF02580F5093EC02515023
:101E5000E52FFF27E258FA4F8DE0808380918005BF
:101E6000823509F05FC00E94742388E190E02CE085
:101E70000FB6F894A895809360000FBE2093600081
:101E8000C09306034FC02091FF02822F9927813013
:101E90009105F9F0823091051CF4892B21F040C0A6
:101EA000029711F13DC08091F002833239F48091A4
:101EB000EF02882319F481E08093FF028091F00201
:101EC00080937E0581E08093FE028091F002992745
:101ED00022C02F5F2093FF02E52FFF27E258FA4F21
:101EE0008091F002808309C0E52FFF27E258FA4F66
:101EF0008091F00280835F3A20F45F5F5093FE028E
:101F000002C01092FF022091F0028091FA0290919B
:101F1000FB02820F911D9093FB028093FA0202C094
:101F20001092FF02FF91EF91CF91BF91AF919F91DE
:101F30008F917F916F915F914F913F912F910F9072
:101F40000FBE0F901F901895AC01A0E0B0E09D016E
:101F5000A817B90748F4EFE2F6E08191280F311D88
:101F60001196A417B507C8F33F70FD01E15DF94F65
:101F7000C90156E0969587955A95E1F7835C808371
:101F80001196FD01E15DF94F2F733070822F835C54
:101F90008083A05DB94F8DE08C93109206018091F3
:101FA0002F068093C6000895A0E0B0E0EAEDFFE0C0
:101FB0000C942D922C859D850E85BB2483E2809305
:101FC0002F069F59909330062093310633E0E32E7D
:101FD000F12C002309F49EC0CF84D888BE016D5E29
:101FE0007F4FA989BA890150109709F493C01097BF
:101FF000B9F0F601EB0DF11DB3949081119791F4B6
:10200000002349F1FB016E5F7F4FDB01C080D1806F
:102010006E5F7F4F0D90BC91A02DBB24015002C07C
:1020200090E019C01097B9F0F601EB0DF11DB394D3
:102030004081119791F4002341F1FB016E5F7F4FC6
:10204000DB01C080D1806E5F7F4F0D90BC91A02DD1
:10205000BB24015002C040E018C01097B1F0F60157
:10206000EB0DF11DB3941081119781F4002371F0F1
:10207000FB013296DB01CD90DC90BF016E5F7F4F9C
:10208000A081B181BB24015001C010E0F701E15DE6
:10209000F94F892F86958695835C80830894E11C8F
:1020A000F11CF701E15DF94F892F9927837090703A
:1020B00024E0880F991F2A95E1F755279A0194E0AB
:1020C000369527959A95E1F7822B835C8083089457
:1020D000E11CF11CF701E15DF94F4F705070440FA6
:1020E000551F440F551F812F992726E096958795F8
:1020F0002A95E1F7842B835C80830894E11CF11C12
:10210000F701E15DF94F1F73135C10830894E11C24
:10211000F11C6ACFC7010E94A40FE9E00C94499218
:10212000A3E07A2F4091EC024650442309F458C0B2
:10213000E72FFF27E258FA4F80818D537F5FE72F0B
:10214000FF27E258FA4F20812D537F5FE72FFF27AB
:10215000E258FA4F30813D537F5FE72FFF27E25867
:10216000FA4F60816D537F5F9927880F991F880F01
:10217000991F522F52955F70582B822F99278F707D
:102180009070F4E0880F991FFA95E1F7232F2695B8
:102190002695282B832F992783709070E6E0880F6F
:1021A000991FEA95E1F7682B41504F3FC9F0EA2F9C
:1021B000FF27E258FA4F5083AF5F41504F3F81F005
:1021C000EA2FFF27E258FA4F2083AF5F41504F3F7D
:1021D00039F0EA2FFF27E258FA4F6083AF5FA5CFAF
:1021E00081E895E09093EB028093EA02A350A093DC
:1021F000E9020895A2E0B0E0E0E0F1E10C9433924E
:102200008091EF02882309F457C40E9490108091B6
:102210007F05823609F023C3809180059927803796
:10222000910509F4AFC081379105C4F48A36910550
:1022300009F480C28B36910544F48B34910571F119
:102240008636910509F45FC10AC38D36910509F4FC
:1022500069C08E36910509F44DC001C384379105DC
:1022600041F1853791054CF48137910509F491C00E
:102270008337910509F4DFC0F2C28737910509F46D
:102280001BC2883791052CF48537910509F4D7C115
:10229000E6C28937910509F46DC1E1C2E091EA0215
:1022A000F091EB0280819181909389018093880164
:1022B000D6C28091EC02A091EA02B091EB02853186
:1022C00040F080E1E9E5F5E00D9001928A95E1F7B3
:1022D0000DC08D919D910D90BC91A02D80935905BD
:1022E00090935A05A0935B05B0935C0580EF8093B3
:1022F000E7024BC0809106018823E1F38DE490E072
:102300009F938F9380E098E09F938F9381E08F93CA
:102310008F938EE48F930E94D40F8DB79EB707964C
:102320008DBF9DC2A091EA02B091EB021C911130C9
:1023300081F48DE4E0E0F8E00D9001928A95E1F7F8
:102340000E9400301983809155058F7E809355053A
:1023500001C01982809106018823E1F381E090E0B9
:102360009F938F93CE0101969F938F9381E08F93DC
:102370008F938DE48F930E94D40FADB7BEB717969D
:10238000ADBF6DC281E08093F2028FEF80930401B4
:1023900066C2E091EA02F091EB02E0818E2F8A5052
:1023A0008A3058F48983882311F481E003C0863091
:1023B00010F085E0898361E00EC08E2F84518A3051
:1023C00070F48983882311F481E003C0863010F013
:1023D00085E0898360E089810E94803012C0E983B2
:1023E000EF3F19F40E94633089838981882311F4B7
:1023F00081E003C0863010F085E0898389810E94E6
:10240000052F809106018823E1F38CE790E09F93EC
:102410008F9383E897E09F938F9381E090E09F9361
:102420008F93CE0101969F938F9382E08F9381E0EB
:102430008F9381E577C12091EA023091EB02D901B7
:102440008C918150853008F045C0F90181818C352F
:1024500009F040C0809106048823E1F52F5F3F4FCB
:102460008CE7E3E8F7E0D9010D9001928A95E1F756
:10247000F90182910E94702F8091C4079927AA27A1
:10248000BB27BC01CD0124EC39E040E050E00E94C4
:102490009591DC01CB018093800190938101A09301
:1024A0008201B09383018091C5079927AA27BB2792
:1024B000BC01CD010E949591DC01CB0180937C0190
:1024C00090937D01A0937E01B0937F010E946330C1
:1024D000898301C01982809106018823E1F381E09C
:1024E00090E09F938F93CE0101969F938F9381E00D
:1024F0008F938F9383E58F930E94D40F8DB79EB7F0
:1025000007968DBF26C0E091EA02F091EB02E081D0
:102510008E2F8150853018F48E2F0E94052F0E9437
:1025200063308983809106018823E1F381E090E0A4
:102530009F938F93CE0101969F938F9381E08F930A
:102540008F9386E48F930E94D40FADB7BEB71796D2
:10255000ADBF80910604882329F46EE670E089817E
:102560000E94183A80E00E9491098091AA070E9477
:10257000918D75C1E091EA02F091EB02808199277B
:1025800087FD90959093D2088093D10881819927F7
:1025900087FD90959093D4088093D30882819927E2
:1025A00087FD90959093D6088093D50883819927CD
:1025B00087FD90959093D8088093D70884819927B8
:1025C00087FD90959093DA088093D90885819927A3
:1025D00087FD90959093DC088093DB08868199278E
:1025E00087FD90959093DE088093DD088781992779
:1025F00087FD90959093E0088093DF088085992768
:1026000087FD90959093E2088093E1088185992752
:1026100087FD90959093E4088093E308828599273D
:1026200087FD90959093E6088093E5088385992728
:1026300087FD90959093E8088093E70810C1E0919A
:10264000EA02F091EB0280810E949A358A83882306
:1026500019F481E0898301C01982809106018823E1
:10266000E1F388E090E09F938F938EE498E09F934E
:102670008F9321E030E03F932F938091EA02909175
:10268000EB029F938F933F932F93CE0102969F93DC
:102690008F933F932F93CE01820F931F9F938F931E
:1026A00084E08F9381E08F9385E58F930E94D40F10
:1026B000EDB7FEB773963CC08091E902893008F40B
:1026C000CEC02091EA023091EB022F5F3F4F88E0AD
:1026D000AEE4B8E0F90101900D928A95E1F7D901D5
:1026E0008E910E94F0348A83882319F481E08983D3
:1026F00001C01982809106018823E1F321E030E0D6
:102700003F932F93CE0102969F938F933F932F93E6
:10271000CE01820F931F9F938F9382E08F9381E06E
:102720008F9387E58F930E94D40FEDB7FEB73B964A
:10273000EDBF95C080910604882309F090C00E94E7
:10274000448D8983823019F0843009F088C020E4F8
:1027500030E0F8948091C1008F738093C100809124
:10276000C9008F738093C9008091C100877E8093D8
:10277000C1008091C900877E8093C9008091C80004
:1027800087FF03C08091CE00F9CF8091C00087FF02
:1027900003C08091C600F9CFE091EA02F091EB020C
:1027A000E081E13021F482E08093DE022EC0E43645
:1027B00011F421E830E081E08093DE02832F992735
:1027C0008093CD002093CC008091CD008093C500F4
:1027D0008091CC008093C4008091CA008F7D80934B
:1027E000CA008091CA008F7E8093CA008091C90080
:1027F0008B7F8093C9008091CA0084608093CA0057
:102800008091CA0082608093CA008091CA00877F4D
:102810008093CA008091C200877F8093C20080911C
:10282000C9008E7F8093C9008091C1008861809328
:10283000C1008091C90088618093C9008091C10066
:1028400080688093C1008091C90080688093C9002E
:1028500010926E0010926F00109270007894809128
:10286000800599278436910509F4BBC0853691050A
:10287000ACF48136910509F46FC0823691052CF4D1
:102880008B34910509F45DC00FC18236910509F4BE
:1028900070C08336910509F47FC006C18C3691055E
:1028A00009F4EDC08D3691054CF48736910509F495
:1028B000F8C08836910509F4B2C0F6C08437910596
:1028C00029F08637910509F4E8C0EEC08091EC024A
:1028D000A091EA02B091EB02803140F080E1E9E59D
:1028E000F5E00D9001928A95E1F70DC08D919D91D3
:1028F0000D90BC91A02D8093590590935A05A093FB
:102900005B05B0935C05809106018823E1F31F927B
:10291000809103018F9384E58F930E94D40F8AEFF7
:102920008093E7028FEF8093040180EA9FE00E948A
:102930006F199093E0028093DF020F900F900F9039
:10294000B3C0E091EA02F091EB0280819181909313
:10295000890180938801A8C0E091EA02F091EB021E
:10296000808180930501803298F08FE1809305018A
:102970000FC0A091EA02B091EB028BE0E1E7F5E035
:102980000D9001928A95E1F780917A058093200756
:102990008FEF8093040188C08091E3029091E4025C
:1029A000892B89F4E091EA02F091EB02E081EE23B9
:1029B00051F08AE0E89FC00111240E946F199093A2
:1029C0004C0580934B05E091EA02F091EB02908177
:1029D0008AE0989FC00111249093E4028093E3025F
:1029E00015C08FEF80930401E091EA02F091EB02B1
:1029F00090818AE0989FC00111249093E602809311
:102A0000E502892B19F081E08093F40280EA9FE0CF
:102A10000E946F199093E0028093DF0245C08FEF10
:102A200080930401E091EA02F091EB02908197FD1E
:102A300008C082E08093F1021092E2021092E1025B
:102A40001AC0909580914603892B8093460391810B
:102A50008AE0989FC00111249093E2028093E102E2
:102A600084E08093F10280EA9FE00E946F199093C6
:102A7000E0028093DF0281E08093F50215C08FEFC2
:102A800080930401E091EA02F091EB02808180934F
:102A9000470381E08093F60207C081E08093F30250
:102AA00003C081E08093F7021092EF021092EB02D4
:102AB0001092EA021092E902E3E0CE5F0C944F928A
:102AC000982F8091C00085FFFCCF9093C600089599
:102AD0000F931F9388E18093C1008091C0008260B2
:102AE0008093C0008091C10080688093C100809174
:102AF000C10080648093C10000E010E00093C50035
:102B00008AE290E08093C4008091E5029091E60211
:102B10000E946F1990934E0580934D058CED90E0C7
:102B20000E946F1990937D0580937C0510924F054C
:102B30008AE58093500583E0809353058BE0809372
:102B40005105109252051093EB020093EA02109285
:102B5000E9021F910F910895A0E1B0E0E2EBF5E1E9
:102B60000C94309280910601882309F4C1C28091AF
:102B7000DF029091E0020E947819882361F01092A0
:102B8000E2021092E1021092E6021092E502109227
:102B9000E4021092E3028091E1029091E202892B1B
:102BA00041F080912D0690912E060E94781988237D
:102BB00029F48091F502882309F460C08091060110
:102BC000882309F45BC08091F10202E317E08430AE
:102BD000A8F00E948A2380E590E09F938F931F9333
:102BE0000F9381E08F938F9388E48F930E94D40F8B
:102BF0002DB73EB7295F3F4F2DBF34C01092480319
:102C00008FE494E09F938F938DE793E29F938F934C
:102C1000E0913B05F0913C05099584E190E09F939C
:102C20008F931F930F9381E090E09F938F9381EF99
:102C300092E09F938F9382E08F9381E08F9388E45B
:102C40008F930E94D40F8091F102982F8F5F809311
:102C5000F1022DB73EB7215F3F4F2DBF943010F0EA
:102C60001092F1028091E1029091E2020E946F19AC
:102C700090932E0680932D061092F5028091F60215
:102C8000882351F180910601882331F10E948A2323
:102C900080E590E09F938F9382E397E09F938F93DB
:102CA00021E030E03F932F9381E291E09F938F9357
:102CB0003F932F9387E493E09F938F9383E08F93C9
:102CC00081E08F938CE48F930E94D40F1092F602D0
:102CD0008DB79EB70F968DBF8091F3028823D1F0F8
:102CE000809106018823B1F08AE090E09F938F9352
:102CF0008FE495E09F938F9381E08F938F9386E588
:102D00008F930E94D40F1092F3022DB73EB7295F24
:102D10003F4F2DBF8091F7028823D9F080910601A3
:102D20008823B9F08BE090E09F938F9381E795E043
:102D30009F938F9381E08F93809103018F9387E41A
:102D40008F930E94D40F1092F7028DB79EB707960B
:102D50008DBF80917C0590917D050E947819882314
:102D600009F461C080910601882309F45CC0809158
:102D70009F079927880F991F880F991F7C010027AB
:102D8000F7FC0095102F8091610490916204A0914E
:102D90006304B0916404BC01CD01A80197010E94B5
:102DA000099230936A0520936905809159049091A6
:102DB0005A04A0915B04B0915C04BC01CD01A80150
:102DC00097010E94099230936C0520936B058091C6
:102DD000E40380936D058091E30380936E0588E0A2
:102DE00090E09F938F9389E695E09F938F9381E086
:102DF0008F9383E08F938BE68F930E94D40F809103
:102E00006F052DB73EB7295F3F4F2DBF853018F0B6
:102E100086E080936F0583E690E00E946F1990939F
:102E20007D0580937C058091E5029091E602892BD7
:102E300041F080914D0590914E050E9478198823AC
:102E400021F48091F402882339F1809106018823CE
:102E500019F10E94EE3882E490E09F938F938EEDFB
:102E600096E09F938F9381E08F938F9384E48F9369
:102E70000E94D40F1092F4028DB79EB707968DBFB3
:102E80008091E5029091E602009731F00E946F195F
:102E900090934E0580934D058091E3029091E4025A
:102EA000892B09F4B8C080914B0590914C050E9484
:102EB0007819882309F4AFC080910601882309F4AA
:102EC000AAC080919F079927880F991F880F991F83
:102ED0007C010027F7FC0095102F809161049091F0
:102EE0006204A0916304B0916404BC01CD01A80107
:102EF00097010E94099230933E0520933D058091F1
:102F0000590490915A04A0915B04B0915C04BC01F7
:102F1000CD01A80197010E940992309340052093AA
:102F20003F0520918009309181094091820950919B
:102F30008309DA01C90163E0880F991FAA1FBB1F2B
:102F40006A95D1F7820F931FA41FB51F820F931F9D
:102F5000A41FB51F20913C0130913D0140913E01DD
:102F600050913F01BC01CD010E940992309342056E
:102F7000209341058091290490912A04A0912B046B
:102F8000B0912C0449E0B595A795979587954A95FA
:102F9000D1F7809343058091250490912604A09158
:102FA0002704B091280439E0B595A79597958795A2
:102FB0003A95D1F780934405809131049091320481
:102FC000A0913304B091340429E0B595A795979565
:102FD00087952A95D1F7809345058EE090E09F93E1
:102FE0008F938DE395E09F938F9381E08F938F93E1
:102FF00083E48F930E94D40F8091E3029091E402C6
:103000000E946F1990934C0580934B052DB73EB7E6
:10301000295F3F4F2DBF809105018F3F71F19927A7
:1030200004E0880F991F0A95E1F7815B9D4F40E10D
:1030300050E0BC01CE0101960E94DF8F80E190E05C
:103040009F938F93CE0101969F938F9381E090E0A1
:103050009F938F9385E091E09F938F9382E08F936E
:1030600081E08F9381E48F930E94D40F8FEF809340
:1030700005018DB79EB70B968DBF809120078823E1
:10308000D1F0809106018823B1F081E090E09F9318
:103090008F9380E297E09F938F9381E08F938F933C
:1030A00082E48F930E94D40F109220072DB73EB771
:1030B000295F3F4F2DBF8091F2028823C9F0809194
:1030C00006018823A9F084E390E09F938F9387EB18
:1030D00098E09F938F9381E08F938F9380E58F93F8
:1030E0000E94D40F1092F2028DB79EB707968DBF43
:1030F000E6E0C05F0C944C921F920F920FB60F92B5
:1031000011242F933F935F936F937F938F939F939C
:10311000AF93BF93EF93FF9320E080910703882341
:1031200029F0809107038150809307038091F60472
:10313000882319F081508093F60480910F03815009
:1031400080930F038F3F09F05BC089E080930F03EA
:1031500080910D0390910E03019690930E0380933E
:103160000D03809110018F5F81708093100188237F
:1031700019F481E080930C03349903C081E08093BB
:1031800010038091080390910903892B21F180910C
:103190000803909109030B9750F0809108039091D8
:1031A00009030A97909309038093080304C01092BF
:1031B000090310920803809108039091090320915C
:1031C000090130910A0182239323892B11F021E018
:1031D00008C020E006C08FEF9FEF90930A01809314
:1031E000090180910101222331F08A3011F45A9AA9
:1031F00007C0479A05C08A3011F45A9801C0479811
:1032000080911003882309F45AC02091970122234A
:1032100009F055C08091700983FF51C086B199278C
:10322000FC01E071F07084FF13C080910A0390915B
:103230000B03019690930B0380930A0380910A037A
:1032400090910B03895E9340D0F12093100337C017
:1032500080910A0390910B03892B69F180910A03F5
:1032600090910B038A56914030F580910A0390911A
:103270000B0369E270E00E94C09180910A03909173
:103280000B03860F971F90930B0380930A03809183
:103290000A0390910B030B9750F080910A039091D1
:1032A0000B030A97909389018093880104C0F093DF
:1032B0008901E093880110920B0310920A03FF9199
:1032C000EF91BF91AF919F918F917F916F915F919E
:1032D0003F912F910F900FBE0F901F901895209146
:1032E0000D0330910E03280F391FC901019608956F
:1032F00020910D0330910E03821B930B892F992788
:103300008695807490700895CF93DF930E946F1913
:10331000EC01CE010E9478198823D9F3DF91CF9177
:103320000895CF93DF930E946F19EC0109C080913B
:103330001101882329F0909311018FEC80937A007A
:10334000CE010E947819982F882389F3DF91CF91BD
:1033500008959FB7F8945F983E9A469A8091B0007E
:103360008F708093B0008091B00083608093B00034
:103370008091B1008B738093B1008091B1008B601C
:103380008093B1001092B2008FEF8093B3008091D0
:10339000B00080688093B000809170008A7F809335
:1033A0007000809170008260809370009FBF0895CC
:1033B0008AE090E00E946F19909322078093210782
:1033C00082E085BD83EA84BD17BC84EB88BD86E0BE
:1033D00086BD80916E00816080936E00089580911B
:1033E000F0072091670182FF30C09091B3078CE312
:1033F000989FB00111249091B20780E5989FA00199
:103400001124922F905897FD9D5F9595959586E094
:103410009802C00111242091070130910801281B56
:10342000390B3093080120930701421753072CF002
:10343000509308014093070108952617370784F039
:1034400070930801609307010895822F992736E051
:10345000880F991F3A95E1F790930801809307012F
:103460000895A0E0B0E0E7E3FAE10C942F92809198
:10347000BA07E82FFF27EE5BFE4F9681D080809140
:103480000F01A92FBB27A7FDB095CB2FDB2F8130D4
:1034900009F017C1209161043091620440916304E6
:1034A00050916404BD01CE010E94959197FF04C024
:1034B00061587F4F8F4F9F4F7B018C01C7E015955F
:1034C0000795F794E794CA95D1F78D2D992787FD35
:1034D0009095A92FB92F2091590430915A04409109
:1034E0005B0450915C04BC01CD010E94959197FF53
:1034F00004C061587F4F8F4F9F4FB7E095958795D8
:1035000077956795BA95D1F7F801E701C61BD70BF8
:10351000E80BF90B2091DB043091DC04C901A3E036
:10352000880F991FAA95E1F7821B930BAA2797FD95
:10353000A095BA2FC81BD90BEA0BFB0B8091B107E2
:103540009927AA27BB27BC01CD019E01AF010E948C
:10355000959197FF04C061507E4F8F4F9F4FFC01A4
:10356000EB0179E0F595E795D795C7957A95D1F771
:103570001091F007609107017091080112FF05C0DA
:1035800070930E0160930D0118C040910D01509190
:103590000E018091B907282F3327CB01841B950B8F
:1035A000B9010E94D49180910D0190910E01860F76
:1035B000971F90930E0180930D0110FF14C080910E
:1035C0000D0190910E0197FD0F9664E095958795FA
:1035D0006A95E1F7AA2797FDA095BA2FC80FD91FC2
:1035E000EA1FFB1F15C080910D0190910E0197FD00
:1035F0000F9654E0959587955A95E1F7AA2797FD80
:10360000A095BA2F8C1B9D0BAE0BBF0BFD01EC01DF
:103610002091ED07222321F133278091020390911D
:103620000303829FA001839F500D929F500D112490
:10363000CA01AA2797FDA095BA2F8C0F9D1FAE1F18
:10364000BF1F2F5F3F4F442737FD4095542FBC01CC
:10365000CD010E940992309303032093020304C01A
:10366000D0930303C09302038091B207282F33271E
:10367000220F331F220F331F809102039091030307
:10368000821793077CF08091B307282F3327220FEE
:10369000331F220F331F80910203909103032817D9
:1036A000390724F43093030320930203809101012E
:1036B000843108F4F7C080910F018F5F80930F0170
:1036C000F3C02091590430915A0440915B04509109
:1036D0005C04BD01CE010E94959197FF04C0615822
:1036E0007F4F8F4F9F4F7B018C0187E0159507958A
:1036F000F794E7948A95D1F78D2D992787FD9095BA
:10370000A92FB92F20916104309162044091630484
:1037100050916404BC01CD010E9495919B01AC01C4
:1037200097FF04C021583F4F4F4F5F4FC7E055955B
:10373000479537952795CA95D1F72E0D3F1D401F08
:10374000511F8091B5079927AA27BB27BC01CD013E
:103750000E94959197FF04C061507E4F8F4F9F4FFD
:10376000FC01EB01B9E0F595E795D795C795BA95BA
:10377000D1F7809166019927A6E0880F991FAA9535
:10378000E1F740910B0150910C012091B9073327CB
:10379000841B950BB9010E94D49180910B019091EB
:1037A0000C01860F971F90930C0180930B01809161
:1037B000F00781FF14C080910B0190910C0197FDDF
:1037C0000F9674E0959587957A95E1F7AA2797FD6E
:1037D000A095BA2FC80FD91FEA1FFB1F15C08091F3
:1037E0000B0190910C0197FD0F9664E095958795DC
:1037F0006A95E1F7AA2797FDA095BA2F8C1B9D0B20
:10380000AE0BBF0BFD01EC012091EE07222321F14D
:1038100033278091000390910103829FA001839F31
:10382000500D929F500D1124CA01AA2797FDA09513
:10383000BA2F8C0F9D1FAE1FBF1F2F5F3F4F442716
:1038400037FD4095542FBC01CD010E940992309361
:1038500001032093000304C0D0930103C09300032D
:103860008091B607282F3327220F331F220F331FD3
:103870008091000390910103821793077CF080915F
:10388000B707282F3327220F331F220F331F8091B2
:103890000003909101032817390724F430930103A2
:1038A0002093000310920F01E7E0CDB7DEB70C9430
:1038B0004B921F920F920FB60F9211242F933F93AA
:1038C0004F935F938F939F93EF93FF9380910101A9
:1038D00090911103843108F04CC0992309F029C15B
:1038E0008091B00086FF24C08091B0008F7B8093D0
:1038F000B000809102039091030387559E4F9093EF
:1039000005038093040325E08D3D920718F08CEDAC
:1039100095E005C08757914030F487E791E0909398
:103920000503809304038091040390910503C2C0B2
:103930008091B00080648093B0008091B807282FF8
:1039400033278DED96E0289FA001299F500D389FC9
:10395000500D1124CA012091120330911303821BD0
:10396000930B909305038093040381E080930F01F0
:10397000DDC0992309F0DDC08091B00086FF9FC0B3
:103980008091B0008F7B8093B000E0911403209170
:10399000B807EE23D9F433278DED96E0289FA001D8
:1039A000299F500D389F500D1124CA0120911203F8
:1039B00030911303821B930B9093050380930403B0
:1039C0001092130310921203469AB0C02E1738F4C7
:1039D0008AE090E09093050380930403A7C089EAEE
:1039E00093E090930503809304038E2F99278330EF
:1039F0009105D9F08430910534F48130910549F076
:103A0000029761F020C08430910591F0059799F0FC
:103A10001AC0809102039091030304C080910003B7
:103A20009091010387559E4F1DC080914C0905C0A0
:103A30008091250902C0809155099927880F991F07
:103A4000880F991FEFCFFF27EE0FFF1FE954F74FA5
:103A500020813181220F331F80910403909105034F
:103A6000820F931F909305038093040380910403B6
:103A70009091050355E08D3D950718F08CED95E08C
:103A800005C08757914030F487E791E09093050394
:103A90008093040320910403309105032C5B304094
:103AA0003093050320930403809112039091130334
:103AB000820F931F909313038093120337C080915A
:103AC000B00080648093B0008CEB90E0909305038D
:103AD00080930403809112039091130384549F4FA9
:103AE000909313038093120380910603882321F09F
:103AF00080910704882321F480910603823011F419
:103B0000469801C0469A809114038F5F80931403F6
:103B1000282F33278091B80799270196821793079A
:103B20002CF481E080930F011092140381E08093C4
:103B30001103209104033091050341E02F3734072E
:103B400030F08FEF8093B3002F5F30400FC02F3FD6
:103B50003105C9F0C0F0A9014F5F50404F37510502
:103B600050F480E88093B300205830403093050330
:103B70002093040312C08FEF8093B300509305038A
:103B8000409304030AC0809104038093B300109211
:103B900005031092040310921103FF91EF919F917E
:103BA0008F915F914F913F912F910F900FBE0F908A
:103BB0001F90189510927C008FEC80937A000895E6
:103BC000CF93DF931092190386E987BD83E090E0DD
:103BD0000E94E72EC82F863E08F4C65FC8BD84E663
:103BE00090E00E94911980911501909116018152E7
:103BF000934010F0C0EF02C0C530F8F0C8BD82E3BA
:103C000090E00E94911984E694E09F938F9380E660
:103C100095E19F938F93E0913B05F0913C050995C9
:103C200080911501909116010F900F900F900F90B9
:103C30008152934010F4C550DFCF6C2F83E090E0A9
:103C40000E94EF2ECF3018F0CCE8D0E002C0C0E0E8
:103C5000D0E0CA3FD105F8F4C7BD82E390E00E94EE
:103C6000911986E694E09F938F9380E695E19F9368
:103C70008F93E0913B05F0913C05099580911501EA
:103C8000909116010F900F900F900F9080529340DB
:103C900010F02196DECFC0932F078091900780FF10
:103CA00009C08C2F8A508B3E28F080915405806487
:103CB00080935405C7BD8CE291E00E949119DF9179
:103CC000CF910895EF92FF921F93CF9310E080ED74
:103CD00097E00E946F197C01CCE8133019F4CB30C7
:103CE00008F0C9E010E080912803909129038C5FCF
:103CF000934024F48091140181500AC080912803DC
:103D0000909129038750944034F0809114018F5F83
:103D10008093140101C011E0809126039091270344
:103D20008C5F934024F48091130181500AC08091EC
:103D30002603909127038750944034F0809113011B
:103D40008F5F8093130101C01F5F809124039091C6
:103D500025038C5F934024F48091120181500AC0A6
:103D6000809124039091250387509440C4F0809162
:103D700012018F5F8093120113C088E694E09F9335
:103D80008F9380E695E19F938F93E0913B05F091AF
:103D90003C0509950F900F900F900F905FC01F5F2B
:103DA00082E18093530380914D038E7F80934D0376
:103DB00085EA8093BC00809114018A3040F48091A0
:103DC00054058160809354058AE0809314018091AA
:103DD0001401863F40F08091540581608093540522
:103DE00085EF80931401809113018A3040F4809113
:103DF00054058260809354058AE08093130180917A
:103E00001301863F40F080915405826080935405F1
:103E100085EF80931301809112018A3040F48091E4
:103E200054058460809354058AE080931201809148
:103E30001201863F40F080915405846080935405C0
:103E400085EF8093120180915303882339F0C701D5
:103E50000E947819882309F090CFF5CF10921101B4
:103E60008FEC80937A00809111018823E1F3CA30AE
:103E700020F48AE090E00E949119C15009F02DCF02
:103E800086E490E00E949119CF911F91FF90EF90EE
:103E900008951F920F920FB60F921124EF92FF9286
:103EA0000F931F932F933F934F935F936F937F9342
:103EB0008F939F93AF93BF93EF93FF9380913103C1
:103EC000282F3327442755278F5F80933103F9012B
:103ED0002231310508F0E3C3EA5BFF4F0C945B929B
:103EE000809178009091790046C0809178009091FF
:103EF000790047C1809178009091790090933403C4
:103F00008093330372C180916A0490916B04209175
:103F1000780030917900821B930B90932407809353
:103F20002307809123079091240790933E03809369
:103F30003D0379C1809178009091790020916C04C3
:103F400030916D04821B930B90932E0780932D0765
:103F500080912D0790912E079093400380933F030B
:103F6000A0C380913703909138032091780030915D
:103F70007900820F931F909338038093370381E079
:103F800091C3809135039091360320917800309150
:103F90007900820F931F909336038093350384E05A
:103FA00081C38091F10783FF1AC080911F01909116
:103FB00020019C01220F331F280F391F40917800E8
:103FC000509179008BE090E0489FB001499F700DBF
:103FD000589F700D1124CB016EE170E00FC08091ED
:103FE0001F01909120019C01220F331F280F391FC0
:103FF000809178009091790063E070E00E94C09118
:10400000260F371F36952795369527953093200133
:1040100020931F0185E046C380917800909179003C
:104020004091660450916704841B950B90931F0385
:1040300080931E0380911E0390911F03029704F149
:1040400072E04E3E570784F4209132032B5F209399
:10405000320325508091D0039091D103845F914029
:1040600018F4215F2093320380913203853684F166
:104070004F5F5F4F5093670440936604845626C099
:1040800080911E0390911F038F5F9F4F0CF572E08C
:1040900047325707ECF0209132032550209332032A
:1040A0002B5F8091D0039091D103845F914018F4ED
:1040B0002F5020933203809132038C394CF44150BD
:1040C000504050936704409366048C5980933203A8
:1040D000809178009091790090932607809325072E
:1040E00080911E0390911F039C01442737FD40954A
:1040F000542F8091210490912204A0912304B09127
:104100002404820F931FA41FB51F80932104909352
:104110002204A0932304B09324042091210430911D
:104120002204409123045091240457FF04C02150DD
:104130003C4F4F4F5F4F6AE0559547953795279510
:104140006A95D1F78091210490912204A0912304D3
:10415000B0912404821B930BA40BB50B8093210414
:1041600090932204A0932304B09324042EC1809141
:104170003503909136032091780030917900820FB9
:10418000931F9093360380933503109230038CC2B3
:10419000809101018A3071F48091780090917900CA
:1041A0002091330330913403820F931F019696952B
:1041B000879517C04091330350913403843158F0F0
:1041C0002091780030917900240F351F8FEF97E010
:1041D000821B930B06C08091780090917900840F28
:1041E000951F909325038093240386E05BC2809102
:1041F0006A0490916B042091780030917900821BC1
:10420000930B909324078093230780912307909129
:10421000240720913D0330913E03820F931F90931A
:1042200023038093220387E03DC280917800909120
:10423000790020916C0430916D04821B930B909354
:104240002E0780932D0780912D0790912E072091A6
:104250003F0330914003820F931F9093210380937B
:1042600020031FC2209137033091380380917800DA
:1042700090917900280F391F30933803209337032A
:10428000809101018A3019F4220F331F04C0220FDC
:10429000331F220F331F30933803209337032091AD
:1042A000370330913803C90137FD079603E0959530
:1042B00087950A95E1F790932903809328038091CD
:1042C000390390913A03820F931F97FD01969595BC
:1042D000879590933A038093390320917604309127
:1042E0007704821B930B90931E0180931D012091F4
:1042F0002E0330912F0380911D0190911E01280FF4
:10430000391F37FF02C02F5F3F4F359527953093F8
:104310002F0320932E0333CE2091350330913603A3
:104320008091780090917900280F391F30933603DF
:1043300020933503809101018A3019F4220F331F35
:1043400004C0220F331F220F331F309336032093F4
:1043500035032091350330913603C90137FD0796A7
:10436000F3E095958795FA95E1F79093270380936D
:10437000260380913B0390913C03820F931F97FD8E
:1043800001969595879590933C0380933B032091EC
:10439000740430917504821B930B90931C018093DD
:1043A0001B0120912C0330912D0380911B019091D2
:1043B0001C01280F391F37FF02C02F5F3F4F359573
:1043C000279530932D0320932C0383E06BC110922B
:1043D000310381E0809311018091150390911603C0
:1043E0000196909316038093150380917800909125
:1043F0007900909316018093150180911501909199
:104400001601AA27BB272091410330914203409116
:10441000430350914403280F391F4A1F5B1F209309
:1044200041033093420340934303509344038091EC
:1044300045038F5F80934503803108F432C180913A
:10444000170190911801A0911901B0911A017C01F6
:104450008D0163E0EE0CFF1C001F111F6A95D1F760
:10446000E81AF90A0A0B1B0BE20EF31E041F151FB4
:1044700080911903992787FD9095A92FB92FBC0129
:10448000CD0120EB30E240E050E00E949591DC014C
:10449000CB01E81AF90A0A0B1B0BD801C7010496D5
:1044A000A11DB11DB7FF05C0D801C7010B96A11D05
:1044B000B11D23E0B595A795979587952A95D1F7D6
:1044C0008093170190931801A0931901B0931A01DA
:1044D00080912707909128077C010027F7FC009521
:1044E000102F8091170190911801A0911901B0919E
:1044F0001A01E81AF90A0A0B1B0BE0920104F09268
:104500000204009303041093040420911A033091D1
:104510001B0340911C0350911D0357FF04C0215FF2
:104520003F4F4F4F5F4F84E05595479537952795FF
:104530008A95D1F780911A0390911B03A0911C03D7
:10454000B0911D03821B930BA40BB50B80931A0330
:1045500090931B03A0931C03B0931D0380911A0337
:1045600090911B03A0911C03B0911D038E0D9F1D04
:10457000A01FB11F80931A0390931B03A0931C03E9
:10458000B0931D0380911A0390911B03A0911C030B
:10459000B0911D03B7FF03C00F96A11DB11D14E01C
:1045A000B595A795979587951A95D1F72091010410
:1045B00030910204281B390B64E0213036071CF0CF
:1045C00020E034E006C07CEF2030370714F420E010
:1045D0003CEF8091170390911803809117039091FD
:1045E000180397FF03C0909581959F4FA901F3E0B1
:1045F000440F551FFA95E1F78D5B9240C4F080910E
:104600001703909118039C01E4E0220F331FEA95F1
:10461000E1F7281B390B240F351F37FF02C0215F3C
:104620003F4F74E0359527957A95E1F717C0809153
:104630001703909118039C0165E0220F331F6A95C0
:10464000E1F7281B390B240F351F37FF02C0215E0D
:104650003F4F45E0359527954A95E1F7309318038C
:10466000209317038091410390914203A09143034B
:10467000B0914403B7FF03C00196A11DB11DB595CC
:10468000A795979587958093410390934203A093B4
:104690004303B093440388E08093450302C0109223
:1046A000310382E0809330038091300380937C005B
:1046B00080913103882319F08FEC80937A00FF9169
:1046C000EF91BF91AF919F918F917F916F915F918A
:1046D0004F913F912F911F910F91FF90EF900F906D
:1046E0000FBE0F901F90189590E2E2E3F7E08FE481
:1046F0009193815087FFFCCF0895909148039035A6
:1047000040F4E92FFF27EE5CF84F80839F5F909382
:1047100048030895AF92BF92CF92DF92FF920F931A
:104720001F93CF93DF932091460320FF0AC080910F
:104730004703882311F0815002C0809121018093AA
:10474000470321FF0CC090914703809121019817E6
:1047500019F41092470303C09F5F90934703822F81
:10476000992780FF04C081FF02C0109247030E9476
:10477000742380914703282F33279DE7C92E93E2A6
:10478000D92EC0913B05D0913C058A3098F481E147
:10479000809348033F932F938FE994E09F938F93E7
:1047A000DF92CF92FE0109952DB73EB72A5F3F4FAA
:1047B0002DBF11C080E1809348033F932F9384EA7B
:1047C00094E09F938F93DF92CF92FE0109958DB76E
:1047D0009EB706968DBF20914703822F9927AA275F
:1047E000BB27FC01419710F00C94E22CE85AFF4FD4
:1047F0000DE7C02E03E2D02EC0913B05D0913C05C1
:104800000C945B921092480389EA94E09F938F93F3
:104810000DE713E2DF92CF92FE01099584E18093C8
:1048200048030F900F900F900F9084E690E09F93B5
:104830008F938AE590E09F938F931F921F928091B0
:1048400001016AE00E94B491892F99279F938F9369
:10485000809101010E94B49199279F938F9389EBD6
:1048600094E09F938F93DF92CF92E0913B05F0917C
:104870003C05099588E280934803EDB7FEB73E9664
:10488000EDBF81E098E09F938F930E94633099275A
:104890009F938F9381ED94E09F938F93DF92CF92BC
:1048A000E0913B05F0913C050995809155059927CC
:1048B0002DB73EB7285F3F4F2DBFEC01C071D070C0
:1048C00084FF06C08CE3809348038FED94E0F1C031
:1048D0009091E204992349F18CE380934803892F56
:1048E00099279F938F938CEE94E09F938F931F93C0
:1048F0000F93E0913B05F0913C050995DF93CF9331
:104900009091E20481E1989FC0011124825C954F4F
:104910009F938F931F930F93E0913B05F0913C057C
:1049200009958DB79EB70C9647C190915405992370
:10493000B1F08CE380934803892F99279F938F933D
:1049400084EF94E09F938F931F930F93E0913B0527
:10495000F0913C050995EDB7FEB7369679C4909174
:104960004E03992371F08CE380934803892F992794
:104970009F938F938BE095E09F938F931F930F935B
:10498000D9C48091360190913701069710F00C94AC
:10499000EB2C8CE38093480380E295E0A5C78091DF
:1049A00070091DE7C12E13E2D12EC0913B05D091B5
:1049B0003C0580FF6BC010924803809101049091E8
:1049C0000204A0910304B0910404BC01CD0125E0D0
:1049D00030E040E050E00E9409923F932F938DE237
:1049E00095E09F938F93DF92CF92FE01099584E12A
:1049F000809348038DB79EB706968DBF8091FD03C7
:104A00009091FE03A091FF03B0910004BC01CD0181
:104A100025E030E040E050E00E9409923F932F9360
:104A20008AE395E09F938F93DF92CF92E0913B05CD
:104A3000F0913C05099588E280934803EDB7FEB7F5
:104A40003696EDBF80911501909116019F938F933B
:104A500087E495E09F938F93DF92CF92E0913B059F
:104A6000F0913C0509958CE3809348032DB73EB740
:104A70002A5F3F4F2DBF87B599279F938F9384E57A
:104A800095E09F938F93DF92CF928EC01092480350
:104A900081E695E09F938F93DF92CF92FE01099577
:104AA00084E1809348030F900F900F900F9080E760
:104AB00095E09F938F93DF92CF921AC7109248038D
:104AC00089E795E09F938F930DE713E2DF92CF92F2
:104AD000FE01099584E1809348030F900F900F9099
:104AE0000F908091610490916204A0916304B09151
:104AF0006404B7FF04C081509C4FAF4FBF4FCAE062
:104B0000B595A79597958795CA95D1F7BF93AF931C
:104B10009F938F9386E895E09F938F931F930F93B6
:104B2000E0913B05F0913C05099588E280934803AC
:104B3000EDB7FEB73896EDBF8091590490915A04B5
:104B4000A0915B04B0915C04B7FF04C081509C4FFE
:104B5000AF4FBF4FFAE0B595A79597958795FA9512
:104B6000D1F7BF93AF939F938F9385E995E09F9380
:104B70008F931F930F93E0913B05F0913C050995AE
:104B80008CE3809348032DB73EB7285F3F4F2DBF7E
:104B900080912D0990912E099F938F9384EA95E03F
:104BA0009F938F931F930F93E0913B05F0913C05EA
:104BB00009958DB79EB706968DBF0DC7E1E0FE2E15
:104BC000C1E0D0E009EB18E09F2D969584E1989F15
:104BD000C001112480934803F801828193819F933F
:104BE0008F932196DF93CF932197808191819F931B
:104BF0008F93DF93CF9383EB95E09F938F938DE714
:104C000093E29F938F93E0913B05F0913C050995CA
:104C10002DB73EB7245F3F4F2DBF32E0F30E2296F3
:104C20000C5F1F4F88E08F1578F6D5C610924803A9
:104C300080918507E82FFF27EE0FFF1FE954F74FFC
:104C4000808191819F938F9380918407E82FFF2724
:104C5000EE0FFF1FE954F74F808191819F938F934F
:104C600085EC95E09F938F93DF92CF92FE0109959B
:104C700084E180934803EDB7FEB73896EDBF80918D
:104C80008707E82FFF27EE0FFF1FE954F74F8081BA
:104C900091819F938F9380918607E82FFF27EE0FD6
:104CA000FF1FE954F74F8081918181589F4F9F9357
:104CB0008F9385ED95E09F938F93DF92CF92E09154
:104CC0003B05F0913C05099588E2809348032DB798
:104CD0003EB7285F3F4F2DBF80918907E82FFF2700
:104CE000EE0FFF1FE954F74F8081918181589F4F4C
:104CF0009F938F9380918807E82FFF27EE0FFF1F68
:104D0000E954F74F8081918181589F4F9F938F93F2
:104D100085EE95E09F938F93DF92CF92E0913B05D4
:104D2000F0913C0509958CE3809348038DB79EB7BD
:104D300008968DBF80918B07E82FFF27EE0FFF1F8E
:104D4000E954F74F8081918181589F4F9F938F93B2
:104D500080918A07E82FFF27EE0FFF1FE954F74FD6
:104D60008081918181589F4F9F938F9385EF95E02C
:104D700063C21092480385E096E09F938F930DE7FE
:104D800013E2DF92CF92FE010995809101010F900D
:104D90000F900F900F908A3009F09DC084E18093AE
:104DA000480380917604909177049C0197FF02C09C
:104DB000295F3F4F287F821B930B9F938F93809196
:104DC00076049091770497FD079673E09595879503
:104DD0007A95E1F79F938F93209176043091770431
:104DE00037FF02C0295F3F4F63E0359527956A95ED
:104DF000E1F78091280390912903821B930B9F93E5
:104E00008F9383E196E09F938F931F930F93E0918D
:104E10003B05F0913C05099588E2809348032DB746
:104E20003EB7265F3F4F2DBF80917404909175046B
:104E30009C0197FF02C0295F3F4F287F821B930B85
:104E40009F938F93809174049091750497FD0796BA
:104E500053E0959587955A95E1F79F938F9320910D
:104E600074043091750437FF02C0295F3F4F43E05F
:104E7000359527954A95E1F7809126039091270370
:104E8000821B930B9F938F9384E296E09F938F9363
:104E90001F930F93E0913B05F0913C0509958CE33E
:104EA000809348038DB79EB70A968DBF8091720498
:104EB000909173049F938F938091720490917304E7
:104EC0002091240330912503821B930B9F938F9392
:104ED00085E396E0ADC08B3019F0843108F4ADC0A5
:104EE00084E18093480380917604909177049C013B
:104EF00097FF02C0215F3F4F207F821B930B97FDDE
:104F00000196959587959F938F93809176049091C4
:104F1000770497FD0F9624E0959587952A95E1F7FC
:104F20009F938F93209176043091770437FF02C0CE
:104F3000295F3F4FC3E035952795CA95E1F78091EA
:104F4000280390912903821B930B9F938F9383E4F3
:104F500096E09F938F931F930F93E0913B05F09101
:104F60003C05099588E2809348032DB73EB7265F3C
:104F70003F4F2DBF80917404909175049C0197FF61
:104F800002C0215F3F4F207F821B930B97FD01964C
:104F9000959587959F938F93809174049091750454
:104FA00097FD0F96A4E095958795AA95E1F79F93B5
:104FB0008F93209174043091750437FF02C0295FEC
:104FC0003F4FF3E035952795FA95E1F78091260359
:104FD00090912703821B930B9F938F9385E596E017
:104FE0009F938F931F930F93E0913B05F0913C05A6
:104FF00009958CE3809348038DB79EB70A968DBFC1
:10500000809172049091730497FD01969595879510
:105010009F938F9380917204909173042091240345
:1050200030912503821B930B9F938F9387E696E025
:105030009F938F931F930F9303C18D3009F0CBC4BF
:1050400084E1809348038091140199279F938F9363
:10505000809176049091770497FD0F9674E0959572
:1050600087957A95E1F79F938F93209176043091FD
:10507000770437FF02C0295F3F4F63E035952795DE
:105080006A95E1F78091280390912903821B930B85
:105090009F938F9386E796E09F938F931F930F9331
:1050A000E0913B05F0913C05099588E28093480327
:1050B0002DB73EB7265F3F4F2DBF80911301992733
:1050C0009F938F93809174049091750497FD0F9630
:1050D00054E0959587955A95E1F79F938F9320918A
:1050E00074043091750437FF02C0295F3F4F43E0DD
:1050F000359527954A95E1F78091260390912703EE
:10510000821B930B9F938F938AE896E09F938F93D4
:105110001F930F93E0913B05F0913C0509958CE3BB
:10512000809348038DB79EB70A968DBF8091120178
:1051300099279F938F93809172049091730497FDA8
:105140000196959587959F938F9380917204909186
:1051500073042091240330912503821B930B9F93AA
:105160008F938EE996E09F938F931F930F93E09117
:105170003B05F0913C050995EDB7FEB73A9668C03E
:105180001092480382EB96E09F938F93DF92CF9229
:10519000FE01099584E1809348030F900F900F90D2
:1051A0000F9080916C0490916D049F938F938091E8
:1051B0002003909121039F938F938FEB96E09F9311
:1051C0008F93DF92CF92E0913B05F0913C050995DA
:1051D00088E2809348032DB73EB7285F3F4F2DBF2D
:1051E00080916A0490916B049F938F938091220326
:1051F000909123039F938F938EEC96E09F938F93D0
:10520000DF92CF92E0913B05F0913C0509958CE34C
:10521000809348038DB79EB708968DBF8091660432
:10522000909167049F938F9380911E0390911F0329
:105230009F938F938DED96E09F938F93DF92CF9204
:10524000E0913B05F0913C050995EDB7FEB7389626
:10525000EDBFC1C31092480380911F0190912001BE
:105260006AE070E00E94D4919F938F9380911F0118
:10527000909120016AE070E00E94D4917F936F9337
:105280008CEE96E09F938F93DF92CF92FE0109956B
:1052900084E1809348032DB73EB7285F3F4F2DBF71
:1052A0008091100A9091110A6AE070E00E94C0910A
:1052B0009F938F938091100A9091110A6AE070E099
:1052C0000E94C0917F936F9380E097E09F938F93AC
:1052D000DF92CF92E0913B05F0913C05099588E281
:1052E000809348038DB79EB708968DBF8091120AB0
:1052F0009091130A9F938F9384E197E09F938F93EC
:10530000DF92CF92E0913B05F0913C0509958CE34B
:1053100080934803EDB7FEB73696EDBF8091140A2F
:105320009091150A9F938F9384E297E09F938F93B8
:10533000DF92CF92E0913B05F0913C0509952DB7A6
:105340003EB72A5F3F4F4FC11092480386E397E074
:105350009F938F93DF92CF92FE01099584E1809312
:1053600048030F900F900F900F908091B708909185
:10537000B8089F938F938FE397E09F938F93DF926B
:10538000CF92E0913B05F0913C05099588E280932E
:1053900048038DB79EB706968DBF80910704992765
:1053A0009F938F938FE497E09F938F93DF92CF9299
:1053B000E0913B05F0913C0509958CE3809348030F
:1053C000EDB7FEB73696EDBF8091B60899270197E5
:1053D0009F938F938FE597E0A9CF109248038FE6B4
:1053E00097E09F938F93DF92CF92FE01099584E11E
:1053F000809348030F900F900F900F908091880139
:10540000909189019F938F9387E797E09F938F9364
:10541000DF92CF92E0913B05F0913C05099588E23F
:10542000809348038DB79EB706968DBF80912D0956
:1054300090912E099F938F9385E897E09F938F9388
:10544000DF92CF92E0913B05F0913C0509958CE30A
:1054500080934803EDB7FEB73696EDBF80911F04E9
:10546000909120049F938F9383E997E05FCFC8E0EA
:10547000CC2EC4E0DC2E20E030E0E901B3E0FB2ECE
:10548000C0934803F60181916F0199279F938F93F1
:1054900089010F5F1F4F1F930F9381EA97E09F933E
:1054A0008F938DE793E29F938F93E0913B05F0916B
:1054B0003C0509952DB73EB7285F3F4F2DBFFA94A5
:1054C00064969801F7FEDCCF86C2ACE0CA2EA4E059
:1054D000DA2EC0E0D0E08E01F3E0FF2E0093480307
:1054E000F60181916F0199279F938F932596DF9302
:1054F000CF938EEA97E09F938F938DE793E29F93EC
:105500008F93E0913B05F0913C0509952DB73EB78F
:10551000285F3F4F2DBFFA940C5E1F4F2497F7FE74
:10552000DDCF59C2109248038BEB97E09F938F9386
:105530000DE713E2DF92CF92FE01099584E180939B
:1055400048030F900F900F900F908091670199275B
:105550009F938F9383EC97E09F938F93DF92CF92EB
:10556000E0913B05F0913C05099588E28093480362
:105570008DB79EB706968DBF80910203909103036D
:1055800097FD039695958795959587959F938F930E
:1055900081ED97E09F938F931F930F93E0913B05CD
:1055A000F0913C0509958CE380934803EDB7FEB775
:1055B0003696EDBF8091B30799279F938F93809183
:1055C000B20799279F938F938FED97E09F938F93C7
:1055D0001F930F93E0913B05F0913C0509952DB782
:1055E0003EB7285F3F4F2DBFF6C1109248038DEEA6
:1055F00097E09F938F937DE7A72E73E2B72EDF92FC
:10560000CF92FE0109950F900F900F900F90C6E575
:10561000D8E000E010E062E0F62E802F8C5E8093F0
:1056200048038B8D99278F7790709F938F938B89E9
:1056300099278F7790709F938F938B8599278F777A
:1056400090709F938F938B8199278F7790709F9302
:105650008F938DEF97E09F938F93BF92AF92E091DE
:105660003B05F0913C0509958DB79EB70C968DBF13
:10567000FA940C5E1F4FA096F7FECFCFACC11092EC
:1056800048038EE098E09F938F935DE7A52E53E249
:10569000B52EDF92CF92FE0109950F900F900F90DB
:1056A0000F90C6E5D8E000E010E042E0F42E802F35
:1056B0008C5E809348038F8D992787FD90959F93EB
:1056C0008F938F89992787FD90959F938F938F85CF
:1056D000992787FD90959F938F938F81992787FDB9
:1056E00090959F938F938DE198E09F938F93BF92B6
:1056F000AF92E0913B05F0913C050995EDB7FEB7FF
:105700003C96EDBFFA940C5E1F4FA096F7FECFCFEC
:1057100062C1109248038EE298E09F938F930DE749
:1057200013E2DF92CF92FE01099584E18093480352
:105730000F900F900F900F9080917108881F88270D
:10574000881F97E0899FC00111248D969F938F93A6
:1057500080916908881F8827881F96E0899FC0016B
:1057600011248D969F938F9380916108881F8827BD
:10577000881F95E0899FC00111248D969F938F9378
:1057800080915908881F8827881F9927880F991F9B
:10579000880F991F8D969F938F938DE398E09F9329
:1057A0008F93DF92CF92E0913B05F0913C050995F4
:1057B00088E2809348032DB73EB7245F3F4F2DBF4B
:1057C00080919108881F8827881F9BE0899FC001CE
:1057D00011248D969F938F9380918908881F882725
:1057E000881F9AE0899FC00111248D969F938F9303
:1057F00080918108881F8827881F99E0899FC001B0
:1058000011248D969F938F9380917908881F882704
:10581000881F992723E0880F991F2A95E1F78D9615
:105820009F938F9381E598E09F938F93DF92CF9220
:10583000E0913B05F0913C0509958CE3809348038A
:105840008DB79EB70C968DBF80919908881F8827C9
:10585000881F9CE0899FC00111248D969F938F9390
:1058600085E698E09F938F93DF92CF92E0913B057E
:10587000F0913C0509958091A108EDB7FEB73696E9
:10588000EDBF87FF12C080E48093480386E798E06D
:105890009F938F93DF92CF92E0913B05F0913C056F
:1058A00009950F900F900F900F908091A90887FF96
:1058B00012C084E48093480389E798E09F938F9314
:1058C0001F930F93E0913B05F0913C0509950F90D4
:1058D0000F900F900F908091B10887FF7CC088E4F3
:1058E000809348038CE798E09F938F931F930F93C7
:1058F000E0913B05F0913C0509950F900F900F90BA
:105900000F9069C0109248038FE798E09F938F93A0
:10591000DF92CF92FE01099584E1809348030F90B6
:105920000F900F900F908091D8029091D9029F9381
:105930008F938DE898E09F938F93DF92CF92E091C1
:105940003B05F0913C05099588E2809348032DB70B
:105950003EB72A5F3F4F2DBF8091DA029091DB0264
:105960009F938F938AE998E09F938F93DF92CF92D2
:10597000E0913B05F0913C05099589E4809348034B
:105980008DB79EB706968DBF87EA98E09F938F9359
:10599000DF92CF92E0913B05F0913C050995809113
:1059A00046030F900F900F900F9083FF14C010923A
:1059B000DB021092DA0260E070E08EE090E00E947C
:1059C000002F09C080912101281719F4215020933C
:1059D00021011092470310924603DF91CF911F914E
:1059E0000F91FF90DF90CF90BF90AF900895F999FD
:1059F000FECF92BD81BDF89A80B599270895F99997
:105A0000FECF1FBA92BD81BD60BD0FB6F894FA9A61
:105A1000F99A0FBE08954AEA20E030E026173707CA
:105A200040F4FC018191480F2F5F3F4F2617370745
:105A3000C8F3842F99270895EAEA40E050E046171A
:105A4000570778F49C01F999FECF32BD21BDF89A31
:105A500080B5E80F4F5F5F4F2F5F3F4F46175707E7
:105A600090F38E2F9927089581E08093860782E036
:105A70008093850783E08093840784E08093870781
:105A800085E08093880786E08093890787E080938C
:105A90008A0788E080938B0789E080938C078AE0EF
:105AA00080938D078BE080938E078CE080938F0727
:105AB00008958CE5809383078CE0E3EFF7E0119283
:105AC0008A95E9F780910101843150F08AE0809352
:105AD000A3071092C7078BE180939F078EE40AC04B
:105AE00083E08093A30780E28093C7078EE18093D1
:105AF0009F0785E58093C4078093C50780E2809364
:105B0000C6071092EF078AE68093900782E280939F
:105B1000F10780E48093F20766E06093AA07109291
:105B2000E7071092E40748E040939D0756EE509334
:105B30009E078093A0079EE1909391078FEF80933B
:105B400093072FE020939407909392071092960763
:105B50004093970784E180939807109299072093C8
:105B600095071092AC071092AD071092AE071092F5
:105B7000AF071092C9071092CA071092CB07109274
:105B8000CC0790E89093B00732E33093B10782E0FE
:105B90008093F0072093B2075093B30784E080937B
:105BA000B8078DE78093BB078093BC078093BD0740
:105BB0009093B40725E52093B50786E48093B60754
:105BC0008CED8093B7078CE38093B9071092BA07E6
:105BD0008FE58093CD0783EF8093CF078AEA809388
:105BE000D1078093D20788E28093CE078093D007B5
:105BF0001092D3073093BE079AE59093BF07309376
:105C0000C0078EEF8093D40784E68093D5079093E6
:105C1000D6079093D7079093D8078BE48093D90742
:105C20002093DA078093DB071092DC076093DD078F
:105C30004093DE079093DF078AE28093E00785EFC9
:105C40008093E1078CE88093E20785E08093E30787
:105C50001092E5071092E60781E28093A70781E49E
:105C60008093A8079093A9071092E8071092E9077C
:105C70001092EA0786E98093EB079093C10787E3C8
:105C80008093C2071092EC071092ED071092EE0776
:105C900008950E94592D8AE080939A0780E18093AD
:105CA0009B0726E020939C079AE59093A10788E73D
:105CB0008093A2079093A4078093A5072093A6073B
:105CC00080E28093AB078CE38093C3078BE48093DF
:105CD000C80786E491E6A3E7B4E78093F3079093BF
:105CE000F407A093F507B093F6076CE770E083E83C
:105CF00097E00E940B2D8093FF070895CF93DF93C9
:105D00000E94592D88E080939A0730E130939B07D9
:105D100026E020939C0794E69093A10788E7809360
:105D2000A2079093A4078093A5072093A60730931A
:105D3000AB0786E48093C3078093C807A3EFB7E05F
:105D4000E2E2F1E0ED01019009922A95E1F76CE7BA
:105D500070E0CD01805790400E940B2D8093FF078B
:105D6000DF91CF9108950E94592D26E020939A0744
:105D70008AE080939B0784E080939C0794E690934D
:105D8000A10788E78093A2079093A4078093A507B3
:105D90002093A60780E18093AB0786E48093C30736
:105DA0008093C80785E491E6A3E7B9E78093F307FA
:105DB0009093F407A093F507B093F6076CE770E0B3
:105DC00083E897E00E940B2D8093FF070895F999CF
:105DD000FECF92BD81BDF89A80B599270895F999B3
:105DE000FECF1FBA92BD81BD60BD0FB6F894FA9A7E
:105DF000F99A0FBE089567EF7CE20E942390089500
:105E00004FEF5CE20E945D900895EF92FF920F9336
:105E10001F93CF93C82F8150853008F0C3E08DE7E2
:105E2000C89F8001112487EEE82E8FEFF82EE00E38
:105E3000F11E6CE770E0C7010E941C2D682F9801CD
:105E40002D593F4F8FB39927AC014270507081FD9F
:105E5000F9CF32BD21BDF89A80B5861711F0CA017D
:105E600023C08FB399279C012270307081FDF9CF38
:105E7000F2BCE1BCF89A80B58C3511F0C90114C0B0
:105E80008DE7C89FC0011124499727EF3CE24DE7F9
:105E900050E0BC0183E897E00E94FE8F0E94D26D23
:105EA0000E94DB8B81E090E0CF911F910F91FF90DA
:105EB000EF900895282F863010F025E003C0882346
:105EC00009F421E0F999FECF1FBA82E090E092BD7B
:105ED00081BD20BD0FB6F894FA9AF99A0FBE0895C5
:105EE000CF93C82F809183078C3509F051C0C630FD
:105EF00010F0C5E003C0CC2309F44AC00E94E78E2D
:105F00008091F20782FF07C08091A807843618F0BD
:105F100080E58093A8076CE770E083E897E00E9433
:105F20000B2D8093FF078DE7C89FC00111242FEF31
:105F30003CE24DE750E063E877E049970E943B90F0
:105F40002FEF3CE24CE050E064E877E080E590E041
:105F50000E943B906CE070E084E897E00E940B2D7B
:105F6000282FF999FECF1FBA8CE590E092BD81BD34
:105F700020BD0FB6F894FA9AF99A0FBE8C2F0E94A2
:105F80005A2F0E94D26D0E94DB8B81E090E002C00C
:105F900080E090E0CF9108956DE470E088EE93E0AA
:105FA0000E941C2D482F8FB399279C0122703070BE
:105FB00081FDF9CF85E394E092BD81BDF89A80B56B
:105FC000841779F48FB399279C012270307081FD7A
:105FD000F9CF88EE93E092BD81BDF89A80B581300B
:105FE00011F0C901089527EF3CE24EE450E068EE5D
:105FF00073E080E098E00E94FE8F81E090E00895D9
:10600000809100088130A9F46DE470E080E098E0B0
:106010000E940B2D80934D082FEF3CE24EE450E0A0
:1060200060E078E088EE93E00E943B9081E090E0B1
:10603000089580E090E00895CF93DF9381E080930E
:106040000008E0E0F8E08FE0158616861786108AD3
:106050008150349687FFF8CF80E480930D088093B9
:106060000E0810920F08809310088093110890EC8E
:1060700090931208109213088093140880931508C7
:106080001092160890931708909318088093190897
:1060900010921A0880931B0890931C08A1E0B8E0A6
:1060A0008CE0E9E2F1E0ED01019009928A95E1F7D7
:1060B0006DE470E0CD0101970E940B2D80934D0897
:1060C000DF91CF910895F999FECF82E090E092BDE3
:1060D00081BDF89A80B5282F863078F023E0322FE2
:1060E000F999FECF1FBA82E090E092BD81BD30BD2C
:1060F0000FB6F894FA9AF99A0FBE822F992708954D
:106100001F93CF93C82F162F863010F0C5E003C021
:10611000882309F4C1E08C2F99278230910541F042
:106120008330910544F4019731F40E94492E05C053
:106130000E947E2E02C00E94B32E1123E1F06CE07B
:1061400070E080E590E00E941C2D282FF999FECF89
:106150008CE590E092BD81BDF89A80B5821759F424
:1061600027EF3CE24CE050E060E570E084E897E027
:106170000E94FE8F02C00E94342D8C2F0E94702F2F
:10618000CF911F910895DF92EF92FF920F931F938B
:10619000CF93FF24DF2CEF2C81E090E00E94E72ECC
:1061A0008C3511F031E0E32E6CE070E080E590E09A
:1061B0000E941C2DC82FF999FECF8CE590E092BD6E
:1061C00081BDF89A80B58C1711F421E0D22EC1E080
:1061D00001E010E0EE2029F48C2F0E94052F882387
:1061E000C9F591E0F92E1F930F938FEA98E09F93E2
:1061F0008F9380E695E19F938F93E0913B05F0911B
:106200003C0509952DB73EB72A5F3F4F2DBF0230A1
:10621000110549F0033011054CF40130110531F43A
:106220000E94492E05C00E947E2E02C00E94B32EFD
:10623000DD2059F027EF3CE24CE050E060E570E0F3
:1062400084E897E00E94FE8F02C00E94342D8C2FBC
:106250000E94702FCF5F0F5F1F4FC63008F4BACF78
:10626000FF2019F083E00E945A2F0E946330C82F4C
:106270000E94052F8C2F99279F938F9385ED98E08F
:106280009F938F9300E615E11F930F93E0913B05D9
:10629000F0913C05099581E090E00E94E72E2DB732
:1062A0003EB72A5F3F4F2DBF8F3F21F00E94CC2F7A
:1062B000882399F48EEE98E09F938F931F930F930A
:1062C000E0913B05F0913C0509950E941C300E942D
:1062D00000300F900F900F900F90EE2029F06CE59A
:1062E00081E090E00E94EF2E1092820790E0EDE0B6
:1062F000F8E0CFE08081349618160CF49F5FC1500F
:10630000C7FFF8CF90938207892F99279F938F9388
:1063100081E098E09F938F938FE099E09F938F9314
:106320001F930F93E0913B05F0913C0509950E9466
:106330004A098DB79EB708968DBFCF911F910F91D7
:10634000FF90EF90DF900895982F2FB7F894399829
:10635000389A88B1836088B98091B9008C7F809326
:10636000B9008AE28093B80010925303109251034F
:1063700010925003992379F0E6E5F8E08BE0108263
:106380001182128213821482158216821782815022
:10639000389687FFF4CF78942FBF08951092530357
:1063A00084E98093BC0080E88093BC001092BD001B
:1063B0001092BA001092BB001092B9001092B8006F
:1063C00010924F0380E00E94A4311092BB0085E838
:1063D0008093BC0080914D03826080934D030895AB
:1063E0001F920F920FB60F9211242F933F934F934A
:1063F0005F938F939F93EF93FF9380915303282F85
:106400003327442755278F5F80935303F9012731A2
:10641000310508F0C2C2E759FF4F0C945B9281E04E
:1064200080934F0309C0809151038C3090F4809188
:1064300051038F5F8093510380915103E82FFF2711
:10644000EE0FFF1FEE0FFF1FE050F84F8585181667
:1064500054F7809151038C3070F010924C031092DD
:106460004B031092510385E08093530380915003B6
:10647000880F8D5A04C080915103880F8E5A8093E3
:10648000BB0085E87FC280915103E82FFF2783E09E
:10649000EE0FFF1F8A95E1F7EA5AF74F818180934B
:1064A000BB0085E88093BC0080915103E82FFF2753
:1064B000EE0FFF1FEE0FFF1FEE0FFF1FEA5AF74F01
:1064C000808180FF91C080915103E82FFF27EE0F5C
:1064D000FF1FEE0FFF1FEE0FFF1FEA5AF74F8281DB
:1064E000882329F080918207873008F46CC280915C
:1064F0004B0390914C03892B09F065C280914903AD
:1065000090914A03892B09F05EC26EC080915103BD
:1065100021E030E002C0220F331F8A95E2F780911C
:10652000490390914A0328233923232B79F0809142
:106530005103E82FFF27EE0FFF1FEE0FFF1FEE0F97
:10654000FF1FEA5AF74F80E184830DC08091510309
:10655000E82FFF27EE0FFF1FEE0FFF1FEE0FFF1FAD
:10656000EA5AF74F148280915103E82FFF2753E036
:10657000EE0FFF1F5A95E1F7EA5AF74F8481282F53
:10658000332743E0220F331F4A95E1F780915103EF
:10659000E82FFF2793E0EE0FFF1F9A95E1F7EA5AE5
:1065A000F74F82818770822B8093BB0085E88093B0
:1065B000BC002091510381E090E002C0880F991F38
:1065C0002A95E2F720914B0330914C0382239323C9
:1065D000892B51F08EE498E09093570380935603F3
:1065E00088E080935803EFC184E089C1E0915603AD
:1065F000F091570381918093BB0085E88093BC00A4
:10660000F0935703E0935603809158038150809391
:106610005803882309F4D7C183E071C18091B90080
:10662000803351F580915403882329F480915103DC
:106630008F5F8093540380915103E82FFF2783E0FD
:10664000EE0FFF1F8A95E1F7EA5AF74F83819927EA
:106650008F7790708F3791057CF480915103E82FEC
:10666000FF27EE0FFF1FEE0FFF1FEE0FFF1FEA5A6F
:10667000F74F83818F5F83831092530384E9809364
:10668000BC008AE090E090933701809336018091BE
:1066900051038F5F80935103109253036DC180911A
:1066A000B9008034C9F180915003E82FFF27EE0F25
:1066B000FF1FEE0FFF1FEE0FFF1FEA5AF74F8381F8
:1066C0008F778383809150038F5F809350038091F5
:1066D00050038C30A0F01092500310924A03109295
:1066E0004903809155038F5F809355038C3038F0B8
:1066F0001092550380914D038D7F80934D038091BF
:106700004D03816080934D031092530384E980937D
:10671000BC0010924F0373C080915003E82FFF27F5
:10672000EE0FFF1FEE0FFF1FEE0FFF1FEA5AF74F8E
:1067300083818068838380915003E82FFF27EE0FC9
:10674000FF1FEE0FFF1FEE0FFF1FEA5AF74F80816A
:1067500080FF2FC080915003E82FFF2753E0EE0FFA
:10676000FF1F5A95E1F7EA5AF74F8481992700975E
:1067700051F04097D9F58EE498E0909357038093B9
:10678000560388E031C080915003992743E0880F79
:10679000991F4A95E1F7855A974F90935703809335
:1067A000560390915003809155039817E1F483E0CC
:1067B0001BC080915003992733E0880F991F3A95A9
:1067C000E1F7855A974F9093570380935603809132
:1067D0004D0381FD06C09091500380915503981799
:1067E00011F482E001C081E0809358038091580346
:1067F000813011F485E801C085EC8093BC00809164
:10680000540380934E0310925403DDC0E09156036D
:10681000F09157038091BB00808380915603909143
:106820005703019690935703809356038091580322
:10683000815080935803823010F085EC5DC0813028
:1068400011F485E859C080914D0381FF2DC08091DE
:10685000CF0380FD1DC080915003E82FFF2723E068
:10686000EE0FFF1F2A95E1F7EA5AF74F86818A3F1C
:1068700079F480915003E82FFF2793E0EE0FFF1F7C
:106880009A95E1F7EA5AF74F8081816080830CC0C6
:1068900080915003E82FFF2783E0EE0FFF1F8A95BA
:1068A000E1F7EA5AF74F1082809150038F5F80938F
:1068B0005003809150038C30A0F01092500310923E
:1068C0004A0310924903809155038F5F80935503CB
:1068D0008C3038F01092550380914D038D7F80935A
:1068E0004D031092530384E98093BC0080914D03C3
:1068F000816080934D0365C08093BC0086E08093E7
:10690000530361C088E9BBCD80915203880F805F3B
:10691000B6CD8091520399278130910561F0823084
:1069200091051CF4892B21F04EC0029739F04BC021
:1069300080911401A4CD80911301A1CD8091120109
:106940009ECD80E89CCD1092530384E98093BC00D7
:1069500010924F038AE090E09093370180933601C4
:1069600080915203823088F4809152038F5F80932C
:10697000520382E18093530380914D038E7F809375
:106980004D0385EA8093BC001EC010925203809193
:106990004D03816080934D0316C01092530384E928
:1069A0008093BC0080914D03816080934D038AE009
:1069B00090E090933701809336011092510310922A
:1069C000500310924F03FF91EF919F918F915F9130
:1069D0004F913F912F910F900FBE0F901F901895E0
:1069E0001F93CF93DF93182F80910604882321F4FF
:1069F0008091E702882319F081E090E097C01D3074
:106A000008F092C01123B1F0E12FFF2723E0EE0F31
:106A1000FF1F2A95E1F7EA5AF74F3597808135969F
:106A200088230CF081C03897808180FD03C083E00B
:106A300090E07CC080914E08823019F084E090E0B4
:106A400075C067E070E08EE498E00E940B2D909195
:106A50005508891719F085E090E068C080ED97E04F
:106A60000E946F19EC0180914D0380FD05C0CE019D
:106A70000E9478198823B9F3112319F48FEF90E05D
:106A80000BC0212F33272150304081E090E002C01D
:106A9000880F991F2A95E2F790934C0380934B033C
:106AA000A1E0B0E0E6E5F8E040E050E06BE0CD01C9
:106AB000042E02C0880F991F0A94E2F720914B031D
:106AC00030914C0382239323892B11F0118212827F
:106AD00061504F5F5F4F389667FFE9CF10925103C7
:106AE0001092530380914D038E7F80934D0385EA6E
:106AF0008093BC0080914D0380FD05C0CE010E94B3
:106B000078198823B9F380914B0390914C03892B1A
:106B100029F0CE010E947819882311F380914B034C
:106B200090914C03009711F082E090E0DF91CF91BB
:106B30001F9108950F931F93CF93DF93982F809108
:106B40000604882321F48091E702882319F081E06C
:106B500090E092C09D30A0F4992319F486E090E073
:106B60008BC0C92FDD27FE0133E0EE0FFF1F3A95E2
:106B7000E1F7EA5AF74F35978081359687FD03C0D4
:106B800082E090E079C03897808180FD03C083E087
:106B900090E072C080ED97E00E946F198C018091A7
:106BA0004D0380FD05C0C8010E9478198823B9F300
:106BB000219721E030E0C90102C0880F991FCA95D2
:106BC000E2F790934A0380934903D901E6E5F8E0A0
:106BD00040E050E06BE0CD01042E02C0880F991F09
:106BE0000A94E2F72091490330914A0382239323C8
:106BF000892B11F01182128261504F5F5F4F3896DE
:106C000067FFE9CF1092500310924E08109255087A
:106C10001092530380914D038E7F80934D0385EA3C
:106C20008093BC0080914D0380FD05C0C8010E9487
:106C300078198823B9F38091490390914A03892BED
:106C400029F0C8010E947819882311F380914E0819
:106C5000823019F084E090E00FC067E070E08EE4CD
:106C600098E00E940B2D90915508891719F085E046
:106C700090E002C080E090E0DF91CF911F910F91F2
:106C80000895CF93DF9380E021E83FEFCBEED8E08B
:106C9000E7EBF8E0DF01853020F411961C921E929C
:106CA00002C0318320831982188222968F5F129648
:106CB00032968A3180F3109273041092720410920B
:106CC0007504109274041092770410927604DF9188
:106CD000CF9108951F920F920FB60F9211240F9328
:106CE0001F932F933F934F935F936F937F938F9354
:106CF0009F93AF93BF93CF93DF93EF93FF938091D5
:106D0000F10782FDE1C0409186005091870080919B
:106D10005A0390915B03481B590B80918600909118
:106D2000870090935B0380935A03CA018D5494406B
:106D3000A0915C03B0915D03835F9A4178F48091E8
:106D40005C038093B608149714F010923A0181E026
:106D500090E090935D0380935C032BC2AD30B1054E
:106D60000CF027C2CA018B5F9040845B914008F011
:106D700086C08091380190913901481B590BE091F0
:106D8000EC07EE2351F0FF27EE0FFF1FE954F74FFA
:106D90008081918184369105ECF4FD01EA0FFB1F9F
:106DA000E954F74F80819181FA01E81BF90BCF017B
:106DB000F7FF03C0909581959F4F06975CF48091F3
:106DC0000704883C20F480910704865F01C088ECAA
:106DD00080930704FD01EA0FFB1FE954F74F808100
:106DE00091819C01220F331F280F391F240F351F5B
:106DF00037FF02C02D5F3F4FE901D595C795D59567
:106E0000C795CA0101968C179D0714F4219706C0F7
:106E100041505040C417D5070CF4219680910704C7
:106E2000833CE0F08D010A0F1B1FF801E954F74F76
:106E3000808191819E01281B390BC90163E070E0BC
:106E40000E94D491CB01880F991F860F971F05517F
:106E5000174FD80111969C938E9307C0AA0FBB1FA2
:106E6000A551B74F11961C921E92E0915C03F091D0
:106E70005D03EE0FFF1FE954F74FD183C0832091CC
:106E80005C0330915D032F5F3F4F30935D03209390
:106E90005C0380910101843108F08BC125303105FC
:106EA00011F45D9A01C05D9880915C0390915D033F
:106EB0008630910511F45C9A01C05C98079711F433
:106EC0005B9A77C15B9875C14091860050918700AD
:106ED00080915E0390915F03481B590B809186005F
:106EE0009091870090935F0380935E03CA018D5455
:106EF00094406091C803835F9A4108F07AC0609320
:106F0000590380915903843008F453C09091B60816
:106F100080915903981709F04CC05091C9035B3018
:106F200008F43FC010923A011092C80340E05F316C
:106F3000C0F0E42FFF27EE0FFF1F9F012C563C4FA0
:106F4000DF01A954B74F8D919C91D9018D939C93EA
:106F5000DF01A551B74F8D919C91E255FC4F918374
:106F60008083E42FFF27EE0FFF1F9F012954374F27
:106F7000DF01A05ABC4F8D919C91D90111969C9331
:106F80008E93DF01A658BC4F8D919C91E551F74F30
:106F900091838083842F8F5F482F8D3040F28093C0
:106FA000C8038091C9038F3FB9F08F5F8093C903F5
:106FB00013C08091C903853620F08AE08093C9030D
:106FC00002C01092C903809101018A3011F084310E
:106FD00010F0289A01C0289881E08093C80380911E
:106FE0000604882309F0E5C0809159038093B60810
:106FF000E0C06D3008F0B5C0CA018B5F9040845B83
:10700000914008F090C08091380190913901481B5F
:10701000590BE62FFF27EE0FFF1FE05AFC4F808130
:107020009181FA01E81BF90BCF0105960B9720F52A
:10703000E091EC07EE2351F0FF27EE0FFF1FE9541C
:10704000F74F8081918184369105B4F48091C90312
:107050008A3120F080910704865F05C08B3028F0CC
:10706000809107048E5F8093070480910704893C18
:1070700018F088EC80930704E62FFF27EE0FFF1F20
:10708000E05AFC4F808191819C01220F331F280F11
:10709000391F240F351F37FF02C02D5F3F4FE90115
:1070A000D595C795D595C795CA0101968C179D07AB
:1070B00014F4219706C041505040C417D5070CF472
:1070C0002196809107048E3BD8F0E62FFF27EE0F24
:1070D000FF1FDF01A05ABC4F8D919C919E01281B80
:1070E000390BC90163E070E00E94D491CB01880F95
:1070F000991F860F971FE658FC4F9183808308C025
:10710000E62FFF27EE0FFF1FE658FC4F118210827B
:107110008091C803E82FFF27EE0FFF1FE05AFC4FB6
:10712000D183C08309C0809101018A3011F084317C
:1071300010F0289A01C0289880910101843188F4C8
:107140008091C803853011F45D9A05C05D98863042
:1071500011F45C9A05C05C98873011F45B9A01C009
:107160005B988091C803843120F48F5F8093C803BB
:1071700020C08431F1F4809101018A3011F0843112
:1071800010F0289A01C028988EE18093C8032CE063
:10719000CBEED8E0A4E9B3E0E7EBF8E08D919D9168
:1071A000918380833296198218822296215027FF7C
:1071B000F5CFFF91EF91DF91CF91BF91AF919F916B
:1071C0008F917F916F915F914F913F912F911F917F
:1071D0000F910F900FBE0F901F901895EF92FF9296
:1071E0000F931F9380919F079927880F991F880FEE
:1071F000991F7C010027F7FC0095102F80916104F6
:1072000090916204A0916304B0916404BC01CD012B
:10721000A80197010E9409923093E1062093E006AD
:107220008091590490915A04A0915B04B0915C0440
:10723000BC01CD01A80197010E9409923093E30699
:107240002093E206809174099091750997FD039649
:1072500095958795959587959093E5068093E40697
:10726000809184099091850997FD0396959587955E
:10727000959587959093E7068093E6068091720432
:10728000909173042091240330912503821B930B6A
:107290009093E9068093E80680910104909102049E
:1072A000A0910304B0910404BC01CD0125E030E0BD
:1072B00040E050E00E9409923093EB062093EA06EA
:1072C00080911E0390911F039093ED068093EC062E
:1072D00080911F01909120019093EF068093EE061C
:1072E0008091570899279093F1068093F00680913A
:1072F0005F0899279093F3068093F20680916708C0
:1073000099279093F5068093F40680916F0899274A
:107310009093F7068093F6068091770899279093CB
:10732000F9068093F80680917F0899279093FB06D1
:107330008093FA068091870899279093FD068093A1
:10734000FC0680918F0899279093FF068093FE0694
:1073500080910704992790930107809300078091FB
:10736000800990918109A0918209B09183092091AF
:107370003C0130913D0140913E0150913F01BC01E3
:10738000CD010E9409923093030720930207809158
:10739000100A9091110A9093050780930407809139
:1073A000140A9091150A909307078093060780911D
:1073B000020390910303909309078093080780913B
:1073C00088019091890190930B0780930A0710928E
:1073D0000D0710920C078091160A992790930F07BA
:1073E00080930E078091D3049091D4049093110759
:1073F000809310078091D1049091D2049093130749
:107400008093120780915405882321F480915505BB
:10741000882321F08091DF06816003C08091DF0620
:107420008E7F8093DF061F910F91FF90EF9008955C
:10743000EF92FF921F93CF93DF93182F7B018091E0
:107440000604882391F5809101018C3010F086317B
:1074500011F4299801C0299A11501F3FE9F0F092C8
:107460000903E0920803E701809108039091090362
:10747000892B11F4209781F380910C038823A1F3C9
:1074800010920C038091080390910903892B09F451
:1074900021970E94FD8EE8CF809101018C3010F081
:1074A000863111F4299A01C02998DF91CF911F915B
:1074B000FF90EF900895CF93DF93809101018D307D
:1074C00011F40E94621E10927A008091280390911C
:1074D000290390933909809338098091260390916C
:1074E0002703909329098093280980912403909180
:1074F000250390937A098093790920912003309194
:107500002103C901880F991F880F991F820F931FAC
:10751000820F931F90937509809374092091220321
:1075200030912303C901880F991F880F991F820F7B
:10753000931F820F931F90938509809384098FEC8A
:1075400080937A00A8E0B4E0C8E8D7E097E089919A
:10755000E82FFF27EE0FFF1FE954F74F0190F0814E
:10756000E02DE158FF4F1E161F061CF0E0E0F0E092
:1075700005C0EF3FF10514F0EFEFF0E08C91282FFC
:107580003327E217F30714F4815004C02E173F0786
:1075900014F48F5F8C939150119697FFD8CF809100
:1075A000C4079927AA27BB27BC01CD0124EC39E0E9
:1075B00040E050E00E949591DC01CB018093800176
:1075C00090938101A0938201B09383018091C507BC
:1075D0009927AA27BB27BC01CD010E949591DC0108
:1075E000CB0180937C0190937D01A0937E01B093A9
:1075F0007F01DF91CF910895A0E0B0E0E2E0FBE3EE
:107600000C942A92882EC0E0D0E07E016E01109288
:107610005405D0936D04C0936C04D0936B04C09355
:107620006A04D0936704C0936604D0937704C09330
:107630007604D0937504C0937404D0937304C093FC
:1076400072041092640110926301109219030E9457
:107650005B3A84E690E00E9491190E945B3A809127
:10766000900780FF10C08091150190911601875BF3
:10767000934038F480911501909116018E5E9240EE
:1076800010F40E94E01D0FE18AE090E00E94911941
:107690008091240390912503C80FD91F809128035E
:1076A00090912903E80EF91E8091260390912703FB
:1076B000C80ED91E015007FFE7CF9701205F3F4F4B
:1076C0003695279536952795309377042093760441
:1076D000C6014096969587959695879590937504E3
:1076E000809374046096F5E0D695C795FA95E1F716
:1076F000D0937304C09372049093710480937004C8
:1077000030936F0420936E04882009F441C0809167
:1077100074099091750997FF03C0909581959F4FCB
:107720006CE070E00E94D4919B0170936D046093B3
:107730006C04809184099091850997FF03C090950E
:1077400081959F4F6CE070E00E94D49170936B0420
:1077500060936A04809125079091260790936704AF
:1077600080936604B90184E090E00E94002F60914C
:107770006A0470916B0486E090E00E94002F609193
:1077800066047091670488E090E00E94002F65C055
:1077900084E090E00E94FB2E90936D0480936C0433
:1077A00086E090E00E94FB2E90936B0480936A0425
:1077B00088E090E00E94FB2E9C01909367048093E8
:1077C000660480916C0490916D048150984050F44F
:1077D00080916A0490916B048150984018F4215074
:1077E0003440D8F180E399E09F938F9380E695E150
:1077F0009F938F93E0913B05F0913C050995809113
:1078000074099091750997FF03C0909581959F4FDA
:107810006CE070E00E94D49170936D0460936C04EE
:10782000809184099091850997FF03C09095819577
:107830009F4F6CE070E00E94D49170936B04609352
:107840006A0480912507909126079093670480939E
:1078500066040F900F900F900F90109239091092BC
:107860003809109229091092280910927A09109269
:10787000790984E690E00E9491198091200390910B
:1078800021039C01220F331F220F331F280F391FA2
:10789000280F391F309375092093740980912203B2
:1078A000909123038C01000F111F000F111F080F6F
:1078B000191F080F191F10938509009384098091DF
:1078C0009F07C82EDD24EE24FF24442737FD409572
:1078D000542FC701B6010E9495914B015C01609342
:1078E000610470936204809363049093640498012C
:1078F000442737FD4095542FC701B6010E9495914A
:10790000DC01CB018093590490935A04A0935B044B
:10791000B0935C048092410490924204A09243048C
:10792000B09244048093390490933A04A0933B04AA
:10793000B0933C041092310410923204109233043C
:10794000109234048091170190911801A0911901AF
:10795000B0911A019093280780932707109218037B
:107960001092170310922104109222041092230403
:107970001092240400918801109189011093200431
:1079800000931F0484E690E0909385018093840126
:1079900082E390E090930903809308038091C407E9
:1079A0009927AA27BB27BC01CD0124EC39E040E090
:1079B00050E00E949591DC01CB018856954CAF4F69
:1079C000BF4F8093800190938101A0938201B09377
:1079D00083018091C5079927AA27BB27BC01CD0148
:1079E0000E949591DC01CB018856954CAF4FBF4F5B
:1079F00080937C0190937D01A0937E01B0937F01E1
:107A00001092410110924001C801AA2797FDA0954C
:107A1000BA2F20913C0130913D0140913E0150919F
:107A20003F01BC01CD010E949591DC01CB01809307
:107A3000800990938109A0938209B09383091092E1
:107A40001C0410921B040E94D26D8091CF038460AD
:107A50008093CF038FEF8093000A1092010A80E297
:107A60008093020AC8E0D4E0A8E8B7E007E08D916F
:107A7000E82FFF27EE0FFF1FE954F74F8081918118
:107A800081588993015007FFF2CF84E68093070461
:107A900080910603882311F0579A06C080E091E197
:107AA0009093080180930701809176049091770468
:107AB00080569940815C9B4228F0809154058160FA
:107AC0008093540580917404909175048056994078
:107AD000815C9B4228F0809154058260809354051C
:107AE00080917204909173048C5291408957954013
:107AF00028F08091540584608093540580916C0433
:107B000090916D048C529140835C914028F080915B
:107B1000540588608093540580916A0490916B04A9
:107B20008C529140835C914028F080915405806193
:107B30008093540580916604909167048050924030
:107B40008355914028F080915405806280935405BC
:107B500086E4809377010E94DB8BECE0CDB7DEB743
:107B60000C944692A3E1B0E0E8EBFDE30C94249280
:107B70008091720490917304209124033091250325
:107B8000821B930B90937A098093790980912E033D
:107B900090912F0397FD07969C0113E0359527954B
:107BA0001A95E1F7309339092093380980912C0315
:107BB00090912D0397FD0796B3E095958795BA951B
:107BC000E1F7909329098093280930934409209381
:107BD000430990933C0980933B09809174099091EB
:107BE0007509AC01440F551F480F591F2091200300
:107BF00030912103C901880F991F880F991F820FA7
:107C0000931F820F931F480F591F57FF02C04D5FEC
:107C10005F4F5595479555954795509375094093F6
:107C200074098091840990918509AC01440F551F16
:107C3000480F591F2091220330912303C901880F57
:107C4000991F880F991F820F931F820F931F480F50
:107C5000591F57FF02C04D5F5F4F5595479555958A
:107C600047955093850940938409209120033091D2
:107C70002103C901880F991F880F991F820F931F35
:107C8000820F931F9C01442737FD4095542F80910C
:107C9000510490915204A0915304B0915404820F66
:107CA000931FA41FB51F8093510490935204A09377
:107CB0005304B09354042091220330912303C9014B
:107CC000880F991F880F991F820F931F820F931F90
:107CD0009C01442737FD4095542F80914D0490918D
:107CE0004E04A0914F04B0915004820F931FA41F23
:107CF000B51F80934D0490934E04A0934F04B0930E
:107D0000500480914D0990914E09209120033091AB
:107D10002103820F931F90934E0980934D09809108
:107D20007C0990917D092091220330912303820FD9
:107D3000931F90937D0980937C09809168049091B2
:107D400069040196909369048093680480912507E3
:107D5000909126072091660430916704821B930B53
:107D60009C01442737FD4095542F80914904909100
:107D70004A04A0914B04B0914C04820F931FA41F9E
:107D8000B51F8093490490934A04A0934B04B09389
:107D90004C048FEC80937A001092110120913904E9
:107DA00030913A0440913B0450913C0429873A8732
:107DB0004B875C8729543B46414050402CF028E4D7
:107DC0003BE641E050E00DC089859A85AB85BC85D6
:107DD000885B9449AE4FBF4F4CF428EB34E94EEF2B
:107DE0005FEF2D833E834F83588708C089859A852E
:107DF000AB85BC858D839E83AF83B887209141047A
:107E00003091420440914304509144042D873E87B1
:107E10004F87588B29543B46414050402CF028E472
:107E20003BE641E050E00DC08D859E85AF85B88969
:107E3000885B9449AE4FBF4F4CF428EB34E94EEFCA
:107E40005FEF29833A834B835C8308C08D859E85D1
:107E5000AF85B88989839A83AB83BC83A091790964
:107E6000B0917A09BB8BAA8BFD01CF01AA2797FDA0
:107E7000A095BA2FA0903104B0903204C090330482
:107E8000D0903404A80EB91ECA1EDB1EA092310485
:107E9000B0923204C0923304D0923404E09080094E
:107EA000F09081090091820910918309E80EF91E72
:107EB0000A1F1B1FE0928009F0928109009382093A
:107EC00010938309F091EA03F98BFF2309F098C11D
:107ED0008091E903882309F093C18091700986FF9E
:107EE0008FC18091280990912909AA2797FDA09513
:107EF000BA2FBC01CD0129813A814B815C810E945E
:107F000095919B01AC0197FF04C02150384F4F4F12
:107F10005F4FBBE05595479537952795BA95D1F7B3
:107F200080916301682E772488249924CA01B901BD
:107F3000A40193010E949591DC01CB0180938204FE
:107F400090938304A0938404B0938504B7FF04C086
:107F50008150904FAF4FBF4F1C012D01ACE05594A5
:107F6000479437942794AA95D1F7209282043092AF
:107F70008304409284045092850480913809909142
:107F80003909AA2797FDA095BA2FBC01CD012D81F3
:107F90003E814F8158850E94959197FF04C06150A2
:107FA000784F8F4F9F4FFBE0959587957795679515
:107FB000FA95D1F7A40193010E949591DC01CB01C0
:107FC0008093860490938704A0938804B0938904D7
:107FD000B7FF04C08150904FAF4FBF4F9C01AD0120
:107FE000ECE05595479537952795EA95D1F720937D
:107FF00086043093870440938804509389048091C9
:108000008204909183049093200980931F098091AA
:108010008604909187049093240980932309221960
:10802000330944095509209386043093870440930B
:10803000880450938904E20EF31E041F151FE0927A
:108040008009F0928109009382091093830980913D
:1080500062018823B1F457FF04C02F5F3F4F4F4F99
:108060005F4F5595479537952795A21AB30AC40ACD
:10807000D50AA0923104B0923204C0923304D09257
:1080800034042A893B8979010027F7FC0095102FD9
:108090008091860490918704A0918804B09189040E
:1080A000E80EF91E0A1F1B1FC801B70129813A817A
:1080B0004B815C810E9495919B01AC0197FF04C0AC
:1080C0002150384F4F4F5F4F6BE05595479537958F
:1080D00027956A95D1F780916401A82EBB24CC2402
:1080E000DD24CA01B901A60195010E949591DC0128
:1080F000CB0180937A0490937B04A0937C04B0938B
:108100007D04B7FF04C08150904FAF4FBF4F3C017B
:108110004D013CE095948794779467943A95D1F714
:1081200060927A0470927B0480927C0490927D0429
:10813000C801B7012D813E814F8158850E949591DC
:1081400097FF04C06150784F8F4F9F4F2BE095955C
:108150008795779567952A95D1F7A60195010E9495
:108160009591DC01CB0180937E0490937F04A093D2
:108170008004B0938104B7FF04C08150904FAF4F8B
:10818000BF4FAC01BD018CE075956795579547953C
:108190008A95D1F740937E0450937F0460938004C6
:1081A000709381042A893B8937FF03C0309521955C
:1081B0003F4F21343105E4F1D401C30197FE07C0DC
:1081C000B095A095909581959F4FAF4FBF4F813847
:1081D0009105A105B10584F4DB01CA0177FF07C051
:1081E000B095A095909581959F4FAF4FBF4F813827
:1081F0009105A105B105E4F081E080931D0418C04C
:1082000010922409109223091092200910921F093C
:1082100010927E0410927F041092800410928104C8
:1082200010927A0410927B0410927C0410927D04C8
:1082300080917E0490917F04A0918004B09181048C
:10824000BC01CD0124E630E040E050E00E940992FC
:10825000E0907A04F0907B04E21AF30AF092370976
:10826000E092360980917A0490917B04A0917C047D
:10827000B0917D04BC01CD0124E630E040E050E047
:108280000E940992DA01C90120917E0430917F0495
:108290008C01021B130B10932B0900932A09809168
:1082A0003C0190913D01A0913E01B0913F01BC0184
:1082B000CD0128E631E040E050E00E949591209108
:1082C00080093091810940918209509183092617D4
:1082D00037074807590764F0261B370B480B590B23
:1082E0002093800930938109409382095093830938
:1082F0002091800930918109409182095091830930
:1083000057FF0CC0260F371F481F591F20938009A5
:108310003093810940938209509383096091280921
:10832000709129096E0D7F1D9B01442737FD4095F3
:10833000542F8091350490913604A0913704B09168
:108340003804820F931FA41FB51F809335049093A8
:108350003604A0933704B09338048091EF039091D2
:10836000F003681B790BCB01AA2797FDA095BA2FC4
:1083700029853A854B855C85820F931FA41FB51F05
:108380008093390490933A04A0933B04B0933C0447
:10839000C0907C01D0907D01E0907E01F0907F0143
:1083A000C816D906EA06FB06C4F488EA91E6A0E0FE
:1083B000B0E08C199D09AE09BF09809339049093F0
:1083C0003A04A0933B04B0933C048093350490930B
:1083D0003604A0933704B093380422273327A90129
:1083E0002C193D094E095F098091390490913A0496
:1083F000A0913B04B0913C0482179307A407B507F2
:10840000B4F4D701C601885A9146A040B040809389
:10841000390490933A04A0933B04B0933C048093B6
:10842000350490933604A0933704B09338046091D8
:10843000380970913909600F711F9B01442737FD7E
:108440004095542F80913D0490913E04A0913F04AB
:10845000B0914004820F931FA41FB51F80933D0469
:1084600090933E04A0933F04B09340048091ED03A9
:108470009091EE03681B790BCB01AA2797FDA0957D
:10848000BA2F2D853E854F855889820F931FA41FD3
:10849000B51F8093410490934204A0934304B0938A
:1084A0004404E0908001F0908101009182011091DC
:1084B0008301E816F9060A071B07C4F488EA91E667
:1084C000A0E0B0E08E199F09A00BB10B809341048E
:1084D00090934204A0934304B093440480933D04DA
:1084E00090933E04A0933F04B09340042227332787
:1084F000A9012E193F09400B510B80914104909125
:108500004204A0914304B091440482179307A40746
:10851000B507B4F4D801C701885A9146A040B040CD
:108520008093410490934204A0934304B093440485
:1085300080933D0490933E04A0933F04B093400485
:108540008091310490913204A0913304B0913404AD
:108550008093450490934604A0934704B093480445
:108560008091410490914204A0914304B09144044D
:108570008093610490936204A0936304B0936404B5
:108580008091390490913A04A0913B04B0913C044D
:108590008093590490935A04A0935B04B0935C04B5
:1085A00080913D0490913E04A0913F04B09140041D
:1085B00080935D0490935E04A0935F04B093600485
:1085C0008091350490913604A0913704B09138041D
:1085D0008093550490935604A0935704B093580485
:1085E00080911D0190911E0197FD079603E09595DE
:1085F00087950A95E1F7909339098093380980911E
:108600001B0190911C0197FD079613E095958795A6
:108610001A95E1F7909329098093280980912803FE
:10862000909129030F9734F488E19CEF90933909D6
:10863000809338098091280390912903079734F497
:1086400080E398EF909339098093380920910101D4
:108650002A30A9F48091280390912903835F9340E5
:1086600034F088EE93E09093390980933809809133
:108670002803909129038A5F9340DCF014C0809115
:10868000280390912903815D974034F088EE93E0B0
:108690009093390980933809809128039091290398
:1086A000805E974034F080ED97E090933909809395
:1086B000380980912603909127030F9734F488E1BD
:1086C0009CEF90932909809328098091260390912B
:1086D0002703079734F480E398EF90932909809358
:1086E00028092A30A9F48091260390912703835FFB
:1086F000934034F088EE93E0909329098093280901
:1087000080912603909127038A5F9340DCF014C088
:108710008091260390912703815D974034F088EE85
:1087200093E09093290980932809809126039091E2
:108730002703805E974034F080ED97E090932909FD
:108740008093280960916E01662309F4AFC04091BF
:108750001D0150911E0180918A0490918B04481B49
:10876000590B509391044093900420911D01309136
:108770001E01280F391F37FF02C02F5F3F4F35956D
:10878000279530938B0420938A04413851051CF0BF
:1087900080E890E005C040585F4F34F480E89FEFD8
:1087A000909391048093900440911B0150911C017F
:1087B00080918C0490918D04481B590B50938F0429
:1087C00040938E0420911B0130911C01280F391F0A
:1087D00037FF02C02F5F3F4F3595279530938D04AB
:1087E00020938C04413851051CF080E890E005C0CE
:1087F00040585F4F34F480E89FEF90938F0480934C
:108800008E04462F55278091900490919104849F67
:10881000B001859F700D949F700D11249B0177FF0F
:1088200002C0215F3F4FF4E035952795FA95E1F7B7
:108830008091380990913909820F931F90933909DB
:108840008093380980918E0490918F04849FD00189
:10885000859FB00D949FB00D1124AD019D01B7FF10
:1088600002C0215F3F4FE4E035952795EA95E1F797
:108870008091280990912909820F931F90932909CB
:108880008093280980911D0190911E01860F971FEA
:1088900090931E0180931D0180911B0190911C01FA
:1088A000840F951F90931C0180931B0100913B093D
:1088B00010913C0980911F09909120091016110612
:1088C0005CF59C0197FF04C022273327281B390B36
:1088D000C901AA2797FDA095BA2F209162013327DD
:1088E00044275527BC01CD010E9495919B01AC0105
:1088F00097FF04C0215C3F4F4F4F5F4F76E0559587
:108900004795379527957A95D1F7809136099091BB
:108910003709820F931F27C097FF03C09095819559
:108920009F4FAA2797FDA095BA2F20916201332768
:1089300044275527BC01CD010E9495919B01AC01B4
:1089400097FF04C0215C3F4F4F4F5F4F66E0559546
:108950004795379527956A95D1F78091360990917B
:108960003709821B930B9093370980933609E09067
:108970004309F090440980912309909124091E1421
:108980001F045CF59C0197FF04C022273327281B96
:10899000390BC901AA2797FDA095BA2F2091620132
:1089A000332744275527BC01CD010E9495919B0197
:1089B000AC0197FF04C0215C3F4F4F4F5F4F96E0E3
:1089C00055954795379527959A95D1F780912A091E
:1089D00090912B09820F931F27C097FF03C090959A
:1089E00081959F4FAA2797FDA095BA2F20916201EC
:1089F000332744275527BC01CD010E9495919B0147
:108A0000AC0197FF04C0215C3F4F4F4F5F4F86E0A2
:108A100055954795379527958A95D1F780912A09DD
:108A200090912B09821B930B90932B0980932A0919
:108A30008091700987FF44C0B989BB2309F040C009
:108A40008091E9038823E1F5E1E0EE16E1E0FE061E
:108A50004CF080913809909139098E0D9F1D8050FE
:108A600091400DC0F0E0EF16FFEFFF0664F4809137
:108A70003809909139098E0D9F1D80509F4F90931A
:108A800039098093380921E0013012074CF08091B8
:108A9000280990912909800F911F805091400CC0A6
:108AA0003FEF0030130764F4809128099091290961
:108AB000800F911F80509F4F909329098093280920
:108AC000E2E1CD5E0C94409280910604882301F58A
:108AD0008091CF038C7F8093CF03A9E5B5E0E6E5D5
:108AE000F8E09BE08091E702882309F48C938D9154
:108AF000818312829150389697FFF4CF8091E702DC
:108B0000882359F08091E70281508093E70205C0E5
:108B10008091CF0381608093CF0380914F0388239E
:108B200019F010924F0308958093510380935303DB
:108B300080914D038E7F80934D0385EA8093BC0026
:108B40000895CF93DF93A8E0B4E0C8E8D7E057E0FA
:108B50009991E92FFF27EE0FFF1FE954F74F01907E
:108B6000F081E02DE158FF4FEF3FF10521F01CF0BF
:108B7000EFEFF0E004C0F7FF02C0E0E0F0E0993171
:108B800011F4EC931BC04C91242F3327E217F30709
:108B9000A9F0CF01821B930B97FD039695958795BE
:108BA00095958795242F280F2C93822F9927E817C6
:108BB000F90714F4215001C02F5F2C9351501196E6
:108BC00057FFC6CF80919207883F38F0EFEFF0E073
:108BD000E81BF109E85FFB4F80818093740180916D
:108BE0007401882329F0843618F084E68093740198
:108BF00080919407883F38F0EFEFF0E0E81BF1092F
:108C0000E85FFB4F8081809372018091720188231D
:108C100029F0843618F084E6809372018091A107D0
:108C2000883F38F0EFEFF0E0E81BF109E85FFB4F19
:108C3000808180936D0180916D018B3010F48AE00A
:108C400002C08F3F11F480936D018091CE07883F61
:108C500038F0EFEFF0E0E81BF109E85FFB4F8081AF
:108C600080934F0980914F09863010F485E002C04F
:108C70008F3F11F480934F098091D007883F38F0DF
:108C8000EFEFF0E0E81BF109E85FFB4F8081809394
:108C9000770980917709863010F485E002C08F3F14
:108CA00011F4809377098091BB07873F19F44299AB
:108CB00005C006C0863F31F4439B02C08CE80BC060
:108CC00086E409C0883F38F0EFEFF0E0E81BF109D7
:108CD000E85FFB4F808180934C098091BC07873F00
:108CE00019F4429905C006C0863F31F4439B02C087
:108CF0008CE80BC086E409C0883F38F0EFEFF0E065
:108D0000E81BF109E85FFB4F808180932509809182
:108D1000BD07883F38F0EFEFF0E0E81BF109E85FAE
:108D2000FB4F80818093550980919307883F38F0ED
:108D3000EFEFF0E0E81BF109E85FFB4F80818093E3
:108D4000730180919607883F38F0EFEFF0E0E81B61
:108D5000F109E85FFB4F8081809371018091980752
:108D6000883F38F0EFEFF0E0E81BF109E85FFB4FD8
:108D7000808180936F018091A007883F38F0EFEFEA
:108D8000F0E0E81BF109E85FFB4F80818093700100
:108D90008091A207883F38F0EFEFF0E0E81BF1097F
:108DA000E85FFB4F808180936C018091A307883F2F
:108DB00038F0EFEFF0E0E81BF109E85FFB4F80814E
:108DC00080936E018091A407883F38F0EFEFF0E0C8
:108DD000E81BF109E85FFB4F808180936B01809174
:108DE000A507883F38F0EFEFF0E0E81BF109E85FF6
:108DF000FB4F808180936A018091AB07883F38F0F8
:108E0000EFEFF0E0E81BF109E85FFB4F8081809312
:108E100068018091AC07883F38F0EFEFF0E0E81B85
:108E2000F109E85FFB4F80818093E4038091AD07F7
:108E3000883F38F0EFEFF0E0E81BF109E85FFB4F07
:108E400080818093E3038091AE07883F38F0EFEF95
:108E5000F0E0E81BF109E85FFB4F80818093E203BB
:108E60008091AF07883F38F0EFEFF0E0E81BF109A1
:108E7000E85FFB4F80818093E1038091C907883FC1
:108E800038F0EFEFF0E0E81BF109E85FFB4F80817D
:108E90008093E0038091CA07883F38F0EFEFF0E05D
:108EA000E81BF109E85FFB4F80818093DF0380912D
:108EB000CB07883F38F0EFEFF0E0E81BF109E85FFF
:108EC000FB4F80818093DE038091CC07883F38F090
:108ED000EFEFF0E0E81BF109E85FFB4F8081809342
:108EE000DD038091B007883F38F0EFEFF0E0E81B3A
:108EF000F109E85FFB4F8081809367018091B4079F
:108F0000883F38F0EFEFF0E0E81BF109E85FFB4F36
:108F10008081809366018091BE07883F38F0EFEF33
:108F2000F0E0E81BF109E85FFB4F80818093650169
:108F30008091C107883F38F0EFEFF0E0E81BF109BE
:108F4000E85FFB4F8081809364018091C207883F76
:108F500038F0EFEFF0E0E81BF109E85FFB4F8081AC
:108F6000809363018091C307883F38F0EFEFF0E012
:108F7000E81BF109E85FFB4F8081809362018091DB
:108F8000EB07883F38F0EFEFF0E0E81BF109E85F0E
:108F9000FB4F8081809334099091DD04992321F067
:108FA00080913409981720F080913409882311F4B6
:108FB0009093340980919007809370098091F10714
:108FC000809354098091C807883F38F0EFEFF0E0B4
:108FD000E81BF109E85FFB4F80818093610180917C
:108FE000E407883F38F0EFEFF0E0E81BF109E85FB5
:108FF000FB4F80818093870980916801282F332758
:109000002F5F3F4F8CE398E2B9010E94D491709397
:1090100076016093750180919E0780937809809115
:109020009D0780933D099091E607933308F44AC069
:1090300081E08093DC03983F58F0EFEFF0E0E91B0C
:10904000F109E85FFB4F8081823310F41092DC035A
:10905000809177012091DC03821721F18330F8F4AD
:1090600030919D01222351F08CED95E090930903FE
:1090700080930803332369F48EE209C088EC90E002
:109080009093090380930803332319F487E18093B5
:109090009D0185E08093F1032093770103C0815007
:1090A000809377018091C7099091C80997FF0FC0FD
:1090B0008091DC03882359F0809154058068809367
:1090C000540505C01092DC038AE0809377018091FB
:1090D000C7099091C80997FF1DC080910604882395
:1090E000C9F08091DC038823A9F080910901909157
:1090F0000A018F5F9F4F71F488E99AE39093090307
:109100008093080380E094EA90930A018093090118
:109110001092DC038091DC03882369F08091CE03F8
:1091200081608093CE0380916401823D48F4825E29
:109130008093640105C08091CE038E7F8093CE031F
:10914000DF91CF910895A7E1B0E0E9EAF8E40C944B
:1091500024920E94B23D8091CF0399278471907030
:10916000892B91F58091F20782FF27C08091EB0354
:109170009091EC030097F1F002E088359007D4F469
:109180009C0197FF02C02D5F3F4F35952795359580
:1091900027958091A8079927289FA001299F500D06
:1091A000389F500D1124CA0164E670E00E94D491EA
:1091B000CB0106C08DE290E003C08091A8079927FB
:1091C0009093CD038093CC032091CA033091CB03BD
:1091D00055E72033350759F4109212041092110408
:1091E00080913D0999279093CD038093CC036091A2
:1091F0001104709112047A83698380913D09992743
:109200000A966817790714F49A8389838091070472
:10921000843608F06AC08091CE0382FD66C08091DA
:10922000A6049091A704009731F001979093A704AA
:109230008093A6040BC0109206049093D1038093F0
:10924000D0038091CF038D7E8093CF038091010165
:109250008A3011F0843110F0289A01C0289880914A
:10926000D0039091D103895E9340E0F18091160A7A
:109270008536C0F18091CC039091CD039A83898388
:109280008091CF0380618093CF0380918407A82FC2
:10929000BB27AA0FBB1FFD01E551F74F11821082BA
:1092A00080918507282F3327220F331FC90185514D
:1092B000974FFC0111821082A954B74F11961C924E
:1092C0001E922954374FD90111961C921E928091FB
:1092D0008707E82FFF27EE0FFF1FE954F74F118292
:1092E00010823FC3109206043CC3809107048D385E
:1092F00008F40DC38091CF038F7E8093CF039091AC
:10930000A90782E3989FC00111249093A70480933A
:10931000A604E981FA81B9978CF08091060488232C
:1093200069F08091D0039091D103FFEF8F3F9F07A9
:1093300029F001969093D1038093D0038091D003BC
:109340009091D1038F3F910509F008F510922904FF
:1093500010922A0410922B0410922C0410922504CF
:10936000109226041092270410922804109292045E
:109370001092930410929404109295041092310468
:1093800010923204109233041092340405C080917C
:10939000CF0382608093CF0380918607E82FFF2759
:1093A000EE0FFF1FE954F74F8081918181359105C0
:1093B0000CF438C120910604222309F033C18091B6
:1093C0008707E82FFF27EE0FFF1FE954F74F808133
:1093D00091818C3491050CF4FFC08091A8048F5FBB
:1093E0008093A804893C08F41DC12093A80410921E
:1093F000D1031092D00330918407E32FFF27EE0FA3
:10940000FF1FE954F74F8081918187349105B4F4AF
:1094100080918507E82FFF27EE0FFF1FE954F74FD4
:10942000808191810190F081E02DF7FF03C0F095DC
:10943000E195FF4FE734F1050CF478C041E020914D
:109440008507A22FBB27AA0FBB1FA954B74F8D9129
:109450009C9111978734910544F0E32FFF27EE0F7D
:10946000FF1FE954F74F808191818D919C91873442
:10947000910574F080918407E82FFF27EE0FFF1FFE
:10948000E954F74F80819181873491050CF042E0D7
:10949000E22FFF27EE0FFF1FE954F74F80819181E4
:1094A0008634910574F480918407E82FFF27EE0F2E
:1094B000FF1FE954F74F80819181873491050CF0AB
:1094C00043E0E22FFF27EE0FFF1FE954F74F8081A3
:1094D00091818A5B9F4F74F480918407E82FFF2766
:1094E000EE0FFF1FE954F74F80819181873491057A
:1094F0000CF044E0E22FFF27EE0FFF1FE954F74F77
:10950000808191818A5B9F4F74F480918407E82F5A
:10951000FF27EE0FFF1FE954F74F808191818634BA
:1095200091050CF445E0842F0E945A2F8091850705
:10953000E82FFF27EE0FFF1FE954F74F808191813D
:109540000190F081E02DF7FF03C0F095E195FF4F0A
:109550007E97CCF480918407E82FFF27EE0FFF1F42
:10956000E954F74F808191818A5B9F4F64F481E0D9
:1095700080936F051092F20388EE93E090930903B5
:10958000809308034FC00E9463300E94052F80E043
:109590000E9491098091AA070E94918D8091700983
:1095A00080FF10C08091150190911601875B934058
:1095B00038F480911501909116018E5E924010F45E
:1095C0000E94E01D80E00E94FC3A81E08093F2035B
:1095D00080930603579A1AC080819181855B9F4FC3
:1095E000FCF48091A8048F5F8093A804893CD0F09C
:1095F000209306042093A8041092D1031092D00364
:1096000081E00E94FC3A81E08093F20388E180933C
:109610009D010E94633068E770E00E94183A02C022
:109620002093A80480918607E82FFF27EE0FFF1FE5
:10963000E954F74F808191818B5A9F4F0CF060C1A4
:109640002091E707E22FFF27EF77F070EE0FFF1F63
:10965000E551F74F80819181069714F084E606C0AA
:10966000808191818B5F9F4F1CF48CE98093AB04C8
:1096700080910604E0918707882309F0ECC0FF275A
:10968000EE0FFF1FE954F74F80819181855B9F4F5B
:109690009CF48091F20783FD0BC0E22FFF27EE0FB1
:1096A000FF1FE954F74F80819181855B9F4FDCF06C
:1096B0008091E7078823B9F08091F20783FFC8C043
:1096C0008091E707E82FFF27EE0FFF1FE954F74FC0
:1096D00080819181875F9F4F0CF4BAC08091AB0469
:1096E000843609F0B5C02091F203222329F080913D
:1096F000CF0388608093CF038091A9048F5F80930C
:10970000A9048E3F08F4EEC01092A904809154057C
:10971000882309F092C0222309F48FC08091E204CB
:10972000882309F08AC081E090E09093D103809370
:10973000D00381E080930604109292041092930467
:1097400010929404109295041092310410923204F5
:10975000109233041092340410922D0410922E04AF
:1097600010922F041092300480919F07E82EFF245E
:109770000027112780917409909175099C01442755
:1097800037FD4095542FC801B7010E949591DC0127
:10979000CB018093410490934204A0934304B0937F
:1097A000440480918409909185099C01442737FDE8
:1097B0004095542FC801B7010E949591DC01CB015F
:1097C0008093390490933A04A0933B04B0933C04F3
:1097D0008091610490916204A0916304B09164044B
:1097E00080933D0490933E04A0933F04B0934004C3
:1097F0008091590490915A04A0915B04B0915C044B
:109800008093350490933604A0933704B0933804C2
:109810001092290410922A0410922B0410922C0406
:109820001092250410922604109227041092280406
:1098300084E68093F10384E350C08CED95E090932F
:10984000090380930803222309F04CC081E045C03E
:109850001092A90447C0FF27EE0FFF1FE954F74FEE
:10986000808191818C3491059CF08091F20783FD79
:109870000BC0E22FFF27EE0FFF1FE954F74F808147
:109880009181855B9F4FCCF08091E7078823A9F0F9
:109890008091F20783FF24C08091E707E82FFF271C
:1098A000EE0FFF1FE954F74F808191818E5C9F4F2F
:1098B000BCF48091AB048C3999F48091AA048F5F39
:1098C0008093AA048B3F70F0109206041092AA04B1
:1098D0001092D1031092D00386E280939D0102C0C2
:1098E0001092AA048091CA039091CB0313E0883EA2
:1098F0009107B8F501969093CB038093CA0331C0CA
:109900001092AB041092CB031092CA032AC02E5EB1
:10991000324038F180918F0990919009805991409F
:1099200000F58091010490910204A0910304B0918C
:1099300004048C5D9540A040B0409CF480E395E722
:109940009093CB038093CA038091D0039091D1036D
:109950008A5E934030F089EE93E09093D103809338
:10996000D00380913A01815080933A0180913A016D
:109970008F3F21F08091CF0384FFA9C30E94A145AE
:10998000B0909A078091B4049091B5049C01220F85
:10999000331F280F391FC0908407AC2DBB27AA0F97
:1099A000BB1FFD01E954F74F4B2D55278081918155
:1099B000849FF001859FF00D949FF00D11242E0FD0
:1099C0003F1F37FF02C02D5F3F4FB9017595679567
:1099D00075956795A551B74F80919B07082F112763
:1099E0008D919C91809F7001819FF00C909FF00C55
:1099F00011246E0D7F1D7093B5046093B4048091A3
:109A0000B6049091B7049C01220F331F280F391F11
:109A1000D0908507AD2DBB27AA0FBB1FFD01E954D0
:109A2000F74F80819181849FF001859FF00D949F75
:109A3000F00D11242E0F3F1F37FF02C02D5F3F4F47
:109A4000A9015595479555954795A551B74F8D91C6
:109A50009C91809F7001819FF00C909FF00C1124CD
:109A60004E0D5F1D5093B7044093B6048091DC0304
:109A7000882309F448C0CB0177FD0396DC01B59536
:109A8000A795B595A795CA0157FD0396FC01F595D5
:109A9000E795F595E79580919801682F772767FD01
:109AA00070956A9F90016B9F300D7A9F300D112445
:109AB0008091E404482F552747FD50954E9FC001E3
:109AC0004F9F900D5E9F900D1124280F391F37FF77
:109AD00002C0295F3F4F93E0359527959A95E1F7AE
:109AE00030931804209317046E9F90016F9F300DE0
:109AF0007E9F300D11244A9FC0014B9F900D5A9FAD
:109B0000900D11243FC08091E507E82FFF27EE5B01
:109B1000FE4F86818093980190819093E404A82F52
:109B2000BB27A7FDB095A69F9001A79F300DB69FBC
:109B3000300D1124E92FFF27E7FDF095E49FC001C8
:109B4000E59F900DF49F900D1124280F391F37FFCA
:109B500002C0295F3F4F83E0359527958A95E1F74D
:109B60003093180420931704A49F9001A59F300DF3
:109B7000B49F300D1124E69FC001E79F900DF69F22
:109B8000900D1124281B390B37FF02C0295F3F4F6E
:109B900003E0359527950A95E1F730931604209355
:109BA000150480918707E82FFF27EE0FFF1FE95468
:109BB000F74F80819181909581959F4F90931404E8
:109BC000809313048530910514F0049705C00FEFBE
:109BD0008C3F900734F404969093140480931304FC
:109BE00004C010921404109213048091D0048823AE
:109BF00009F43EC0282F3327809117049091180450
:109C000097FD079613E0959587951A95E1F7289F9C
:109C1000A001299F500D389F500D1124CA0157FDF6
:109C20000F96B4E095958795BA95E1F7909318044F
:109C300080931704809115049091160497FD079660
:109C4000A3E095958795AA95E1F7289FB001299FF4
:109C5000700D389F700D1124CB0177FD0F96F4E045
:109C600095958795FA95E1F79093160480931504DE
:109C700080901704909018048091D3049091D4049C
:109C8000881A990A9092180480921704009115047A
:109C9000109116048091D1049091D204081B190BE5
:109CA000109316040093150480918607E82FFF2770
:109CB000EE0FFF1FE954F74FE080F1808FE790E04F
:109CC000E80EF91EF0921204E092110480916D01E9
:109CD0009927AA2797FDA095BA2FBC01CD010E9414
:109CE0000991DC01CB0120E030E040E251E4BC010D
:109CF000CD010E947790DC01CB01BC01CD010E9417
:109D0000DB90DC01CB0180937E0980916C01809314
:109D1000560980916B019927AA2797FDA095BA2F24
:109D2000BC01CD010E940991DC01CB0120E030E0B3
:109D300040E251E4BC01CD010E947790DC01CB01EF
:109D4000BC01CD010E94DB90DC01CB0180932F0987
:109D500080916A018093450980917B0580FF59C0FD
:109D600080918709813808F454C08091740599273F
:109D700087FD90952B2D3327829FD001839FB00DB7
:109D8000929FB00D11248A0E9B1E9092180480920F
:109D9000170480917505992787FD9095829FF001A2
:109DA000839FF00D929FF00D11240E0F1F1F109333
:109DB00016040093150480917605282F332727FD7C
:109DC00030958091130490911404820F931F909307
:109DD00014048093130480917805282F332727FDDE
:109DE0003095809195079927289F8001299F100D14
:109DF000389F100D11241093410100934001809170
:109E0000770599278E159F0524F49093120480936B
:109E10001104809111049091120497FF04C01092D4
:109E20001204109211048091700982FF02C01092F6
:109E300056094091170450911804CA0157FD039622
:109E40009C01359527953595279537FF03C03095AB
:109E500021953F4F8091D4039091D50382179307AA
:109E6000B4F4CA0157FF03C0909581959F4F97FDA9
:109E7000039695958795959587959093D5038093AF
:109E8000D4038536910544F084E690E001C0019743
:109E90009093D5038093D4034091150450911604F8
:109EA000CA0157FD03969C01359527953595279551
:109EB00037FF03C0309521953F4F8091D203909199
:109EC000D30382179307B4F4CA0157FF03C09095D8
:109ED00081959F4F97FD03969595879595958795C5
:109EE0009093D3038093D2038536910544F084E6A2
:109EF00090E001C001979093D3038093D2038091A7
:109F0000CF0384FF08C01092D5031092D40310929F
:109F1000D3031092D203ED2DFF27EE0FFF1FE9545C
:109F2000F74F4091BF07242F332780819181281755
:109F3000390744F48091EF0782FF04C081E08093E9
:109F4000E80313C0ED2DFF27EE0FFF1FE954F74F75
:109F5000842F99272091C007821B9109208131818C
:109F60002817390714F41092E80340918507E42F6D
:109F7000FF27EE0FFF1FE954F74F5091BF07852FC2
:109F8000992722273327281B390B8081918182173B
:109F9000930744F48091EF0783FF04C081E080932E
:109FA000E70316C08091E703882391F0E42FFF2791
:109FB000EE0FFF1FE954F74F8091C0079927851BCB
:109FC0009109208131818217930714F41092E703DD
:109FD000EC2DFF27EE0FFF1FE954F74F4091BF070D
:109FE000242F3327808191812817390744F48091E9
:109FF000EF0780FF04C081E08093E50317C08091E4
:10A00000E503882399F0EC2DFF27EE0FFF1FE9549D
:10A01000F74F842F99272091C007821B9109208137
:10A0200031812817390714F41092E5034091840711
:10A03000E42FFF27EE0FFF1FE954F74F5091BF07A2
:10A04000852F992722273327281B390B808191815F
:10A050008217930744F48091EF0781FF04C081E0E9
:10A060008093E60316C08091E603882391F0E42FE5
:10A07000FF27EE0FFF1FE954F74F8091C007992784
:10A08000851B9109208131818217930714F4109266
:10A09000E6038091E803882319F48091E703811196
:10A0A00081E08093E9038091E503882321F4809186
:10A0B000E603882351F081E08093EA031092E903DC
:10A0C0001092E8031092E70302C08093EA038091A4
:10A0D000E903882321F48091EA03882369F08091C1
:10A0E000BE07992729813A818217930714F49A832E
:10A0F000898381E080931D048091CE0399279C0180
:10A100002470307082FF2DC08091D3049091D404CC
:10A11000909581959F4F9093180480931704809198
:10A12000D1049091D204909581959F4F90931604FD
:10A130008093150480917A0190917B019093120491
:10A1400080931104809170098B778B6680937009DE
:10A15000809154098C7B8093540988EC809373011F
:10A160001EC08091CF0384FF1AC030931404209343
:10A17000130430931804209317043093160420938B
:10A1800015049AE590937E0988E780935609909389
:10A190002F09809345091092E9031092EA038091F8
:10A1A000480990914909A0914A09B0914B09209121
:10A1B0006104309162044091630450916404820F01
:10A1C000931FA41FB51F8093480990934909A0933A
:10A1D0004A09B0934B098091500990915109A0917F
:10A1E0005209B0915309E0905904F0905A0400913B
:10A1F0005B0410915C04EB82FC820D831E838E0D48
:10A200009F1DA01FB11F8093500990935109A093E7
:10A210005209B093530980913F0990914009A09150
:10A220004109B0914209E0905D04F0905E04009114
:10A230005F0410916004EF82F88609871A878E0DFB
:10A240009F1DA01FB11F80933F0990934009A093C9
:10A250004109B09342098091300990913109A09150
:10A260003209B0913309E0905504F0905604009102
:10A27000570410915804EB86FC860D871E878E0DBF
:10A280009F1DA01FB11F8093300990933109A093A7
:10A290003209B0933309F090EA03FF86FF2029F4D6
:10A2A0008091E903882309F460C010925104109250
:10A2B0005204109253041092540410924D041092C0
:10A2C0004E0410924F0410925004109248091092BC
:10A2D000490910924A0910924B09109250091092A4
:10A2E0005109109252091092530910923F0910928D
:10A2F00040091092410910924209109230091092BF
:10A3000031091092320910923309809141049091E1
:10A310004204A0914304B091440480933D0490937F
:10A320003E04A0933F04B09340048091390490917F
:10A330003A04A0913B04B0913C048093350490937F
:10A340003604A0933704B093380410921603109289
:10A3500015031092EE031092ED031092F003109289
:10A36000EF030F85002309F0D0C18091E903882312
:10A3700009F0CBC18091250790912607815092402A
:10A380002CF480910604882309F4BFC19090000A40
:10A39000A0909F072090740930907509409084091F
:10A3A0005090850919140CF0BBC0BB24CC24DD24CB
:10A3B000CA01B901A60195010E94099279018A0199
:10A3C0008091C9099091CA09281A390AC101AA279E
:10A3D00097FDA095BA2FE81AF90A0A0B1B0B6B819F
:10A3E0007C818D819E81A60195010E94099259016F
:10A3F0006A018091CB099091CC09481A590AC2018F
:10A40000AA2797FDA095BA2FA81AB90ACA0ADB0A8B
:10A41000292C332427FC3094432C532CC801B7013A
:10A42000A20191010E94959197FF04C061507E4F57
:10A430008F4F9F4F3B014C0109E09594879477948F
:10A4400067940A95D1F7C601B501A20191010E9456
:10A45000959197FF04C061507E4F8F4F9F4F5B01D6
:10A460006C0119E0D594C794B794A7941A95D1F7C5
:10A470008091D4039091D503813491053CF480916F
:10A48000D2039091D30381349105D4F0D401C30158
:10A4900097FE03C00196A11DB11D3C014D0195948D
:10A4A000879477946794D601C501D7FE03C00196BF
:10A4B000A11DB11D5C016D01D594C794B794A794FB
:10A4C0008091020A282F332727FD3095432F532FE1
:10A4D000261537054805590514F439014A0199270D
:10A4E00087FD9095909581959F4FAA2797FDA09500
:10A4F000BA2F681679068A069B0614F43C014D01B2
:10A500002A153B054C055D0514F459016A01A8168E
:10A51000B906CA06DB060CF0D0C05C016D01CDC0E7
:10A52000EA2CFF2400271127CA01B901A8019701CD
:10A530000E94099239014A01C101AA2797FDA095FD
:10A54000BA2F681A790A8A0A9B0A6B817C818D81ED
:10A550009E81A80197010E94099259016A01C201D6
:10A56000AA2797FDA095BA2FA81AB90ACA0ADB0A2A
:10A57000D401C30197FE03C00F96A11DB11D3C017C
:10A580004D01F4E09594879477946794FA95D1F708
:10A59000D601C501D7FE03C00F96A11DB11D5C01F8
:10A5A0006D01E4E0D594C794B794A794EA95D1F7E8
:10A5B0008091D4039091D503813491053CF480912E
:10A5C000D2039091D30381349105A4F0C401B30167
:10A5D00023E030E040E050E00E94099239014A0156
:10A5E000C601B50123E030E040E050E00E9409924E
:10A5F00059016A0180918707E82FFF27EE0FFF1F9F
:10A60000E954F74F808191810190F081E02DF7FFAF
:10A6100003C0F095E195FF4F7A97A4F0C401B30110
:10A6200023E030E040E050E00E94099239014A0105
:10A63000C601B50123E030E040E050E00E940992FD
:10A6400059016A0189E18093860121E26216710451
:10A65000810491042CF070E2672E712C812C912CD6
:10A6600030EE63163FEF73063FEF83063FEF93062E
:10A6700044F460EE662E6FEF762E6FEF862E6FEF4E
:10A68000962E41E2A416B104C104D1042CF050E28C
:10A69000A52EB12CC12CD12C50EEA5165FEFB5061E
:10A6A0005FEFC5065FEFD50644F440EEA42E4FEFF2
:10A6B000B42E4FEFC42E4FEFD42E809141049091D1
:10A6C0004204A0914304B091440486199709A80953
:10A6D000B9098093410490934204A0934304B0933A
:10A6E00044048091390490913A04A0913B04B091C4
:10A6F0003C048A199B09AC09BD09809339049093E5
:10A700003A04A0933B04B0933C04809115039091CC
:10A7100016038F3F910509F008F4C4C56F856623C1
:10A7200009F04EC58091E903882309F049C580915D
:10A730001D04882309F044C57091C707788B7723DF
:10A7400009F43EC58091480990914909A0914A09B0
:10A75000B0914B09B7FF04C081509F4FAF4FBF4F1F
:10A76000E92EFA2E0B2F112707FD1A95E0924809C2
:10A77000F092490900934A0910934B0980915009BE
:10A7800090915109A0915209B0915309B7FF04C0AB
:10A7900081509F4FAF4FBF4F892F9A2FAB2FBB27B1
:10A7A000A7FDBA95898B9A8BAB8BBC8B8093500994
:10A7B00090935109A0935209B093530980919F0738
:10A7C000A82EBB24CC24DD242091510430915204C6
:10A7D0004091530450915404C601B5010E949591D3
:10A7E00097FF04C061507F4F8F4F9F4F672E782E89
:10A7F000892E992487FC9A94609251047092520495
:10A80000809253049092540420914D0430914E0450
:10A8100040914F0450915004C601B5010E9495919A
:10A8200097FF04C061507F4F8F4F9F4F272E382EC8
:10A83000492E552447FC5A9420924D0430924E04E0
:10A8400040924F04509250048091490490914A04E0
:10A85000A0914B04B0914C04B7FF04C081509F4FAE
:10A86000AF4FBF4F892F9A2FAB2FBB27A7FDBA95AC
:10A870008093490490934A04A0934B04B0934C04F2
:10A88000D801C70186199709A809B90980939E04C0
:10A8900090939F04A093A004B093A1042091C607B5
:10A8A000E22EFF2400271127BC01CD01A80197014A
:10A8B0000E94099259016A012093AC043093AD04BF
:10A8C0004093AE045093AF0489899A89AB89BC89BF
:10A8D00082199309A409B5098093A2049093A30453
:10A8E000A093A404B093A504BC01CD01A8019701D5
:10A8F0000E9409922093B0043093B1044093B204B3
:10A900005093B304D601C501D7FE04C081509F4FB8
:10A91000AF4FBF4F892F9A2FAB2FBB27A7FDBA95FB
:10A920009093EE038093ED0357FF04C021503F4FF7
:10A930004F4F5F4FBB2757FDBA95A52F942F832FFD
:10A940009093F0038093EF038091D4039091D5030B
:10A9500081349105DCF48091D2039091D30381344A
:10A960009105A4F480918707E82FFF27EE0FFF1FC2
:10A97000E954F74F808191810190F081E02DF7FF3C
:10A9800003C0F095E195FF4F7A97E4F08091000ABB
:10A990008F3FC1F48091ED039091EE0397FD0196F6
:10A9A000959587959093EE038093ED038091EF0347
:10A9B0009091F00397FD0196959587959093F003FC
:10A9C0008093EF0380913F0990914009A091410944
:10A9D000B0914209B7FF04C081509F4FAF4FBF4FA6
:10A9E000892F9A2FAB2FBB27A7FDBA9580933F09DC
:10A9F00090934009A0934109B09342098091300996
:10AA000090913109A0913209B0913309B7FF04C088
:10AA100081509F4FAF4FBF4F892F9A2FAB2FBB272E
:10AA2000A7FDBA958093300990933109A09332091C
:10AA3000B09333098091610490916204A091630402
:10AA4000B09164042F81388549855A85281B390BBC
:10AA50004A0B5B0B20939604309397044093980421
:10AA6000509399048091590490915A04A0915B04E9
:10AA7000B0915C04EB84FC840D851E85E81AF90A0C
:10AA80000A0B1B0BE0929A04F0929B0400939C0427
:10AA900010939D0420939E0430939F044093A00440
:10AAA0005093A104E092A204F092A3040093A404A2
:10AAB0001093A50480913D0490913E04A0913F0421
:10AAC000B0914004821B930BA40BB50B80933D0403
:10AAD00090933E04A0933F04B093400480913504CA
:10AAE00090913604A0913704B09138048E199F09D3
:10AAF000A00BB10B8093350490933604A0933704D8
:10AB0000B093380488898823E1F020911B043091A8
:10AB10001C04213831054CF080917204909173042B
:10AB20000196909373048093720420583F4F4CF425
:10AB300080917204909173040197909373048093B1
:10AB4000720410921C0410921B0481E090E0909318
:10AB5000B9048093B804E0909E04F0909F040091A3
:10AB6000A0041091A104D801C70117FF07C08827CE
:10AB70009927DC018E199F09A00BB10B81509240DF
:10AB8000A040B04034F084E090E09093B90480930A
:10AB9000B8048091BE049091BF04A091C004B0910C
:10ABA000C104209148093091490940914A095091C6
:10ABB0004B09821B930BA40BB50B815E914BAF4FDE
:10ABC000BF4F8F539C49A040B04028F08091010AAC
:10ABD00089310CF4FFC021E0E21620E1F20620E00A
:10ABE000020720E012070CF473C08091BA04882396
:10ABF00009F46AC0D801C70117FF07C08827992741
:10AC0000DC018E199F09A00BB10B9C01AD01B7FFB0
:10AC100004C021503E4F4F4F5F4FF9E05595479587
:10AC200037952795FA95D1F78091B8049091B9049A
:10AC3000820F931F9093B9048093B804D801C70181
:10AC400017FF03C00796A11DB11DE3E0B595A795B9
:10AC500097958795EA95D1F78093AC049093AD04CE
:10AC6000A093AE04B093AF0489589341A040B04084
:10AC700064F088E893E1A0E0B0E08093AC049093A6
:10AC8000AD04A093AE04B093AF042091AC04309116
:10AC9000AD044091AE045091AF0457FF04C0215061
:10ACA0003F4F4F4F5F4F232F342F452F552747FDE1
:10ACB0005A958091ED039091EE03820F931F90932C
:10ACC000EE038093ED0306C081E08093BA0402C0D6
:10ACD0001092BA0440E0E41640EFF4064FEF040788
:10ACE0004FEF14070CF073C08091BB04882309F464
:10ACF0006AC0D801C70117FF07C088279927DC0160
:10AD00008E199F09A00BB10B9C01AD01B7FF04C0C8
:10AD100021503E4F4F4F5F4F69E05595479537950E
:10AD200027956A95D1F78091B8049091B904820F64
:10AD3000931F9093B9048093B804D801C70117FFFB
:10AD400003C00796A11DB11D23E0B595A795979562
:10AD500087952A95D1F78093AC049093AD04A09386
:10AD6000AE04B093AF0488579C4EAF4FBF4F64F40E
:10AD700088E79CEEAFEFBFEF8093AC049093AD04F7
:10AD8000A093AE04B093AF042091AC043091AD0415
:10AD90004091AE045091AF0457FF04C021503F4F83
:10ADA0004F4F5F4F232F342F452F552747FD5A957F
:10ADB0008091ED039091EE03820F931F9093EE0329
:10ADC0008093ED0311C081E08093BB040DC010920D
:10ADD000BB040AC01092B9041092B80484E690E053
:10ADE00090938501809384016889262F3327809171
:10ADF000B8049091B9042817390724F43093B904A2
:10AE00002093B8041091010A112379F0212F3327E0
:10AE100027FD30958091B8049091B904281739071F
:10AE200024F43093B9042093B80440919E045091C7
:10AE30009F046091A0047091A104413851056105FF
:10AE4000710574F080917604909177042091B80494
:10AE50003091B904820F931F909377048093760406
:10AE600040585F4F6F4F7F4F74F4809176049091FC
:10AE700077042091B8043091B904821B930B90930E
:10AE800077048093760481E090E09093B9048093F6
:10AE9000B804C090A204D090A304E090A404F09061
:10AEA000A504D701C601F7FE07C088279927DC0152
:10AEB0008C199D09AE09BF0981509240A040B04055
:10AEC00034F084E090E09093B9048093B8048091CA
:10AED000C2049091C304A091C404B091C504209110
:10AEE0005009309151094091520950915309821BE8
:10AEF000930BA40BB50B815E914BAF4FBF4F8F539C
:10AF00009C49A040B04018F019310CF4FFC001E09A
:10AF1000C01600E1D00600E0E00600E0F0060CF408
:10AF200073C08091BC04882309F46AC0D701C601AC
:10AF3000F7FE07C088279927DC018C199D09AE0907
:10AF4000BF099C01AD01B7FF04C021503E4F4F4FD8
:10AF50005F4F09E055954795379527950A95D1F7A5
:10AF60008091B8049091B904820F931F9093B90413
:10AF70008093B804D701C601F7FE03C00796A11D50
:10AF8000B11D13E0B595A795979587951A95D1F7BB
:10AF90008093B0049093B104A093B204B093B3042F
:10AFA00089589341A040B04064F088E893E1A0E064
:10AFB000B0E08093B0049093B104A093B204B09336
:10AFC000B3042091B0043091B1044091B204509187
:10AFD000B30457FF04C021503F4F4F4F5F4F232F03
:10AFE000342F452F552747FD5A958091EF039091B7
:10AFF000F003820F931F9093F0038093EF0306C03A
:10B0000081E08093BC0402C01092BC0420E0C21610
:10B0100020EFD2062FEFE2062FEFF2060CF073C0FE
:10B020008091BD04882309F46AC0D701C601F7FEE8
:10B0300007C088279927DC018C199D09AE09BF0933
:10B040009C01AD01B7FF04C021503E4F4F4F5F4FF1
:10B05000E9E05595479537952795EA95D1F7809181
:10B06000B8049091B904820F931F9093B904809310
:10B07000B804D701C601F7FE03C00796A11DB11D94
:10B0800073E0B595A795979587957A95D1F78093B5
:10B09000B0049093B104A093B204B093B304885762
:10B0A0009C4EAF4FBF4F64F488E79CEEAFEFBFEF0D
:10B0B0008093B0049093B104A093B204B093B3040E
:10B0C0002091B0043091B1044091B2045091B30486
:10B0D00057FF04C021503F4F4F4F5F4F232F342F56
:10B0E000452F552747FD5A958091EF039091F00326
:10B0F000820F931F9093F0038093EF0311C081E0C0
:10B100008093BD040DC01092BD040AC01092B90412
:10B110001092B80484E690E09093850180938401B6
:10B120004889242F33278091B8049091B9042817B7
:10B13000390724F43093B9042093B8048091010AAC
:10B14000882379F0282F332727FD30958091B80484
:10B150009091B9042817390724F43093B904209347
:10B16000B8044091A2045091A3046091A40470918A
:10B17000A504413851056105710574F0809174048E
:10B18000909175042091B8043091B904820F931FF7
:10B19000909375048093740440585F4F6F4F7F4FB6
:10B1A000CCF480917404909175042091B80430918E
:10B1B000B904821B930B90937504809374040AC0A6
:10B1C0001092F0031092EF031092EE031092ED0331
:10B1D00010921D0480915609882341F41092F003C7
:10B1E0001092EF031092EE031092ED038091480944
:10B1F00090914909A0914A09B0914B098093BE04EE
:10B200009093BF04A093C004B093C10480915009EF
:10B2100090915109A0915209B09153098093C204B1
:10B220009093C304A093C404B093C5041092510436
:10B2300010925204109253041092540410924D0430
:10B2400010924E0410924F04109250041092490430
:10B2500010924A0410924B0410924C041092480928
:10B260001092490910924A0910924B091092500904
:10B2700010925109109252091092530910923F09ED
:10B28000109240091092410910924209109230091F
:10B29000109231091092320910923309109216035C
:10B2A00010921503E0901304F0901404C701F7FE08
:10B2B00004C0882799278E199F0904973CF0809134
:10B2C000700984FD03C082E38093F10310919C0711
:10B2D000A12EBB24CC24DD24B701882777FD8095DF
:10B2E000982F9701F7FE04C0222733272E193F0914
:10B2F000442737FD4095542F0E9495919B01AC0146
:10B30000C601B5010E94959197FF04C061507E4F20
:10B310008F4F9F4F59E095958795779567955A95EB
:10B32000D1F79B01812F99278E9DD0018F9DB00D64
:10B330009E9DB00D1124CD01B7FD0396959587957F
:10B3400095958795280F391F8091F3039091F40309
:10B35000280F391F442737FD4095542F209392041E
:10B360003093930440939404509395048091310456
:10B3700090913204A0913304B0913404821B930B5A
:10B38000A40BB50B8093310490933204A093330443
:10B39000B09334048155934CA040B04064F080E5F4
:10B3A00093ECA0E0B0E08093310490933204A0933A
:10B3B0003304B09334048091310490913204A0910D
:10B3C0003304B0913404805B9C43AF4FBF4F64F4AF
:10B3D00080EB9CE3AFEFBFEF809331049093320496
:10B3E000A0933304B0933404009188011091890133
:10B3F00017FDFCC08091700983FFF8C08091870120
:10B40000815080938701882309F0F4C08DE08093F8
:10B4100087018091610490916204A0916304B091CE
:10B420006404B7FF04C081509E4FAF4FBF4F39E057
:10B43000B595A795979587953A95D1F77C0197FF94
:10B4400004C0F094E194F108F39480915904909130
:10B450005A04A0915B04B0915C04B7FF04C0815012
:10B460009E4FAF4FBF4F29E0B595A795979587950C
:10B470002A95D1F79C0197FF03C0309521953F4F46
:10B48000E216F3060CF47901B701F7FE02C0695F1A
:10B490007F4F2B01A3E055944794AA95E1F722E052
:10B4A00030E0420E531E60908009709081098090B8
:10B4B00082099090830920913C0130913D01409197
:10B4C0003E0150913F01C401B3010E94099259010C
:10B4D0006A0130932E0920932D09021B130BC8011A
:10B4E000845E9D4F68E671E00E94D4919C01245BCC
:10B4F00030408091840190918501009731F001974F
:10B5000090938501809384011BC049E1E416F10406
:10B51000BCF480911B0490911C04820F931F9093A4
:10B520001C0480931B048091F103882349F081500F
:10B530008093F103882321F4B0922004A0921F0489
:10B540008091840190918501892BF9F48091860185
:10B550009927289FB001299F700D389F700D1124E5
:10B56000CB01B2010E94D491CB01AA2797FDA095EF
:10B57000BA2F680E791E8A1E9B1E609280097092F7
:10B58000810980928209909283098091F103882336
:10B5900069F580911F049091200420912D0930912C
:10B5A0002E09821B930B845E9D4F68E671E00E941A
:10B5B000D4919C01245B304080917001869599273D
:10B5C000289FD001299FB00D389FB00D11249D01F7
:10B5D000B7FF02C0215F3F4FF4E035952795FA95FC
:10B5E000E1F73093F4032093F30304C01092F403C3
:10B5F0001092F30380911D04882381F0109225049A
:10B600001092260410922704109228041092290404
:10B6100010922A0410922B0410922C04F090EA034A
:10B62000FF20F1F480915609282F3327442755270E
:10B630008091610490916204A0916304B0916404CC
:10B64000BC01CD010E949591DC01CB01BC01CD0173
:10B6500028EF3AE240E050E00E940992390102C02E
:10B6600066247724E090E903EE20F1F480915609F6
:10B67000282F3327442755278091590490915A0445
:10B68000A0915B04B0915C04BC01CD010E94959136
:10B69000DC01CB01BC01CD0128EF3AE240E050E0F3
:10B6A0000E940992290102C04424552480912A094C
:10B6B00090912B09893C91051CF088EC90E005C025
:10B6C00088539F4F34F488E39FEF90932B09809326
:10B6D0002A098091360990913709893C91051CF01F
:10B6E00088EC90E005C088539F4F34F488E39FEFC7
:10B6F00090933709809336098091380990913909E0
:10B70000AA2797FDA095BA2F20917E09A22EBB24CF
:10B71000CC24DD24BC01CD01A60195010E949591A8
:10B720009B01AC0180912A0990912B09AA2797FDD2
:10B73000A095BA2FE7E0880F991FAA1FBB1FEA95B3
:10B74000D1F7280F391F4A1F5B1F57FF04C0215C28
:10B750003F4F4F4F5F4F76E055954795379527956B
:10B760007A95D1F78301020F131F109339090093C3
:10B7700038098091280990912909AA2797FDA09559
:10B78000BA2FBC01CD01A60195010E9495919B01A4
:10B79000AC018091360990913709AA2797FDA095B1
:10B7A000BA2F67E0880F991FAA1FBB1F6A95D1F7B0
:10B7B000280F391F4A1F5B1F57FF04C0215C3F4FF2
:10B7C0004F4F5F4FF6E05595479537952795FA957A
:10B7D000D1F74201820E931E909229098092280986
:10B7E0008091790990917A09880F991FAA2797FD6E
:10B7F000A095BA2F20912F09332744275527BC0144
:10B80000CD010E9495915B016C0197FF08C02FE369
:10B8100030E040E050E0A20EB31EC41ED51EE6E0AC
:10B82000D594C794B794A794EA95D1F78091450928
:10B83000282F3327442755278091450490914604AB
:10B84000A0914704B0914804BC01CD010E9495919C
:10B85000DC01CB01BC01CD0120EF35E540E050E03B
:10B860000E940992B501620F731F70937A09609369
:10B8700079090150104134F080E090E1909339094A
:10B880008093380980913809909139098050904F00
:10B8900034F480E090EF909339098093380951E0B7
:10B8A000851650E1950634F080E090E190932909E7
:10B8B0008093280980912809909129098050904F00
:10B8C00034F480E090EF9093290980932809615027
:10B8D000704134F080E090E190937A098093790987
:10B8E0008091790990917A098050904F34F480E0EA
:10B8F00090EF90937A098093790980910001482F05
:10B90000552780911F01909120014817590794F401
:10B9100020911F013091200109811A81049FC001EB
:10B92000059F900D149F900D1124B9010E94C091A4
:10B930007A83698329813A81220F331F220F331FB3
:10B940003A8329834091700940FD02C00C94B06491
:10B95000EE2011F00C94B064FF2011F00C94B06450
:10B9600000E010E048018091EB039091EC0390938C
:10B970000B0780930A0720917804309179042115F0
:10B98000310509F03FC08091150190911601895948
:10B99000934058F087B5803F20F48091190381507F
:10B9A00011C081E08093CF044EC080911501909129
:10B9B00016018436910508F587B58031D0F0809165
:10B9C00019038F5F809319039FE08902900111246E
:10B9D00080912F07821B87BD8CE291E09093090331
:10B9E000809308038EE591E0909379048093780426
:10B9F0002AC081E08093CE0426C0F092CE04F0925B
:10BA0000CF0421C08091010490910204A09103040D
:10BA1000B091040464E0880F991FAA1FBB1F6A95A8
:10BA2000D1F780931A0390931B03A0931C03B09348
:10BA30001D031093180300931703215030403093D7
:10BA40007904209378042091730141FF3CC0223394
:10BA500048F580918A01815080938A018F3F09F0D7
:10BA600052C080919D01882339F480911E0488235F
:10BA700019F088E280939D0110921E0480910104C8
:10BA800090910204A0910304B09104048093FD03FB
:10BA90009093FE03A093FF03B093000481E0809392
:10BAA0008A0131C0273478F180919D01882339F4CF
:10BAB00080911E04882319F487E280939D0188EC0D
:10BAC00080938A011DC08091400190914101820FB5
:10BAD000911D209195073327829FA001839F500DD0
:10BAE000929F500D1124CA01AA2797FDA095BA2F45
:10BAF0008093FD039093FE03A093FF03B093000493
:10BB000081E080931E048091610490916204A09171
:10BB10006304B0916404E0903C01F0903D01009119
:10BB20003E0110913F01BC01CD01A80197010E9487
:10BB3000099259016A018091590490915A04A09187
:10BB40005B04B0915C04BC01CD01A80197010E9487
:10BB50000992B901C5010E9443845C01CC971CF095
:10BB60005CE3A52EB12CC5010E9441725C0180E20C
:10BB700080933B011092FC031092FB0380911E0402
:10BB8000882309F45FC58091CF0399279C01207118
:10BB9000307084FD57C58091CE0382608093CE03C0
:10BBA00070915409872F992741E0C42ED12CC822C7
:10BBB000D92280FD04C08091700981FD10C0C98028
:10BBC000DA803093C7042093C6043093FC0320939B
:10BBD000FB038091CF03806C8093CF03ABC2809135
:10BBE000CF0381FF7AC200917A0110917B01C801D5
:10BBF0000F962090110430901204821593050CF0DA
:10BC000058C08091CE04882309F053C08091CF039F
:10BC100087FF15C08091CF038F778093CF038091EA
:10BC2000010490910204A0910304B0910404809354
:10BC3000FD039093FE03A093FF03B0930004809153
:10BC4000CF0380648093CF03E0903409EE20F1F0BD
:10BC50008091FD039091FE03A091FF03B091000439
:10BC6000BC01CD0124E630E040E050E00E940992A2
:10BC70008E2D9927AA27BB2782179307A407B507FC
:10BC80002CF4D092FC03C092FB0310C0C101801BB6
:10BC9000910B0F9797FF03C0909581959F4F9093BD
:10BCA000FC038093FB038BE280933B011092F5032E
:10BCB00016C1C8010F9728163906C4F52091CF0484
:10BCC0002223A1F58091CF0386FF15C08091CF0379
:10BCD0008F7B8093CF038091010490910204A09107
:10BCE0000304B09104048093FD039093FE03A0939A
:10BCF000FF03B09300048091CF0380688093CF034B
:10BD0000C101801B910B0F9697FF03C09095819501
:10BD10009F4F909581959F4F9093FC038093FB03D9
:10BD20008DE280933B012093F503D9C08DE380938E
:10BD30003B016091F603662371F12091F703309186
:10BD4000F8034091F9035091FA038091FD0390911B
:10BD5000FE03A091FF03B091000482179307A4078C
:10BD6000B507CCF48091CF0380648093CF03862FF6
:10BD700099279093FC038093FB038AE08093F5035B
:10BD80008EE580933B018091CF0387FFA8C080910F
:10BD9000CF038F7733C0662309F443C02091F703A4
:10BDA0003091F8034091F9035091FA038091FD031B
:10BDB0009091FE03A091FF03B0910004281739076A
:10BDC0004A075B0774F58091CF0380688093CF03A7
:10BDD000862F9927909581959F4F9093FC03809390
:10BDE000FB0386EF8093F50386E780933B01809108
:10BDF000CF0386FF74C08091CF038F7B8093CF03E6
:10BE00008091010490910204A0910304B091040474
:10BE10008093FD039093FE03A093FF03B09300046F
:10BE20005EC08091CF03807C09F459C08091F503F6
:10BE3000882379F5E0900104F09002040091030456
:10BE400010910404D801C70180589040A040B04030
:10BE50002091FD033091FE034091FF0350910004B7
:10BE600082179307A407B5075CF4D801C70180586F
:10BE70009F4FAF4FBF4F281739074A075B075CF04A
:10BE80008093FD039093FE03A093FF03B0930004FF
:10BE900002C01092F5038091CF038F738093CF037C
:10BEA0001092C7041092C60471FF06C084EF91E09F
:10BEB000909309038093080380910504882379F403
:10BEC0008091010490910204A0910304B0910404B4
:10BED000C397A105B1051CF081E080930504609132
:10BEE000C6047091C7048091FB039091FC03680F16
:10BEF000791F7093C7046093C604CB0177FF04C019
:10BF000088279927861B970B855F91400CF4CEC03C
:10BF10004091F503442389F18091F7039091F80350
:10BF20002091FD033091FE03821B930B09964397EA
:10BF300048F48091F7039091F803A091F903B09130
:10BF4000FA0312C0242F332727FD3095432F532F98
:10BF50008091FD039091FE03A091FF03B091000436
:10BF6000820F931FA41FB51F8093FD039093FE03C0
:10BF7000A093FF03B093000424C080919507209103
:10BF8000FD033091FE034091FF035091000416160B
:10BF9000170644F463E00E94B491280F311D411D3F
:10BFA000511D07C063E00E94B491281B310941096B
:10BFB00051092093FD033093FE034093FF035093F8
:10BFC00000041092C7041092C604E0900104F0909F
:10BFD00002040091030410910404D801C7018050A9
:10BFE0009440A040B0402091FD033091FE03409169
:10BFF000FF035091000482179307A407B5075CF470
:10C00000D801C70180509C4FAF4FBF4F2817390749
:10C010004A075B0744F08093FD039093FE03A093CF
:10C02000FF03B09300048091540981FF06C084E6A9
:10C0300090E09093090380930803809199078823E7
:10C04000A9F58091F603882389F54091EB0350917F
:10C05000EC0357FF02C04D5F5F4F559547955595CF
:10C06000479580911F019091200120910001332775
:10C07000489FF001499FF00D589FF00D1124CF010A
:10C08000B9010E94D49170937B0160937A01663468
:10C0900071051CF486E490E005C06739710534F041
:10C0A00086E990E090937B0180937A0180917804F7
:10C0B00090917904892BD1F180910104909102042F
:10C0C000A0910304B09104048093FD039093FE03B8
:10C0D000A093FF03B093000429C0809101049091C4
:10C0E0000204A0910304B091040480599140A0403F
:10C0F000B0408093FD039093FE03A093FF03B093A1
:10C10000000480919907882311F0992702C088E7DD
:10C1100090E090937B0180937A01E980FA80F0921D
:10C12000EC03E092EB038EE280933B01C090EB03C3
:10C13000D090EC03E0900104F0900204009103041D
:10C14000109104042091FD033091FE034091FF0300
:10C15000509100042E153F054007510724F08091AF
:10C16000540980FDBBC28091780490917904892B99
:10C1700039F0C090EB03D090EC0300E010E0D7C0A2
:10C18000D801C701821B930BA40BB50B80939604B7
:10C1900090939704A0939804B0939904823000E898
:10C1A00090070FEFA0070FEFB0072CF481E090E8A5
:10C1B000AFEFBFEF09C08F5F9F47A040B04064F072
:10C1C0008FEF9FE7A0E0B0E08093960490939704F0
:10C1D000A0939804B0939904009196041091970449
:10C1E00080917201282F3327442755278091960488
:10C1F00090919704A0919804B0919904BC01CD014D
:10C200000E94959197FF04C0615E7F4F8F4F9F4FB3
:10C2100025E095958795779567952A95D1F7609351
:10C2200096047093970480939804909399046530D2
:10C230002EEF72072FEF82072FEF92072CF484E086
:10C240009EEFAFEFBFEF09C0605074408040904058
:10C2500064F080E094E0A0E0B0E0809396049093D6
:10C260009704A0939804B0939904809096049090BA
:10C270009704209117033091180337FF02C0295FFC
:10C280003F4F83E0359527958A95E1F74FEF2238A8
:10C2900034071CF421E83FEF05C02038310514F0C5
:10C2A00020E830E0C901AA2797FDA095BA2F209178
:10C2B0007401332744275527BC01CD010E94959175
:10C2C00097FF04C06D5F7F4F8F4F9F4FB2E09595F2
:10C2D000879577956795BA95D1F79B015FEF6130A8
:10C2E00075071CF420E03FEF06C06F3F710519F0A1
:10C2F00014F020E031E08091CF03807C49F0C90147
:10C3000037FD03969C0135952795359527950DC0EA
:10C310008091540980FF09C0C90137FD07969C012F
:10C32000F3E035952795FA95E1F7820E931E20915B
:10C330007101222309F454C06091210470912204F8
:10C34000809123049091240497FF04C061587F4F8B
:10C350008F4F9F4FE7E09595879577956795EA957D
:10C36000D1F73327442755270E94959197FF04C0A2
:10C37000615E7F4F8F4F9F4F55E0959587957795DD
:10C3800067955A95D1F760939604709397048093BC
:10C390009804909399046138AFEF7A07AFEF8A075A
:10C3A000AFEF9A072CF480E89FEFAFEFBFEF0AC022
:10C3B0006F3F71058105910569F064F080E091E0BF
:10C3C000A0E0B0E08093960490939704A093980423
:10C3D000B09399048091960490919704880E991EC9
:10C3E00080916F01282F33278091040A992787FDB8
:10C3F0009095289FF001299FF00D389FF00D112492
:10C400009F01F7FF02C021583F4F220F232F221F09
:10C41000330BFFEF21383F071CF420E83FEF06C045
:10C420002F3F310519F014F020E031E0820E931E09
:10C43000C401AA2797FDA095BA2FE090EB03F090D6
:10C44000EC039701442737FD4095542FBC01CD01E3
:10C450000E94959197FF04C061507E4F8F4F9F4F70
:10C4600029E095958795779567952A95D1F7C61A0E
:10C47000D70A8091FB039091FC03892B09F060C0DF
:10C480001E141F040CF05CC0980117FF03C0309508
:10C4900021953F4F2D33310540F48091190490913F
:10C4A0001A048C159D0574F526C02C53304085E088
:10C4B000369527958A95E1F72031310510F02FE068
:10C4C00030E04091190450911A0410161106E4F45A
:10C4D00080E190E0821B930B489F9001499F300DB3
:10C4E000589F300D1124B4E036952795BA95E1F7A1
:10C4F0002C153D0520F58091780190917901C816A1
:10C50000D906F4F06C011CC0205F3F4F8091780188
:10C5100090917901829F8001839F100D929F100D51
:10C5200011249801A4E036952795AA95E1F74C15BA
:10C530005D0514F06A0104C0C216D30608F0690153
:10C54000C601AA2797FDA095BA2FFDE0880F991F75
:10C55000AA1FBB1FFA95D1F79501442737FD4095D7
:10C56000542FBC01CD010E94099220939A0430936C
:10C570009B0440939C0450939D04C0909A04D090D7
:10C580009B048091C8049091C9049C01220F331F21
:10C59000280F391F2C0D3D1D37FF02C02D5F3F4F67
:10C5A000A90155954795559547955093C9044093D2
:10C5B000C80480919107282F3327220F331F220FA1
:10C5C000331F241735076CF480917809282F3327FF
:10C5D000220F331F220F331F2055304042175307BD
:10C5E00024F03093C9042093C8048091540980FF3B
:10C5F00014C08091C8049091C90429813A8182179E
:10C60000930724F03093C9042093C8044091C804D0
:10C610005091C9045A83498361C029813A812E19F6
:10C620003F0937FF02C02D5F3F4F35952795359560
:10C6300027956091C8047091C904620F731F7A83B3
:10C6400069834CC080919907882301F56091EB03C1
:10C650007091EC0377FF02C06D5F7F4F7595679512
:10C660007595679540911F015091200180910001BF
:10C67000282F3327649FC001659F900D749F900DF4
:10C680001124B9010E94D491CB0101C09927909344
:10C690007B0180937A0180917A0190917B018734AC
:10C6A00091051CF486E490E005C08639910534F0CC
:10C6B00086E990E090937B0180937A0189819A8149
:10C6C0009093C9048093C8048091CF03806C8093B9
:10C6D000CF038091CE038D7F8093CE038091CF03D3
:10C6E00099279C012270307081FF2BC18091CA0470
:10C6F0009091CB04A091CC04B091CD040097A105FA
:10C70000B10521F0809105048130B1F4E981FA810D
:10C71000CF01AA2797FDA095BA2F1EE0880F991F79
:10C72000AA1FBB1F1A95D1F78093CA049093CB041C
:10C73000A093CC04B093CD0480910504813019F40A
:10C7400082E080930504E980FA80C701AA2797FD5B
:10C75000A095BA2F9501442737FD4095542FBC0171
:10C76000CD010E949591DC01CB0180939A049093B6
:10C770009B04A0939C04B0939D04B7FF04C0815018
:10C78000904EAF4FBF4F7C018D01ADE015950795E1
:10C79000F794E794AA95D1F7E0929A04F0929B045B
:10C7A00000939C0410939D046091D0037091D10379
:10C7B0002FE0603A720750F58091CA049091CB0443
:10C7C000A091CC04B091CD049C01AD01FAE0569546
:10C7D000479537952795FA95D1F7821B930BA40BB4
:10C7E000B50BA8019701E4E0220F331F441F551F2A
:10C7F000EA95D1F7820F931FA41FB51F8093CA0437
:10C800009093CB04A093CC04B093CD0460547F41AB
:10C8100018F58091CA049091CB04A091CC04B091FA
:10C82000CD049C01AD016CE0569547953795279551
:10C830006A95D1F7821B930BA40BB50BA801970146
:10C84000F2E0220F331F441F551FFA95D1F7820FD4
:10C85000931FA41FB51F38C0809117039091180330
:10C86000809117039091180397FF03C090958195CD
:10C870009F4F8436910584F58091010490910204C4
:10C880002091FD033091FE03821B930B81509F4F3B
:10C890008F5F914008F58091CA049091CB04A091DC
:10C8A000CC04B091CD049C01AD01EEE056954795C6
:10C8B00037952795EA95D1F7821B930BA40BB50BFF
:10C8C0008E0D9F1DA01FB11F8093CA049093CB04AF
:10C8D000A093CC04B093CD048091CA049091CB0472
:10C8E000A091CC04B091CD047EE0B695A795979524
:10C8F00087957A95D1F79093EC038093EB03409161
:10C900009707442399F055279C01BA010E94D491BE
:10C91000C901861B970B90931A0480931904260F64
:10C92000371F30937901209378011FC010921A04A9
:10C93000109219048FEF93E090937901809378011E
:10C9400014C0109205041092CA041092CB041092E5
:10C95000CC041092CD043093EC032093EB0305C07C
:10C960008091CF03806C8093CF038091DE0481FFA0
:10C9700037C089819A8197FD0396959587959595FE
:10C9800087952091CC033091CD032817390760F4A7
:10C990008091EB039091EC03892B31F0220F331F30
:10C9A000220F331F3A83298380910104909102045E
:10C9B000A0910304B09104048093FD039093FE03BF
:10C9C000A093FF03B093000488E99AE390930903CE
:10C9D0008093080380E09EE090930A018093090110
:10C9E00020913D09822F9927880F991F880F991F41
:10C9F000889669817A818617970714F09A838983CC
:10CA0000709178097D8B872F9927880F991F880F40
:10CA1000991F80559040A981BA818A179B0714F409
:10CA20009A83898380914E03882341F48091160A6A
:10CA30008F3F21F48091E2048823E9F08091D003B4
:10CA40009091D1030297C097B0F4E981FA811E1644
:10CA50001F068CF481E090E09093D1038093D00383
:10CA6000E22EFF24EE0CFF1CEE0CFF1C8701085D7C
:10CA70001F4F1A83098329813A813093EF0620934F
:10CA8000EE068091920490919304A0919404B09149
:10CA9000950412E0880F991FAA1FBB1F1A95D1F7A2
:10CAA0000091790910917A09081B190B213A310577
:10CAB0008CF0C90137FD01969595879580179107F0
:10CAC0000CF48C01909581959F4F081719076CF411
:10CAD0008C010BC00135110514F000E510E03FEFAB
:10CAE000003B130714F400EB1FEF4D89242F33276D
:10CAF000220F331F220F331FC90169817A81861BE0
:10CB0000970B801791070CF48C0189819A81821B05
:10CB1000930B081719070CF48C0180913809909138
:10CB200039096091170470911804861B970B909334
:10CB3000470980934609D0905609209129043091E5
:10CB40002A0440912B0450912C04DD2041F0661AF8
:10CB5000770AC301AA2797FDA095BA2F04C0AA2778
:10CB600097FDA095BA2F280F391F4A1F5B1F2093EE
:10CB7000290430932A0440932B0450932C04809171
:10CB8000290490912A04A0912B04B0912C04815087
:10CB90009A4FA040B04064F080E09AEFA0E0B0E08F
:10CBA0008093290490932A04A0932B04B0932C041F
:10CBB0008091290490912A04A0912B04B0912C0417
:10CBC00080509640AF4FBF4F64F480E096E0AFEFE7
:10CBD000BFEF8093290490932A04A0932B04B09371
:10CBE0002C04C090A607209146093091470978E0AF
:10CBF000E72EEC1498F08C2D9927829FA001839F3B
:10CC0000500D929F500D1124CA0157FD07967C01CB
:10CC100063E0F594E7946A95E1F712C08C2D869550
:10CC20009927829FB001839F700D929F700D1124F0
:10CC3000CB0177FD03967C01F594E794F594E79496
:10CC4000A0907501B09076019501442737FD40957D
:10CC5000542F8091290490912A04A0912B04B09123
:10CC60002C04BC01CD010E940992E20EF31E9090AB
:10CC70006101692D772788279927980117FF04C03C
:10CC800022273327201B310B37FF02C02F5F3F4F76
:10CC900035952795A981BA812A0F3B1F442737FD77
:10CCA0004095542F0E94959197FF04C0615C7F4F7F
:10CCB0008F4F9F4F26E095958795779567952A9595
:10CCC000D1F79B016E157F050CF47B013095219502
:10CCD0003F4FE216F3060CF47901809128099091F8
:10CCE00029096091150470911604861B970B909387
:10CCF000270980932609209125043091260440912C
:10CD0000270450912804DD2041F0461A570AC20139
:10CD1000AA2797FDA095BA2F04C0AA2797FDA09532
:10CD2000BA2F280F391F4A1F5B1F20932504309309
:10CD30002604409327045093280480912504909161
:10CD40002604A0912704B091280481509A4FA04056
:10CD5000B04064F080E09AEFA0E0B0E0809325045A
:10CD600090932604A0932704B0932804809125046F
:10CD700090912604A0912704B091280480509640F9
:10CD8000AF4FBF4F64F480E096E0AFEFBFEF80930A
:10CD9000250490932604A0932704B093280420919F
:10CDA00026093091270948E04C1598F08C2D9927D9
:10CDB000829FB001839F700D929F700D1124CB0153
:10CDC00077FD07966C01B3E0D594C794BA95E1F767
:10CDD00012C0C6948C2D9927829FD001839FB00DDD
:10CDE000929FB00D1124CD01B7FD03966C01D5942F
:10CDF000C794D594C7949501442737FD4095542F87
:10CE00008091250490912604A0912704B0912804D4
:10CE1000BC01CD010E940992C20ED31E692D772755
:10CE200088279927980117FF04C022273327201B42
:10CE3000310B37FF02C02F5F3F4F35952795E981B2
:10CE4000FA812E0F3F1F442737FD4095542F0E9433
:10CE5000959197FF04C0615C7F4F8F4F9F4FE6E035
:10CE60009595879577956795EA95D1F79B016C1510
:10CE70007D050CF46B01309521953F4FC216D3060A
:10CE80000CF4690180913D09282E33245090E80765
:10CE900066E5862E68E0962E5DE0A52E58E0B52E5C
:10CEA0004BE0442E37E5632E39E0732ED5012C91EB
:10CEB00012160CF029C1203429F4E981FA81FF8B84
:10CEC000EE8B1FC049815A81CA01AA2797FDA09500
:10CED000BA2F332727FD3095432F532FBC01CD01A7
:10CEE0000E94959197FF04C0615C7F4F8F4F9F4FC9
:10CEF00026E095958795779567952A95D1F77F8B4D
:10CF00006E8BF5012181203439F42E893F892E0D55
:10CF10003F1D3F8B2E8B2AC0203C39F44E895F8900
:10CF20004E195F095F8B4E8B21C0C701AA2797FD61
:10CF3000A095BA2F332727FD3095432F532FBC01DF
:10CF4000CD010E94959197FF04C0615C7F4F8F4F88
:10CF50009F4FB6E09595879577956795BA95D1F7E8
:10CF6000AE89BF89A60FB71FBF8BAE8BF50122819B
:10CF7000203439F42E893F892C0D3D1D3F8B2E8B9B
:10CF80002AC0203C39F44E895F894C195D095F8BBA
:10CF90004E8B21C0C601AA2797FDA095BA2F332733
:10CFA00027FD3095432F532FBC01CD010E94959151
:10CFB00097FF04C0615C7F4F8F4F9F4FA6E0959510
:10CFC000879577956795AA95D1F7AE89BF89A60F02
:10CFD000B71FBF8BAE8BF5012381203439F42E8926
:10CFE0003F89200F311F3F8B2E8B2AC0203C39F404
:10CFF0004E895F89401B510B5F8B4E8B21C0C8014E
:10D00000AA2797FDA095BA2F332727FD3095432FE8
:10D01000532FBC01CD010E94959197FF04C0615C24
:10D020007F4F8F4F9F4FF6E0959587957795679542
:10D03000FA95D1F7AE89BF89A60FB71FBF8BAE8B0C
:10D04000F301808191812E893F898217930764F4CF
:10D05000B901680F791F77FF02C06F5F7F4F759529
:10D0600067957F8B6E8B1DC0552049F44E895F8973
:10D07000440F551F481B590B5F8B4E8B12C051E05C
:10D08000551578F4252D33276E897F89861B970BDC
:10D09000B9010E94D491AE89BF89A60FB71FBF8B7B
:10D0A000AE8BC101880F991F880F991FEE89FF89E8
:10D0B0008E179F0764F4FD898F2F9927880F991F7A
:10D0C000880F991F2E893F892817390714F09F8BE5
:10D0D0008E8B8E899F8997FD03969595879595955B
:10D0E0008795F4018183880F991F880F991F2E89D6
:10D0F0003F89281B390BC901880F8283EE89FF897C
:10D10000D301ED93FC9303C0F401118212824A947F
:10D1100022E030E0620E731E44E050E0A40EB51E23
:10D1200068E070E0860E971E47FEC0CEE2E1C95E61
:10D130000C94409284B1806A84B93D9A82E58CBD9A
:10D140001DBC459A81E080938A098AEA80939B09F5
:10D1500083E880939C098AE080939D0910929F093F
:10D1600010929E091092A1091092A0091092030A30
:10D170001092BF09089530918A09332309F085C0C0
:10D180000DB407FE82C084E080930703459A2EB554
:10D190008091E50499278130910589F082309105CD
:10D1A0001CF4892B21F03EC00297B9F03BC03093AC
:10D1B000BE092093E6042138A9F581E008C0253591
:10D1C00049F48091E604820F8093E60482E0809324
:10D1D000E50428C03093E50425C08091BE09E82FFE
:10D1E000FF27E052F64F20838F5F8093BE09909116
:10D1F000E6048032A0F0291769F480E2A0EEB9E0DD
:10D20000E0ECF9E00D9001928A95E1F781E08093DE
:10D21000BF0902C03093BF091092E50403C0920F0A
:10D220009093E60420919A09223208F028C045988C
:10D2300000000000000000000000000000000000EE
:10D2400000000000000000000000000000000000DE
:10D2500000000000000000000000000000000000CE
:10D26000E0919309F0919409E20FF11D80818EBD48
:10D270008091BC099081890F8093BC0903C081E033
:10D2800080938A092F5F20939A090895EF92FF9265
:10D290000F931F9380919F079927880F991F880FDD
:10D2A000991F7C010027F7FC0095102F80916104E5
:10D2B00090916204A0916304B0916404BC01CD011B
:10D2C000A80197010E94099230939F0920939E091B
:10D2D0008091590490915A04A0915B04B0915C0430
:10D2E000BC01CD01A80197010E9409923093A109C8
:10D2F0002093A009209180093091810940918209F1
:10D3000050918309DA01C90163E0880F991FAA1FB0
:10D31000BB1F6A95D1F7820F931FA41FB51F820F01
:10D32000931FA41FB51F20913C0130913D014091F6
:10D330003E0150913F01BC01CD010E940992309302
:10D34000A7092093A60980917204909173042091FB
:10D35000240330912503821B930B9093AD09809396
:10D36000AC09E0916804F091690480914D099091B5
:10D370004E09BF010E94D4919B01220F331F220F3F
:10D38000331F260F371F260F371F37FF02C02D5FB1
:10D390003F4F35952795359527953093A3092093D1
:10D3A000A20980917C0990917D09BF010E94D491CE
:10D3B0009B01220F331F220F331F260F371F260F0B
:10D3C000371F37FF02C02D5F3F4F359527953595A5
:10D3D00027953093A5092093A4091092690410920F
:10D3E000680410924E0910924D0910927D09109216
:10D3F0007C0980919D099927AA27BB27FC013A97B0
:10D40000E830F10508F0FEC1E058FF4F0C945B9244
:10D410008091E4038093B0098091E3038093B10984
:10D420008091E2038093B2098091E1038093B30974
:10D430008091E0038093B4098091DF038093B50964
:10D440008091DE038093B6098091DD038093B70954
:10D450008091CF038093B8098091CF03837F80931D
:10D46000CF030E9463308093B9098091E9078093CC
:10D47000BA098091CE03C4C18091100A9091110A1B
:10D480009093B1098093B0098091140A9091150A84
:10D490009093B3098093B20980911F01909120016C
:10D4A0008093B409809100018093B50980913B017C
:10D4B0008093B6099091E7049093B709E92FFF276D
:10D4C000A3E0EE0FFF1FAA95E1F7EA5AF74F868116
:10D4D0008093B80983818093B90987818093BA09C1
:10D4E00085818093BB09892F8F5F6CE00E94B49186
:10D4F0009093E70487C18091D4078093B00980910D
:10D50000D5078093B1098091D6078093B2098091A5
:10D51000D7078093B3098091D8078093B40980918D
:10D52000DC078093B5098091DD078093B60980916F
:10D53000DE078093B7098091E1078093B809809155
:10D54000DF078093B9098091E0078093BA09809141
:10D55000E20756C18091D3078093B0098091AA0752
:10D56000863081F08091D402823451F00E9483731E
:10D57000E82FFF27EB55FF4E84918093D40202C021
:10D580000E94837380910A058093B1093BC1F8948E
:10D5900080918607E82FFF27EE0FFF1FE954F74F12
:10D5A0000190F081E02DE038F1051CF0EFE7F0E0AC
:10D5B00006C02FEFE138F20714F4E1E8FFEFE09343
:10D5C000B00980918707E82FFF27EE0FFF1FE9546E
:10D5D000F74F0190F081E02DE038F1051CF0EFE706
:10D5E000F0E006C07FEFE138F70714F4E1E8FFEF61
:10D5F000E093B10980918507E82FFF27EE0FFF1F09
:10D60000E954F74F0190F081E02DE038F1051CF06E
:10D61000EFE7F0E006C08FEFE138F80714F4E1E837
:10D62000FFEFE093B20980918407E82FFF27EE0F08
:10D63000FF1FE954F74F0190F081E02DE038F1052C
:10D640001CF0EFE7F0E006C02FEFE138F20714F42A
:10D65000E1E8FFEF7894E093B309809108048093A8
:10D66000B409809109048093B50980910A048093DC
:10D67000B60980910B048093B70980910C048093C4
:10D68000B80980910D048093B90980910E048093AC
:10D69000BA0980910F04B4C080916F05863018F0EC
:10D6A00010926F0585E08093B0098091E307809325
:10D6B000B1098091010490910204A0910304B091FA
:10D6C0000404BC01CD0125E030E040E050E00E94C0
:10D6D00009923093B3092093B2098091FD03909190
:10D6E000FE03A091FF03B0910004BC01CD0125E031
:10D6F00030E040E050E00E9409923093B509209359
:10D70000B4098091D9078093B6098091DA07809394
:10D71000B7098091DB078093B80980910704809353
:10D72000B9098091B7089091B8088093BA0980919F
:10D73000EE069091EF0697FD039695958795959542
:10D7400087955EC01092B0098AE58093B10983E0A5
:10D750008093B20984E38093B3098091010180939F
:10D76000B409809154058093B50990915505909323
:10D77000B6098F77809354059071909355058091E9
:10D7800056058093B709809170098093B8098091FC
:10D7900054098093B9098091E5078093BA09809173
:10D7A000F2072EC08091B8078093B0098091F007EE
:10D7B0008093B109809167018093B2098091B1078C
:10D7C0008093B3098091B2078093B4098091B30725
:10D7D0008093B509809166018093B6098091B50761
:10D7E0008093B7098091B6078093B8098091B707F5
:10D7F0008093B9098091160A8093BA09809118071D
:10D800008093BB098091BF09882309F47DC1609191
:10D81000C00980919901681719F08AEF80939701E8
:10D820006093990181E0809387014091C1095091F3
:10D83000C209CA0181509E4F8F5F9340B0F420917E
:10D84000C3093091C409C90181509E4F8F5F934035
:10D8500060F48091900785FF08C05093D4044093F2
:10D86000D3043093D2042093D1048091C7099091BE
:10D87000C80921E08936920724F4909389018093A6
:10D8800088012091D1093091D209809108039091AB
:10D8900009038217930740F48091DC02882321F466
:10D8A0003093090320930803862F99278936910521
:10D8B00009F4A5C08A36910544F48736910571F0C4
:10D8C0008836910509F462C027C18A36910509F4AA
:10D8D00014C18B36910509F4E2C01EC18091D309B1
:10D8E0008093000A8091D4098093020A8091D5091F
:10D8F0008093010A8091D609809386018091D7098F
:10D900008093040A8091D809809398018091D90965
:10D910008093E4048091DA098093D0048091DC0341
:10D920008823F9F02091DB093091DC0937FD19C01B
:10D930003093200420931F049091BA07992389F013
:10D940008FE0989FC0011124281B390BC901885909
:10D950009E4F68E671E00E94D491909320048093DA
:10D960001F042091DB043091DC048091DD0990914B
:10D97000DE09280F391F37FF02C02F5F3F4F359553
:10D9800027953093DC042093DB04C6C08091D30933
:10D99000809395098091D409809396098091D50947
:10D9A000809397098091D609809398098091D7092F
:10D9B000809399098091DE069091D809892B8093F4
:10D9C000DE069091DF0693708091D9098C70982BB8
:10D9D0009093DF068091DA098093E2048091DB095D
:10D9E00080938B018091DC098093030A8091DD098B
:10D9F0008093DE048091DE098093DD048DC08091E8
:10DA0000D30980938B098091D40980938C098091EC
:10DA1000D50980938D098091D60980938E098091D4
:10DA2000D7099091D8099093900980938F0980919C
:10DA3000D9099091DA099093920980939109809184
:10DA4000DB09992787FD90959093EA088093E90870
:10DA50008091DC098093F6038091DD099091DE09C5
:10DA60009C01442737FD4095542FDA01C90163E03A
:10DA7000880F991FAA1FBB1F6A95D1F7820F931FAA
:10DA8000A41FB51F820F931FA41FB51F8093F70318
:10DA90009093F803A093F903B093FA033DC08091EB
:10DAA000D3098093E1048091D4098093E0048091AC
:10DAB000D5098093DF049091D609992349F080918C
:10DAC0009D01882319F08151833010F490939D01BA
:10DAD0008091D70980930F058091D80980930E0516
:10DAE0008091D9099091DA0990930C0580930B05E8
:10DAF0008091DB0980930D050FC08091AA078630C5
:10DB000059F40E94DC7308C01092D4041092D3041C
:10DB10001092D2041092D1041F910F91FF90EF90B8
:10DB2000089580918A09882309F43BC045988BE9C0
:10DB300099E090939409809393099091E304E92FDD
:10DB4000FF27E457FE4F9F5F9093E304808180930B
:10DB50009D099B3010F01092E30410928A090E94F4
:10DB6000466981E080939A090000000000000000EF
:10DB700000000000000000000000000000000000A5
:10DB80000000000000000000000000000000000095
:10DB9000000000000000000080919B098093BC09F8
:10DBA0008EBD089587B18C6087B9429843981092D2
:10DBB000E90480E880939B011092E80480939A0125
:10DBC00008958091EE0481508093EE048F3F09F018
:10DBD00055C189E08093EE048091E9089091EA08AC
:10DBE00081589F4F39F08091E9089091EA08815857
:10DBF0008093F3048091CF03992780739070892BD1
:10DC000021F48091550580FF1DC08091D1078823A4
:10DC100051F08091F104882319F484E08093E904A1
:10DC200081E08093F1048091D2078823B9F080913C
:10DC3000F204882319F484E08093E80481E080935F
:10DC4000F2040CC01092F1041092F2048091CD07FE
:10DC50008093EF048091CF078093F0048091F104CA
:10DC6000882309F073C08091EF07282F332724FF02
:10DC700007C080910604882319F425FD80C081C067
:10DC80009091CE07983F48F080914F098D3D28F044
:10DC90008091EF0488236CF00AC0983F68F080916F
:10DCA0004F09853049F48091EF0487FF02C0429804
:10DCB00001C0429A81E032C08091E9048150809392
:10DCC000E9048F3F09F05EC08091F20785FF29C00B
:10DCD0009091F304892F86958093E904992351F458
:10DCE0008091EF0487FF02C0429801C0429A1092CF
:10DCF0009B0148C080919B019091EF04882341F4DF
:10DD00008093F30480E880939B019923D4F137C07A
:10DD1000982311F0429A01C04298869580939B0106
:10DD200031C080914F0986958093E90480919B01D1
:10DD3000813021F41092F30480E801C0869580932D
:10DD40009B0180919B019091EF0417C08091E904A1
:10DD500081508093E9048F3FA9F489E08093E9041E
:10DD600080919B01813011F480E801C086958093F9
:10DD70009B0180919B019091D107892311F0429AD8
:10DD800001C042988091F204882309F043C0909129
:10DD9000EF0797FF07C080910604882319F496FDCA
:10DDA00052C053C09091D007983F48F080917709B6
:10DDB0008D3D28F08091F00488236CF00AC0983FD4
:10DDC00078F080917709853059F48091F00487FFCD
:10DDD00002C0439801C0439A81E080939A0136C003
:10DDE0008091E80481508093E8048F3F79F5809119
:10DDF000770986958093E80480919A01813011F427
:10DE000080E801C0869580939A0180919A01909153
:10DE1000F00417C08091E80481508093E8048F3F9C
:10DE2000A9F489E08093E80480919A01813011F48B
:10DE300080E801C0869580939A0180919A01909123
:10DE4000D207892311F0439A01C04398429B04C032
:10DE50008091CE03886003C08091CE03877F80933A
:10DE6000CE03439B06C08091CE0380618093CE0396
:10DE700008958091CE038F7E8093CE0308950F93F3
:10DE80001F93CF93DF93482FEB0180910704E42F7A
:10DE9000FF27843BD8F08F010E0F1F1FF801E954B4
:10DEA000F74F808191819B01281B390BC90163E0E9
:10DEB00070E00E94D491CB01880F991F860F971FA5
:10DEC0000551174FF8019183808306C0EE0FFF1FA5
:10DED000E551F74F11821082E42FFF27EE0FFF1F4D
:10DEE000E954F74FD183C083DF91CF911F910F91F8
:10DEF00008954FB724E130E0F8948091C9008F77FE
:10DF00008093C9008091C9008F7B8093C900809164
:10DF1000C9008F7D8093C9005A9A52985B9A539A90
:10DF2000832F99278093CD002093CC008091C80047
:10DF300082608093C80080E18093C9008091CA000C
:10DF40008F778093CA008091CA008F7B8093CA002C
:10DF50008091CA008F7D8093CA008091CA008F7E15
:10DF60008093CA008091CA00877F8093CA00809105
:10DF7000C9008B7F8093C9008091CA008460809320
:10DF8000CA008091CA0082608093CA008091C80054
:10DF900087FF03C08091CE00F9CF8091C9008068CF
:10DFA0008093C9004FBF0895EF92FF920F931F9384
:10DFB000CF93DF93482F00E010E080919C018130E7
:10DFC00061F410929C0184E48093F6041092F804AA
:10DFD0001092F7041092F90403C28091F60488238A
:10DFE00019F421E030E001C098019091F7049923E1
:10DFF00071F4232B11F081E010C084E48093F604C7
:10E000009093F8049093F7049093F904D2C191305F
:10E0100069F4232B09F0C3C182E08093F704809157
:10E02000F8048F5F8093F80483E0C1C19230D1F48B
:10E03000232B09F0B4C183E08093F6044093F904E4
:10E040009091F804923039F41092FA0447FF03C01B
:10E0500081E08093FA0483E08093F7049F5F9093BC
:10E06000F804A7C1933009F09AC1232B09F097C196
:10E070009093F60482E08093F7048091F8048F5F18
:10E080008093F8042091F904822F9927782F66272E
:10E09000842F9927682B792B8091AA07813051F41E
:10E0A0007370CB018050924063E070E00E94D49185
:10E0B000EB0119C0823069F47770CB018050944035
:10E0C00066E070E00E94D491EB0126952695269596
:10E0D0000CC0EB01D370C856D140CE01D7FD0196DC
:10E0E000EC01D595C79526952695022F11270F701F
:10E0F00010700F5F1F4F0D30110508F049C102303D
:10E10000110519F404E010E005C00430110511F404
:10E1100002E010E0D801A00FB11FFD01E954F74F54
:10E12000808191819E01281B390BC90137FF03C0F3
:10E13000909581959F4F069704F5E091EC07EE23AB
:10E1400051F0FF27EE0FFF1FE954F74F80819181B7
:10E150008436910594F480910704883C30F48091D2
:10E160000704865F8093070408C088EC8093070447
:10E1700080916F008F7D80936F00A954B74F8D9170
:10E180009C91BC01660F771F680F791F6C0F7D1F74
:10E1900077FF02C06D5F7F4F7B01F594E794F594A4
:10E1A000E794CE0101968E159F0524F40894E108AA
:10E1B000F10808C0CE010197E816F9061CF408948E
:10E1C000E11CF11C0630110509F0CEC0C536D105A1
:10E1D0000CF4A5C09091F504E92FFF27EB5FF54FF4
:10E1E000E081ED3729F48091F40480958093F40464
:10E1F000963061F48091F404882311F0E338B9F08B
:10E20000882309F088C0ED3791F085C0993009F076
:10E2100082C08091F404882329F480910E0A833807
:10E2200031F079C080910E0A8D3709F074C0809169
:10E23000060A8D3739F48091070A833899F463E828
:10E240007FEF0DC0833871F48091070A833819F489
:10E2500060E070E004C08D3729F46DE770E085E080
:10E260000E943F6F8091080A992787FD9095BC0115
:10E2700086E00E943F6F8091090A992787FD90955B
:10E28000BC018BE00E943F6F80910A0A992787FDAD
:10E290009095BC018CE00E943F6F8091F50489301D
:10E2A000D1F580910C0A8D3749F48091C70890917F
:10E2B000C8080596BC0188E00E943F6F80910D0A56
:10E2C0008D3749F48091C7089091C8080597BC0123
:10E2D00088E00E943F6F8091C7089091C8088358DA
:10E2E0009F4F1CF483E89FEF09C08091C70890916D
:10E2F000C8088E37910534F08DE790E09093C808F8
:10E300008093C70880910B0A992787FD9095BC01DF
:10E310008AE00E943F6F1092F5041092F404CA3014
:10E32000D1055CF48091F5048F5F8093F504E82FAC
:10E33000FF27EB5FF54F83E880838091F5048A30F7
:10E3400011F41092F5048FEFCC39D8076CF480915A
:10E35000F504E82FFF27EB5FF54F8DE78083809171
:10E36000F40480958093F4040530110518F4B70186
:10E37000802F0BC00530110519F4BE0187E005C0E0
:10E3800007301105B1F4BE0189E00E943F6F11C052
:10E390000231110570F081E080939C010AC081E098
:10E3A00080939C011092F8041092FA0484E4809304
:10E3B000F6048091F804803198F08091FA04882363
:10E3C00031F480919C01882311F480933A011092DA
:10E3D000F8041092FA041092F70484E48093F6048F
:10E3E000E6E0CDB7DEB70C944C92CF93FC0197FFDB
:10E3F00005C0CFEFF095E195FF4F01C0C1E028E6E1
:10E4000031E0CF01B9010E94D491FC018B35910517
:10E4100054F08B5590408A35910538F484EB90E0A8
:10E420008E1B9F0BFC0141E00DC0CF01855B90402E
:10E430008A35910518F4E45BF04003C02E1B3F0BB6
:10E44000F9014FEFEE0FFF1FE85BF64F2591349176
:10E450008C2F992787FD9095289FB001299F700DDB
:10E46000389F700D1124842F992787FD9095689F00
:10E47000A001699F500D789F500D1124CA01CF91C2
:10E4800008952AE530E0281B390BC9010E94F57177
:10E4900008950895089508950895089580E090E0FE
:10E4A00008951092110A1092100A1092150A1092F3
:10E4B000140A1092130A1092120A1092160A8AE095
:10E4C00090E00E946F199093FC048093FB040895E0
:10E4D000CF93DF938091FB049091FC040E94781904
:10E4E000882309F4AFC08091FB049091FC040A9644
:10E4F0009093FC048093FB04E0E0F0E09F0190E047
:10E500005FEFA6E5B8E04BE0ED018B8187FF0BC024
:10E510009F5F8D81E80FF11D8981280F311D8E814C
:10E52000851708F4582F4150189647FFEDCF5093A8
:10E53000160A232B41F520910105309102054091E7
:10E54000030550910405BB27A52F942F832F90938B
:10E5500000058093FF04AA27BB27281B390B4A0B11
:10E560005B0BCF01AA27BB27280F391F4A1F5B1F50
:10E570002093010530930205409303055093040551
:10E58000E5E0F0E013C02091FF04309100052E1764
:10E590003F0718F4E21BF30B02C0E0E0F0E0892F24
:10E5A0009927880F991FE80FF91F3596F093110AE4
:10E5B000E093100AEF3FF10578F480911F019091EC
:10E5C00020018E9F90018F9F300D9E9F300D112452
:10E5D000C90164E670E013C0CF01969587959695C2
:10E5E000879520911F0130912001289FA001299F2C
:10E5F000500D389F500D1124CA0169E170E00E944E
:10E60000C0917093130A6093120A2091FD04309117
:10E61000FE042E0F3F1F3093FE042093FD045EE0A6
:10E620002131350778F08091140A9091150A0196EE
:10E630009093150A8093140A20513E403093FE04B3
:10E640002093FD04DF91CF91089530911005E32FC1
:10E65000FF2783E0EE0FFF1F8A95E1F7EA5AF74F95
:10E660002781422F552747FD509580911105992705
:10E67000841795072CF420931105309313050AC0D5
:10E68000222341F08091120599274817590714F465
:10E6900020931205832F8F5F809310058D30D0F06B
:10E6A00010921005809112058F3F19F08093060596
:10E6B00002C0109206058091110580930705809194
:10E6C0001305809305058FEF8093120510921105B5
:10E6D00010921305089595E1899F802D11240E94C1
:10E6E000D68B8AE89CE09F938F9388EA9BE89F9360
:10E6F0008F93E0913B05F0913C0509950F900F90A9
:10E700000F900F900895CF93C0E020919D0120932A
:10E710000A058091CF0385FF02C0C0E123C090911C
:10E72000E2049923B1F080910604882349F4E92F8B
:10E73000FF27EE0FFF1FE150F64F8491882349F425
:10E74000E92FFF27EE0FFF1FE250F64FC491CC23B5
:10E7500049F48091F20786FD03C010929D0104C028
:10E76000C22F02C0C0930A05809114058C1771F462
:10E7700080911505909116050E947819882319F447
:10E7800080E090E017C088E893E102C080ED97E058
:10E790000E946F199093160580931505CC2331F0D4
:10E7A00080919D01C81711F410929D01C09314052A
:10E7B0008C2F9927CF91089540E050E030E0809170
:10E7C000DE0999278A38910589F08B38910524F460
:10E7D0008938910541F013C08D38910569F08E3864
:10E7E000910539F00CC04FE65AE008C047E45BE001
:10E7F00005C047E15AE002C043E45AE03CE2909190
:10E80000D30920E08091D409281770F4931760F49D
:10E81000DA01A90FB11DE22FFF27E054F64F8589D9
:10E820008C939F5F2F5FEECF089520E335E78091B3
:10E830003B018B3211F08D32F9F480919507282F2E
:10E8400033278091FB039091FC03829FA001839F5B
:10E85000500D929F500D1124CA0163E070E00E9498
:10E86000D491CB019B01205D3A48C196C19708F035
:10E870003FC02EEF34E73CC0803229F58091CF03B2
:10E8800081FF36C02091080530910905205D3A4886
:10E8900055E72133350748F085E72439380718F460
:10E8A00020E335E702C02456304045E720333407E3
:10E8B000F8F454E72D3C350718F020E335E718C08D
:10E8C0002C593F4F15C08E3549F49091F6038AE0DC
:10E8D000989F90011124205D3A480AC0863741F480
:10E8E0009091F6038AE0989FC0011124281B390BF0
:10E8F000C9010895EF92FF920F931F9399278A38C9
:10E90000910509F444C18B38910524F489389105A7
:10E9100051F0DEC28D38910509F424C28E3891057C
:10E9200009F486C1D5C28091010490910204A0919E
:10E930000304B0910404BC01CD0124E630E040E0C2
:10E9400050E00E940992DA01C9018C509E4F9093C9
:10E95000750A8093740A0E94157490937B0A8093C1
:10E960007A0A90937D0A80937C0A90937F0A809321
:10E970007E0A2091740A3091750A8091780A9091EC
:10E98000790A2817390724F43093790A2093780AF2
:10E990008091760A9091770A8217930724F4309336
:10E9A000770A2093760A1092710A8FE69AE0909384
:10E9B00027058093260580913B018093950A8091DD
:10E9C000CE0380FF02C083E401C080E28093960AF8
:10E9D0002091E204222309F1822F6AE00E94B4917F
:10E9E000805D8093800A822F0E94B491892F805D80
:10E9F0008093810A8AE38093820A81E1289FF00153
:10EA00001124A3E8BAE0E25CF54F9FE084918D9376
:10EA10009150319697FFFACF58C28091CF0385FF6E
:10EA20000CC0A0E8BAE0EEE5FCE094E184918D939F
:10EA30009150319697FFFACF48C230910E0533239B
:10EA400009F499C087E58093800A80E58093810A64
:10EA500040E24093820A20910F05822F6AE00E94D3
:10EA6000B491805D8093830A822F0E94B491892F94
:10EA7000805D8093840A8FE28093850A832F0E94B1
:10EA8000B491805D8093860A832F0E94B491892F70
:10EA9000805D8093870A4093880A20910B0530910E
:10EAA0000C0583E0293E380780F0C90168EE73E069
:10EAB0000E94C091CB01805D8093890AC90168EEF4
:10EAC00073E00E94C0919C0102C04093890A2536E0
:10EAD000310580F0C90164E670E00E94C091CB016D
:10EAE000805D80938A0AC90164E670E00E94C0914B
:10EAF0009C0103C080E280938A0AC9016AE070E049
:10EB00000E94C091CB01805D80938B0AC9016AE0AD
:10EB100070E00E94C091805D80938C0A8DE68093A6
:10EB20008D0A80E280938E0A20910D05253660F0D3
:10EB3000822F64E60E94B491805D80938F0A822FB9
:10EB40000E94B491292F02C080938F0A822F6AE01D
:10EB50000E94B491805D8093900A822F0E94B491AC
:10EB6000892F805D8093910A83E78093920A80E2E7
:10EB70008093930AAAC1A0E8BAE0E4E7FCE094E13C
:10EB800084918D939150319697FFFACF9EC18091D9
:10EB9000010490910204A0910304B0910404BC010B
:10EBA000CD0124E630E040E050E00E940992DA0115
:10EBB000C9018C509E4F90935D0B80935C0B0E941B
:10EBC000157490935F0B80935E0B88E78093600BC6
:10EBD00080918C098093610B0E9483738093490B11
:10EBE00080918B0981FF02C084E407C080918D0968
:10EBF000833011F480E201C081E28093620B87E4EC
:10EC00009BE0909327058093260580918B0180934C
:10EC10006E0B8091620B8093700B809191099091A3
:10EC2000920997FD0196959587958093630B4DC149
:10EC30000E9425738091010490910204A091030425
:10EC4000B0910404BC01CD0124E630E040E050E086
:10EC50000E940992DA01C9018C509E4F9093320AAA
:10EC60008093310A80911F019091200190932C0A8A
:10EC700080932B0A80911F019091200190932E0A7E
:10EC800080932D0A80912D0990912E0997FD019670
:10EC90009595879580931D0A8093240A2091910968
:10ECA0003091920937FF02C02F5F3F4F359527956E
:10ECB0002093220A80918F099091900964E170E07D
:10ECC0000E94C0916093230A2093290A60932A0A24
:10ECD0000E94157490933A0A8093390A88E78093CA
:10ECE0003B0A80911F01909120019093360A8093F6
:10ECF000350A809106058C5E80932F0A8091070566
:10ED00008C5E8093300A8091140A9091150A6AE013
:10ED100070E00E94C0917093380A6093370A109295
:10ED2000190A8091100A9091110A9093340A8093E5
:10ED3000330A87E19AE09093270580932605209176
:10ED4000D6023091D702C9016CE370E00E94C091F5
:10ED500060933E0AC9016CE370E00E94C091809309
:10ED60003F0AB3C00E94257380918F09909190094A
:10ED700064E670E00E94C0917093590A6093580A4B
:10ED800080912D0990912E0997FD01969595879573
:10ED90008093490A809191099091920997FD01967B
:10EDA0009595879580934E0A80910001482F5527AD
:10EDB0009A012B5F3F4F80911F01909120012817EE
:10EDC000390784F480911F0190912001841B950BD9
:10EDD0009C01220F331F280F391F822F82518093ED
:10EDE000550A02C01092550AE0900104F090020406
:10EDF0000091030410910404C801B70124E630E037
:10EE000040E050E00E9409923093570A2093560A3E
:10EE100037FF04C01092570A1092560AC801B70172
:10EE200024E630E040E050E00E940992DA01C90196
:10EE30008C509E4F90935B0A80935A0A80911F01D9
:10EE4000909120019093500A80934F0A80911F0166
:10EE5000909120019093520A8093510A0E94157458
:10EE600090935D0A80935C0A88E780935E0A8091A4
:10EE70001F01909120019093620A8093610A809112
:10EE800006058C5E8093530A809107058C5E809303
:10EE9000540A8091140A9091150A6AE070E00E9469
:10EEA000C0917093640A6093630A1092450A80913E
:10EEB000100A9091110A9093600A80935F0A83E48C
:10EEC0009AE090932705809326052CE230E002C05B
:10EED00020E030E0C9011F910F91FF90EF9008955D
:10EEE000EF92FF920F931F93CF93DF9380910805CA
:10EEF000909109059C0153E0220F331F5A95E1F7C9
:10EF0000281B390B8091170390911803280F391F84
:10EF100037FF02C0295F3F4F43E0359527954A955B
:10EF2000E1F730930905209308059091180599237E
:10EF300009F020C380911705282F33274427552730
:10EF40008F5F80931705F9012131310508F00FC358
:10EF5000E857FF4F0C945B928091CF0385FF2AC046
:10EF600080E00E94D68B80911F01909120016AE081
:10EF700070E00E94D4919F938F9380911F01909194
:10EF800020016AE070E00E94D4917F936F9380EA41
:10EF90009CE09F938F9389EC9BE89F938F93E091E4
:10EFA0003B05F0913C0509952DB73EB7285F3F4FD3
:10EFB0002DBF28C080E00E94D68B80911F019091C8
:10EFC00020016AE070E00E94D4919F938F9380911A
:10EFD0001F01909120016AE070E00E94D4917F931C
:10EFE0006F938DEA9CE09F938F9388EA9BE89F93B1
:10EFF0008F93E0913B05F0913C0509958DB79EB745
:10F0000008968DBF8091700980FF39C080911E04E1
:10F010008823E9F08AE00E94D68B80913B019927F2
:10F020009F938F938091010490910204A091030417
:10F03000B0910404BC01CD0124E630E040E050E092
:10F040000E9409923F932F938AEB9CE099C68AE035
:10F050000E94D68B8091010490910204A091030438
:10F06000B0910404BC01CD0124E630E040E050E062
:10F070000E9409923F932F9386EC9CE0ADC78AE0F3
:10F080000E94D68B81ED9CE09F938F9388EA9BE84A
:10F090000C941D818091CF0385FF2AC085E10E94D9
:10F0A000D68B8091D6029091D7026CE370E00E94DB
:10F0B000C0919F938F938091D6029091D7026CE379
:10F0C00070E00E94C0917F936F938BED9CE09F93C3
:10F0D0008F9389EC9BE89F938F93E0913B05F09190
:10F0E0003C0509952DB73EB7285F3F4F2DBF28C07F
:10F0F00085E10E94D68B8091D6029091D7026CE375
:10F1000070E00E94C0919F938F938091D60290915E
:10F11000D7026CE370E00E94C0917F936F9388EEFA
:10F120009CE09F938F9388EA9BE89F938F93E09155
:10F130003B05F0913C0509958DB79EB708968DBFAC
:10F140008FE10E94D68B80E690E09F938F93809111
:10F150002D0990912E099F938F9385EF9CE09F93AB
:10F160008F93C8EADBE8DF93CF93E0913B05F09102
:10F170003C0509958091CE032DB73EB7285F3F4FE0
:10F180002DBF80FF06C089E20E94D68B80E09DE003
:10F1900073C389E20E94D68B82E09DE0B9C680915C
:10F1A000CF0385FF1BC08AE20E94D68B8091140A90
:10F1B0009091150A9F938F9384E09DE09F938F9386
:10F1C00089EC9BE89F938F93E0913B05F0913C0580
:10F1D00009958DB79EB706968DBF1BC08AE20E9427
:10F1E000D68B8091140A9091150A9F938F938CE08F
:10F1F0009DE09F938F9388EA9BE89F938F93E09184
:10F200003B05F0913C0509952DB73EB72A5F3F4F6E
:10F210002DBF86E30E94D68B8091100A9091110A2F
:10F220006AE070E00E94C0919F938F938091100AD2
:10F230009091110A6AE070E00E94C0917F936F93F1
:10F2400084E19DE09F938F9388EA9BE89F938F933F
:10F25000E0913B05F0913C0509958DB79EB7089666
:10F26000C9C689E00E94D68B80E29DE09F938F9370
:10F2700008EA1BE81F930F93E0913B05F0913C05D2
:10F2800009958EE10E94D68B0F900F900F900F90F2
:10F2900082E29DE09F938F931F930F93E0913B0534
:10F2A000F0913C05099583E30E94D68B0F900F9057
:10F2B0000F900F9084E29DE09F938F931F930F9385
:10F2C000E0913B05F0913C0509958FE30E94D68BB8
:10F2D0000F900F900F900F9086E29DE09F938F9379
:10F2E0001F930F93E0913B05F0913C0509958EE744
:10F2F0000E94D68B0F900F900F900F908CE39DE0A3
:10F300009F938F931F930F939AC7809197018823A0
:10F3100009F462C08DE50E94D68B82E59DE09F9343
:10F320008F93C8EADBE8DF93CF93E0913B05F09140
:10F330003C05099584E50E94D68B0F900F900F90A5
:10F340000F9080918C0999279F938F9384E59DE07E
:10F350009F938F93DF93CF93E0913B05F0913C0512
:10F3600009958EE50E94D68B2DB73EB72A5F3F4F99
:10F370002DBF80918F09909190096AE070E00E9402
:10F38000C0917F936F938DE59DE09F938F93DF9363
:10F39000CF93E0913B05F0913C0509958DB79EB761
:10F3A00006968DBF80918D09833081F480918B0901
:10F3B00081FF06C08BE50E94D68B87E69DE0A8C53D
:10F3C0008BE50E94D68B8AE69DE0A2C58BE50E9464
:10F3D000D68B8DE69DE02DC784E0D3C38091970145
:10F3E000882309F47AC080911A0598EAE92E9BE8EF
:10F3F000F92E882309F44BC089E60E94D68B8091B0
:10F40000E10499279F938F9380E79DE09F938F93CB
:10F41000FF92EF92E0913B05F0913C05099585E75D
:10F420000E94D68B2DB73EB72A5F3F4F2DBF8091EC
:10F430008B0199279F938F9300E610E01F930F9302
:10F4400080919109909192099F938F938BE79DE012
:10F450009F938F93FF92EF92E0913B05F0913C05D3
:10F46000099582E70E94D68B8DB79EB70A968DBF0D
:10F470008091DF0499279F938F931F930F9380911F
:10F48000E00499279F938F9387E89DE073C689E6F0
:10F490000E94D68B80918B0199279F938F9380E652
:10F4A00090E09F938F9380919109909192099F93FF
:10F4B0008F9380918E0999279F938F9387E99DE081
:10F4C0009F938F93FF92EF92E0913B05F0913C0563
:10F4D00009958DB79EB70C968DC585E052C3909166
:10F4E000E2049923D1F080912305882381F09032A2
:10F4F00070F487E00E946B7383E90E94D68B809141
:10F50000E20499279F938F9380EB9DE0A4C383E946
:10F510000E94D68B8BEB9DE0B3C38091CF0308EAAA
:10F52000E02E0BE8F02E85FF06C084E90E94D68B02
:10F5300081EC9DE0DAC383E90E94D68B84ED9DE0E7
:10F54000D4C38091AC0B863059F480911A0588237E
:10F5500019F010921A059AC681E080931A0596C692
:10F56000883009F093C60E94DB8B81E0DBC3909367
:10F57000170594C6913009F0E0C380911705282F34
:10F580003327442755278F5F80931705F9012131D1
:10F59000310508F07EC6E756FF4F0C945B928091D0
:10F5A000CF0385FF43C080E00E94D68B8091140A70
:10F5B0009091150A9F938F9380911F019091200144
:10F5C0006AE070E00E94D4919F938F9380911F0115
:10F5D000909120016AE070E00E94D4917F936F9334
:10F5E0008091D6029091D7026CE370E00E94C091A6
:10F5F0009F938F938091D6029091D7026CE370E035
:10F600000E94C0917F936F938AEE9DE09F938F93AA
:10F6100089EC9BE89F938F93E0913B05F0913C052B
:10F6200009952DB73EB7225F3F4FB1C580E00E94DC
:10F63000D68B8091140A9091150A9F938F93809195
:10F640001F01909120016AE070E00E94D4919F9385
:10F650008F9380911F01909120016AE070E00E94D9
:10F66000D4917F936F938091D6029091D7026CE3EF
:10F6700070E00E94C0919F938F938091D6029091E9
:10F68000D7026CE370E00E94C0917F936F9385E096
:10F690009EE0C2C285E10E94D68B80E690E09F93F7
:10F6A0008F9380918801909189019F938F9380E23D
:10F6B0009EE09F938F93C8EADBE8DF93CF93E091BE
:10F6C0003B05F0913C050995809170092DB73EB737
:10F6D000285F3F4F2DBF80FF51C080911E048823BB
:10F6E00039F18FE10E94D68B809101049091020440
:10F6F000A0910304B0910404BC01CD0124E630E0E4
:10F7000040E050E00E9409923F932F938AE29EE0EE
:10F710009F938F9388EB9BE89F938F93E0913B059A
:10F72000F0913C0509958DB79EB706968DBF38C000
:10F730008FE10E94D68B8091010490910204A091E8
:10F740000304B0910404BC01CD0124E630E040E0A4
:10F7500050E00E9409923F932F9383E39EE09F9392
:10F760008F93DF93CF93E0913B05F0913C05099592
:10F770002DB73EB72A5F3F4F2DBF12C08FE10E94C9
:10F78000D68B8CE39EE09F938F93DF93CF93E09192
:10F790003B05F0913C0509950F900F900F900F904D
:10F7A00089E20E94D68B80913B0199279F938F938A
:10F7B00086E49EE09F938F93DF93CF9313C4809151
:10F7C00097018823F9F08BE20E94D68B80918B0100
:10F7D00099279F938F9380918F09909190096AE068
:10F7E00070E00E94C0917F936F9380E690E09F93BA
:10F7F0008F9380919109909192099F938F9389E4BF
:10F800009EE058C182E0BDC18FE30E94D68B8091FB
:10F81000120A9091130A9F938F938091100A9091EE
:10F82000110A6AE070E00E94C0919F938F938091CB
:10F83000100A9091110A6AE070E00E94C0917F93D3
:10F840006F9380E69EE09F938F93C8EADBE8DF9397
:10F85000CF93E0913B05F0913C0509958091CE0353
:10F860002DB73EB7265F3F4F2DBF80FF0AC082E510
:10F870000E94D68B84E79EE09F938F9388EB9BE852
:10F88000DCC482E50E94D68B87E79EE041C380916D
:10F89000970118EAE12E1BE8F12E882309F449C0EC
:10F8A00084E50E94D68B80918C0999279F938F9332
:10F8B00080918E0999279F938F938AE79EE09F936B
:10F8C0008F93E701FF92EF92E0913B05F0913C05A9
:10F8D00009958DB79EB708968DBF80918D098330AD
:10F8E00051F484E60E94D68B8DE89EE09F938F931F
:10F8F000FF92EF920BC084E60E94D68B83E99EE0D4
:10F900009F938F9389EC9BE89F938F93E0913B05A6
:10F91000F0913C0509950F900F900F900F908091FA
:10F920008B0981FFBBC484E60E94D68B89E99EE0E7
:10F93000EFC284E50E94D68B8FE99EE0D6C180910C
:10F940001905C8EAEC2ECBE8FC2E882309F450C038
:10F9500089E60E94D68B809173086AE00E94B49178
:10F96000892F99279F938F93809173080E94B49158
:10F9700099279F938F9380916B080E94B491892F50
:10F9800099279F938F9380916B080E94B491992738
:10F990009F938F93809163080E94B491892F992738
:10F9A0009F938F93809163080E94B49199279F93AE
:10F9B0008F9380915B080E94B491892F99279F9320
:10F9C0008F9380915B080E94B49199279F938F93A6
:10F9D00085EB9EE09F938F93FF92EF92E0913B0522
:10F9E000F0913C0509952DB73EB72C5E3F4FCFC334
:10F9F00089E60E94D68B80E690E09F938F9380915A
:10FA00007508992787FD90959F938F9380916D0836
:10FA1000992787FD90959F938F93809165089927EB
:10FA200087FD90959F938F9380915D08992787FD1F
:10FA300090959F938F9382ED9EE09F938F93FF927B
:10FA4000EF92E0913B05F0913C0509958DB79EB78B
:10FA50000E96D0C28091190590918207882309F4EF
:10FA60008DC0943009F48CC09630A1F58EE70E94C9
:10FA7000D68B809183086AE00E94B491892F9927E0
:10FA80009F938F93809183080E94B49199279F93AD
:10FA90008F9380917B080E94B491892F99279F931F
:10FAA0008F9380917B080E94B49199279F938F93A5
:10FAB00085EE9EE09F938F9388EA9BE89F938F93B8
:10FAC000E0913B05F0913C0509952DB73EB7245FC9
:10FAD0003F4F5DC3973008F4E1C38EE70E94D68B99
:10FAE000809193086AE00E94B491892F99279F938F
:10FAF0008F93809193080E94B49199279F938F933D
:10FB000080918B080E94B491892F99279F938F939E
:10FB100080918B080E94B49199279F938F93809135
:10FB200083080E94B491892F99279F938F93809186
:10FB300083080E94B49199279F938F9380917B08AB
:10FB40000E94B491892F99279F938F9380917B086E
:10FB50000E94B49199279F938F9384EF9EE09F9387
:10FB60008F9388EA9BE89F938F93E0913B05F091F8
:10FB70003C0509958DB79EB744963CC2943021F45C
:10FB800086E00E946B738AC39630F1F48EE70E9480
:10FB9000D68B80E690E09F938F938091850899277C
:10FBA00087FD90959F938F9380917D08992787FD7E
:10FBB00090959F938F9381E19FE09F938F9388EA25
:10FBC0009BE89F938F93DAC2973008F467C38EE760
:10FBD0000E94D68B80E690E09F938F93809195084A
:10FBE000992787FD90959F938F9380918D089927F2
:10FBF00087FD90959F938F9380918508992787FD26
:10FC000090959F938F9380917D08992787FD90957C
:10FC10009F938F9384E29FE09F938F9388EA9BE862
:10FC20009F938F930ECF9091E204992309F44AC0D9
:10FC3000809123058823F9F09032E8F487E00E9450
:10FC40006B7383E90E94D68B8091E20499279F937E
:10FC50008F9387E39FE09F938F9388EB9BE89F931D
:10FC60008F93E0913B05F0913C0509952DB73EB788
:10FC70002A5F3F4F8CC283E90E94D68B82E49FE0CB
:10FC80009F938F9308EA1BE81F930F93E0913B0526
:10FC9000F0913C0509951F921F929091E20481E139
:10FCA000989FC0011124825C954F9F938F931F935F
:10FCB0000F93E0913B05F0913C0509958DB79EB7F8
:10FCC0000A9698C18091CF03B8EAEB2EBBE8FB2ED1
:10FCD00085FF06C084E90E94D68B88E49FE005C0BA
:10FCE00083E90E94D68B8BE59FE09F938F93FF92D1
:10FCF000EF92A5C28091AC0B863079F48091190502
:10FD0000882319F01092190503C081E0809319052A
:10FD100085E00E946B7386E0AEC2883031F40E94A9
:10FD2000DB8B82E080931805AFC2813009F0AEC250
:10FD30000E94DB8B10921805A7C2923009F0ACC26A
:10FD400080911705282F3327442755278F5F8093ED
:10FD50001705F9012131310508F09BC2E655FF4F27
:10FD60000C945B9280E00E94D68B83EF97E09F9388
:10FD70008F930E94633099279F938F9381E79FE031
:10FD80009F938F9388EB9BE89F938F93E0913B0524
:10FD9000F0913C0509952DB73EB7285F3F4FF7C15D
:10FDA00085E10E94D68B81E098E09F938F938091AC
:10FDB00000016AE00E94B491892F99279F938F9345
:10FDC000809100010E94B49199279F938F9380E8BE
:10FDD0009FE09F938F9388EA9BE89F938F93E09196
:10FDE0003B05F0913C05099569CF8AE20E94D68BCC
:10FDF00081E99FE09F938F93C8EADBE8DF93CF937D
:10FE0000E0913B05F0913C050995809170090F90B8
:10FE10000F900F900F9080FF41C0809190079091BC
:10FE2000730181FD0BC0892F99279F938F9386E9DA
:10FE30009FE09F938F93DF93CF9313CFE0913B0588
:10FE4000F0913C05933318F080EA9FE002C087EA06
:10FE50009FE09F938F93DF93CF9309950F900F901F
:10FE60000F900F9080915409E0913B05F0913C0573
:10FE70009091730180FF0BC0892F99279F938F93D7
:10FE80008EEA9FE09F938F93DF93CF93AFC0892F2C
:10FE900099279F938F9384EB9FE0CFC08AEB9FE0DD
:10FEA00037C08FE30E94D68B83EC9FE09F938F93A4
:10FEB000C8EADBE8DF93CF93E0913B05F0913C0586
:10FEC00009950F900F900F900F908091E60788236F
:10FED00019F487EC9FE01CC08091DC03E0913B05A6
:10FEE000F0913C05882319F080ED9FE002C087ED7A
:10FEF0009FE09F938F93DF93CF9309950F900F907F
:10FF00000F900F908091F10786FFC8C18EED9FE0A2
:10FF10009F938F93DF93CF9392C184E50E94D68BFA
:10FF200085EE9FE09F938F93C8EADBE8DF93CF9342
:10FF3000E0913B05F0913C050995809170090F9087
:10FF40000F900F900F9085FD03C08AEE9FE011C0C7
:10FF50008091D407883F10F4E82F07C0EFEFF0E05E
:10FF6000E81BF109E85FFB4FE081E23358F483EFCF
:10FF70009FE09F938F93DF93CF93E0913B05F091A8
:10FF80003C0516C0E43B18F08AEF9FE0F2CF809169
:10FF9000F107E0913B05F0913C0585FF03C081E04E
:10FFA00090E102C088E090E19F938F93DF93CF931D
:10FFB00009950F900F900F900F908091EA0788237A
:10FFC00009F46CC18EE50E94D68B8091EA079927CF
:10FFD0009F938F938FE090E19F938F9388EA9BE8A4
:10FFE0009F938F93E0913B05F0913C0509958DB768
:10FFF0009EB706968DBF52C189E60E94D68B8AE1D4
:020000021000EC
:1000000090E19F938F93C8EADBE8DF93CF93E09171
:100010003B05F0913C0509950F900F900F900F90C4
:100020008091E907E0913B05F0913C05882351F070
:1000300099279F938F9384E290E19F938F93DF930F
:10004000CF9313CE88E290E19F938F93DF93CF936A
:10005000FAC080911B05A8EAEA2EABE8FA2E8823A5
:1000600009F053C08EE70E94D68B809167019927D3
:100070009F938F9380918507E82FFF27EE0FFF1F37
:10008000E954F74F808191819F938F9380918407EA
:10009000E82FFF27EE0FFF1FE954F74F8081918172
:1000A0009F938F938EE290E19F938F93FF92EF92B5
:1000B000E0913B05F0913C05099583E90E94D68BC0
:1000C0008DB79EB70A968DBF80918707E82FFF27CF
:1000D000EE0FFF1FE954F74F808191819F938F931B
:1000E00080918607E82FFF27EE0FFF1FE954F74F97
:1000F0008081918181589F4F9F938F9382E490E1FB
:100100009F938F93FF92EF9241CE8EE70E94D68B02
:1001100080910A0499279F938F93809109049927CE
:100120009F938F938091080499279F938F9381E5E4
:1001300090E19F938F93FF92EF92E0913B05F091B6
:100140003C05099583E90E94D68B8DB79EB70A9628
:100150008DBF80910D0499279F938F9380910C04FC
:1001600099279F938F9380910B0499279F938F9347
:1001700085E690E19F938F93FF92EF92E0913B058C
:10018000F0913C0509952DB73EB7265F3F4F2DBF37
:1001900085C080912305882309F480C08EE70E94E2
:1001A000D68B8091700986FD11C089E790E19F93FD
:1001B0008F9389EC9BE89F938F93E0913B05F0919F
:1001C0003C0509950F900F900F900F908091EF07CD
:1001D00099278F709070892B89F088E890E19F9320
:1001E0008F9389EC9BE89F938F93E0913B05F0916F
:1001F0003C0509950F900F900F900F90809170091A
:1002000082FF11C082E990E19F938F9389EC9BE874
:100210009F938F93E0913B05F0913C0509950F90DA
:100220000F900F900F908091700983FD37C087E980
:1002300090E19F938F9389EC9BE89F938F93E0913C
:100240003B05F0913C0509950F900F900F900F9092
:1002500025C00091AC0B063089F480911B058823E2
:1002600019F010921B0503C081E080931B0586E006
:100270000E946B7387E00E946B7308C0013031F4F9
:100280000E94DB8B00931805109217051092AC0B9F
:1002900005C01092170502C010921805E6E0CDB710
:1002A000DEB70C944C924FB728E130E0F89480917F
:1002B000C9008F778093C9008091C9008F7B80939C
:1002C000C9008091C9008F7D8093C9005A9A5298C5
:1002D0005B9A539A832F99278093CD002093CC006B
:1002E0008091C80082608093C80080E18093C9003B
:1002F0008091CA008F778093CA008091CA008F7B5B
:100300008093CA008091CA008091CA008F7E80933A
:10031000CA008091CA0088608093CA008091C90099
:100320008B7F8093C9008091CA0084608093CA004B
:100330008091CA0082608093CA008091C80087FFC4
:1003400003C08091CE00F9CF8091C900806880936E
:10035000C90080918A0B846080938A0B4FBF0895F7
:100360009091F604992341F48F3031F490931D0558
:1003700080E58093F6040895E0911D05EF5FE0931A
:100380001D05E83121F481E080931C050895E931D1
:1003900020F089E180931D050895FF27ED58F44F63
:1003A00080830895A0E0B0E0E8EDF1E80C942C9291
:1003B00091E0D92E82E0A82EBD2CE12C01E0F02E98
:1003C00080918A0B82FDB5C080916F008F7D8093F4
:1003D0006F00E091EC07EE2351F0FF27EE0FFF1FB7
:1003E000E954F74F80819181843691055CF48091C6
:1003F0000704883C20F4809107048C5E01C088ECDF
:10040000809307048091740B682F772780911E05D5
:10041000815080931E058F3F31F41CE7C12E82E08E
:1004200080931E0502C0C4E2CC2E40E04C1508F0BB
:100430007EC0EA2DFF27ED58F44F80818D2111F009
:100440006E297F298D2D9927880F991FD82E8823F3
:1004500019F4B1E0DB2EAD0CEE0CFF1C20E0E2162F
:1004600028E0F20609F061C0A1E0EA2EF12CCB01F0
:100470008050944065E070E00E94D491AB2DBB2782
:10048000FD01EA0FFB1FE954F74F808191819C0128
:10049000220F331F280F391F260F371F37FF02C0C7
:1004A0002D5F3F4FE901D595C795D595C795CB01F0
:1004B00001968C179D0714F4219706C06150704077
:1004C000C617D7070CF4219680910704833CD8F017
:1004D0008D010A0F1B1FF801E954F74F80819181AC
:1004E000FE01E81BF90BCF0163E070E00E94D4919C
:1004F000CB01880F991F860F971F0551174FF801E1
:100500009183808307C0AA0FBB1FA551B74F1196D7
:100510001C921E92EB2DFF27EE0FFF1FE954F74FA1
:10052000D183C08360E070E0B3944F5F7FCF1092BF
:100530003A0110921C05EAE0CDB7DEB70C94489260
:100540000895089540E050E080911F0590912005A6
:100550009C01220F331F280F391F809117039091A0
:100560001803280F391F37FF02C02D5F3F4F359505
:100570002795359527953093200520931F05809169
:100580003B018B32D9F480919507282F3327809136
:10059000FB039091FC03829FA001839F500D929FCB
:1005A000500D1124CA0157FD4F96AC0125E0559519
:1005B00047952A95E1F74B5F5F4F3DC08D32D9F4E7
:1005C00080919507282F33278091FB039091FC039E
:1005D000829FA001839F500D929F500D1124CA014C
:1005E00057FD4F96AC0195E0559547959A95E1F7E3
:1005F0004550504020C0803271F48091CF0381FF7C
:100600001AC0C90137FD4F96AC0185E05595479555
:100610008A95E1F710C08E3529F48091F603482FB2
:10062000552709C0863739F48091F6039927442766
:100630005527481B590BCA01AA2797FDA095BA2F29
:100640008093900290939102A0939202B0939302B0
:1006500008950F931F930E94257380911F0190911D
:100660002001AA2797FDA095BA2F8093BF019093F0
:10067000C001A093C101B093C2018091100A909172
:10068000110AAA27BB278093D2019093D301A0938C
:10069000D401B093D5010AE010E08091140A909142
:1006A000150AB8010E94C091CB01AA27BB278093ED
:1006B000E5019093E601A093E701B093E8018091F2
:1006C000010490910204A0910304B0910404BC01C0
:1006D000CD0124E630E040E050E00E9409922093F2
:1006E000F8013093F9014093FA015093FB01809196
:1006F000880190918901AA2797FDA095BA2F809330
:100700000B0290930C02A0930D02B0930E02809105
:100710008C099927AA27BB2780931E0290931F025A
:10072000A0932002B093210280918E099927AA27D5
:10073000BB278093310290933202A0933302B0938F
:10074000340280918F0990919009B8010E94C09164
:10075000CB01AA27BB278093440290934502A09324
:100760004602B09347028091910990919209AA277D
:1007700097FDA095BA2F8093570290935802A093AB
:100780005902B0935A02809107059927AA27BB27DF
:1007900080936A0290936B02A0936C02B0936D02F7
:1007A0008091E1049927AA27BB2780937D0290932B
:1007B0007E02A0937F02B09380028091E204992789
:1007C000AA27BB278093A3029093A402A093A5021B
:1007D000B093A6021F910F9108950024222733277A
:1007E000442751E0BB27EE27FF27A0E1660F771FC4
:1007F000881F991F001C221F331F441F660F771F7D
:10080000881F991F001C221F331F441F2AF4050E46
:100810002B1F3E1F4F1F04C0051A2B0B3E0B4F0B07
:10082000550FBB1FEE1F587F556047FD5250AA95CC
:10083000E9F6E695B7955795E695B7955795852FBF
:100840009B2F08952227332741E0552768E0880F22
:10085000991F221F331F880F991F221F331F1AF45D
:10086000240F351F02C0241B350B440F551F487F32
:10087000456037FD42506A9551F756954795569514
:100880004795842F0895AA2797FF04C080959095D7
:100890008A1F9A1F77FF04C0609570956A1F7A1FA0
:1008A000669F9001779FA001679F300D411D5A1FE1
:1008B000300D411D5A1F889FF001999F2E0F3F1F39
:1008C000401D511D899F300D411D5A1F300D411D86
:1008D0005A1FCA01B901112480CF4FB720E430E07C
:1008E000F8948091C9008F778093C9008091C900E6
:1008F0008F7B8093C9008091C9008F7D8093C90050
:100900005A9A52985B9A539A832F99278093CD00D5
:100910002093CC008091C80082608093C80088E159
:100920008093C9008091CA008F778093CA0080911C
:10093000CA008F7B8093CA008091CA008F7D80930C
:10094000CA008091CA008F7E8093CA008091CA003D
:10095000877F8093CA008091C9008B7F8093C900F4
:100960008091CA0084608093CA008091CA0082602E
:100970008093CA008091C80087FF03C08091CE0099
:10098000F9CF8091C90080688093C9004FBF089556
:100990000F931F93CF93DF93482F4F5F893108F058
:1009A0008BC08091B608841720F44F5F4093B6083F
:1009B0004150CB0183539B4268E170E00E94D49187
:1009C000A42FBB27FD01EA0FFB1FE954F74F8081DD
:1009D00091819B01281B390BC90137FF03C09095FA
:1009E00081959F4F069794F480910704883C30F4DA
:1009F00080910704865F8093070408C088EC809389
:100A0000070480916F008F7D80936F00FD01EA0FD6
:100A1000FB1FE954F74F808191819C01220F331F06
:100A2000280F391F260F371F37FF02C02D5F3F4F9A
:100A3000E901D595C795D595C795CB0101968C173A
:100A40009D0714F4219706C061507040C617D70760
:100A50000CF4219680910704843BD8F08D010A0F95
:100A60001B1FF801E954F74F80819181FE01E81BBB
:100A7000F90BCF0163E070E00E94D491CB01880FA5
:100A8000991F860F971F0551174FF8019183808397
:100A900007C0AA0FBB1FA551B74F11961C921E92FB
:100AA000E42FFF27EE0FFF1FE954F74FD183C083D8
:100AB000443011F410923A01DF91CF911F910F91C0
:100AC0000895CF93DF932091AD0B822F9927807FDC
:100AD0009070409709F06CC02F3109F046C08091AA
:100AE000AE0B80932A052091B00B20932C058091AA
:100AF000B10B80932B05822F99279093B808809390
:100B0000B708222309F054C080918407282F332787
:100B1000220F331FF901E551F74F118210828091A6
:100B20008507A82FBB27AA0FBB1FFD01E551F74F73
:100B30001182108280918707E82FFF27EE0FFF1F99
:100B4000CF018551974FEC01198218822954374FF4
:100B5000E90119821882A954B74F11961C921E926E
:100B6000E954F74F1182108223C0C22FCF70CA30D0
:100B7000F8F48091AE0B8093D90B8091AF0B8093EA
:100B8000D80B8091B00B8093DB0B8091B10B8093DD
:100B9000DA0B6091D80B7091D90B8C2F0E94C8840E
:100BA0006091DA0B7091DB0B8C2F8F5F0E94C884F1
:100BB000DF91CF910895CF93C82F8F3F49F4809153
:100BC0002D058F3F29F410922F0510922E0532C06B
:100BD00020912F05222339F4CF3111F485E001C093
:100BE00084E0809330058091300590912E05821726
:100BF000A0F4892F809580932E058F3F19F48EEFF6
:100C000080932E0580912E05C81711F40E946185EE
:100C100010922F0510922E050BC0E22FFF27E355EF
:100C2000F44FC0832F5F20932F059C0F90932E05C8
:100C3000C0932D05CF91089590912905933240F4EA
:100C4000E92FFF27EB54F44F80839F5F9093290592
:100C50000895833218F48D5F80932905089590E2FA
:100C6000E8EBFBE08FE19193815087FFFCCF089583
:100C7000CF93CFB723E031E0F8948091C9008F770C
:100C80008093C9008091C9008F7B8093C9008091B7
:100C9000C9008F7D8093C9005A9A52985B9A539AE3
:100CA000832F99278093CD002093CC008091C8009A
:100CB00082608093C80088E18093C9008091CA0057
:100CC0008F778093CA008091CA008F7B8093CA007F
:100CD0008091CA0080628093CA008091CA008061BE
:100CE0008093CA008091CA0088608093CA00809176
:100CF000C90084608093C9008091CA008460809399
:100D0000CA008091CA0082608093CA008091C800A6
:100D100087FF03C08091CE00F9CF8091C900806821
:100D20008093C9008091C90080648093C9000E94AB
:100D30002F86CFBFCF910895282F99278F7090705D
:100D4000892B31F4209580912805822B80932805EA
:100D500008951F920F920FB60F9211248F93EF9365
:100D6000FF938091D002882309F068C0E09132059A
:100D7000EE2389F480913105882369F48091B50BC5
:100D8000882321F081E08093330505C08091C9005C
:100D900081608093C90080913305882379F4EF5FE7
:100DA000E093320580918C0B8E1720F481E08093C4
:100DB00033051CC0FF27E457F44F3CC08091310538
:100DC000882361F48091B50B882311F483E003C07C
:100DD000813999F481E0809331050FC0833099F413
:100DE0008091B50B882349F01092B50B8091C90012
:100DF0008E7F8093C9008EEF1EC08091C9008160F4
:100E00008093C9000EC0833261F48091C9008E7F47
:100E10008093C9008FEF8093CE0081E08093D00251
:100E200018C080913105E82FFF27EB54F44F8F5FF6
:100E30008093310580818093CE000BC010923105E4
:100E400010923205109233058091C9008061809321
:100E5000C900FF91EF918F910F900FBE0F901F90DF
:100E60001895682727E0322F67FF06C0862F99273D
:100E7000880F991F832702C0862F880F682F215063
:100E800027FFF2CF992708950F931F93CF93DF93F6
:100E9000062F60E0162F601740F4EC0189910E9444
:100EA0003187682F1F5F1017C8F3862F9927DF91AE
:100EB000CF911F910F910895DC0190E0961758F49F
:100EC0008C91803241F09F5F961728F4FD01E90F65
:100ED000F11D8081F6CF892F99270895A0E0B0E019
:100EE000E4E7F7E80C942D928FE980938D0B80E175
:100EF00080938F0B84EA8093900B85E58093910B10
:100F00008DE58093920B1092930B80913505882389
:100F100009F06AC08091340513E1819FC00111245A
:100F200063E088559E4F0E945C87082F80913405AE
:100F3000819FC00111246AE082569E4F0E945C8707
:100F4000982F800F865F80938C0B4EEFB42EB80ED7
:100F5000B0928E0B209134052093940BE92EFF2440
:100F6000C70133E0880F991F3A95E1F7802B8093F2
:100F7000950B822F992723E1C22ED12C8C9D9001B5
:100F80008D9D300D9C9D300D1124C90182569E4FC0
:100F9000A701BC0186E99BE00E94F58F1127809193
:100FA000340599278C9DE0018D9DD00D9C9DD00D21
:100FB0001124CE0188559E4FA801BC01C7018A5655
:100FC000944F0E94F58F0457144F0E0D1F1D6B2D6B
:100FD0008EE89BE00E944487F80182878091350566
:100FE0008F5F8093350570C01091930B0E94298309
:100FF0004091D1024031C8F563E170E0812F99271B
:10100000DC01AA0FBB1FA80FB91FA457B44F842F30
:101010009927869FF001879FF00D969FF00D112470
:10102000E256FE4F2585C4E0880F991FCA95E1F767
:10103000282BED012887268537853F7982899927D6
:10104000982F88279295990F907E282B392B2987E6
:10105000832F99278A87842F8F5F1F5F163018F49C
:10106000482F803158F28093D10283E0189F90017D
:101070001124822F885F80938C0B825C80938E0B6F
:10108000812F99278C01000F111F080F191F04577A
:10109000144F822F8A5F682F8EE89BE00E9444875E
:1010A000F80180878091D102803170F081E08093D7
:1010B000D10210923505809134058F5F80933405FD
:1010C000803110F010923405E9E0CDB7DEB70C9412
:1010D00049928091D002882309F447C08091CF03C0
:1010E00085FD04C08091D402882381F082E9809339
:1010F000B50B83E28093B60B8091D402882309F468
:1011000085E58093B70B1092D40202C08093B50B93
:101110008091D2028F3071F4809128050E944E7226
:10112000882341F081E98093B50B8093B60B81E36E
:101130008093B70B1092D0028091C80085FFFCCF3E
:101140008091C9008F7E8093C9008091C9008E7FF5
:101150008093C9000E946E878EE78093CE008091B5
:1011600028058093D202109228050895EF92FF92ED
:101170000F931F93CF93DF937C018B01EA01452BE3
:1011800039F0F80181918F01F70109952197C9F78D
:10119000E6E0CDB7DEB70C944C92EF92FF920F933E
:1011A0001F93CF93DF937C018B01EA01452B41F024
:1011B000F8010F5F1F4F8491F70109952197C1F73F
:1011C000E6E0CDB7DEB70C944C920F931F93CF930C
:1011D0008C01C62F161634F480E2F8010995C1502F
:1011E0001C16D4F3CF911F910F9108950F931F9365
:1011F000CF938C01C62F161634F480E3F8010995BD
:10120000C1501C16D4F3CF911F910F910895A5E3FF
:10121000B0E0EDE0F9E80C9424922E96EEADFFAD2F
:101220002E9788249924540180912205882321F443
:101230002C961FAE1EAE2C97AEE44A2E512C4C0EAF
:101240005D1E6F01B60105C0153239F00894C11C4E
:10125000D11CF60114911123B9F7A601461B570BB7
:1012600031F02C968EAD9FAD2C970E94CD88112326
:1012700009F46AC20894C11CD11CFF24FDA6FCA677
:10128000FFEFEF2EF9A6F6010894C11CD11C1491B2
:10129000153721F0812F80628837B1F4F0FE0AC043
:1012A000F20124E030E0420E531E80809180A28043
:1012B000B3800AC0F20142E050E0440E551E808126
:1012C00091814C01AA24BB24103221F489A58823E2
:1012D000D1F61DC0133219F458E0F52AD4CF1A32D2
:1012E00011F01D3291F41A3259F4F20182E090E0CB
:1012F000480E591EE081ECA7EE232CF6E195ECA7F1
:1013000090E1F92AAFEDFA22BECF1B3211F419A7F2
:10131000BACF1E32C1F5F6010894C11CD11C14913C
:101320001A3279F4F20122E030E0420E531E40817D
:1013300051813FEF4F3F530714F44FEF5FEFE42E1F
:10134000A2CF40E050E0812F80538A30A0F4CA0140
:10135000E3E0880F991FEA95E1F7840F951F480F86
:10136000591F410F511D40535040F6010894C11CB4
:10137000D11C1491E8CF8FEF4F3F580714F44FEF73
:101380005FEFE42E85CF103329F4F4FC7CCF90E29C
:10139000F92A79CF812F81538930D8F440E050E089
:1013A000CA0173E0880F991F7A95E1F7840F951FA2
:1013B000480F591F410F511D40535040F6010894EA
:1013C000C11CD11C1491812F80538A3048F34CA743
:1013D0005FCF183619F4A4E0FA2A55CF1C3619F459
:1013E000B1E0FB2A50CF133661F43E010894611C32
:1013F000711CF20122E030E0420E531E808189838D
:101400003CC1143421F0143611F0193651F514345E
:1014100011F431E0F32AF0FE0AC0F20144E050E09A
:10142000440E551E80809180A280B3800CC0F201D2
:1014300082E090E0480E591E808191814C01AA24DF
:1014400097FCA094BA2CB7FE0AC0B094A0949094D4
:101450008094811C911CA11CB11C8DE289A70AE01B
:101460006FC01F3411F01F3631F41F3411F491E0B6
:10147000F92A08E064C0103779F4F201A2E0B0E084
:101480004A0E5B1E808191814C01AA24BB2400E19D
:10149000B0E4FB2A18E753C01337C1F5F20122E08C
:1014A00030E0420E531E608071806114710489F433
:1014B0003E010894611C711C88E289838EE6F30169
:1014C000818385E78B838CE68C838D8389E28E8391
:1014D0001F82E7FC13C08E2D992787FD9095AC01E4
:1014E00060E070E0C3010E94E88F009729F0382E79
:1014F0003618E3140CF0C3C03E2CC1C0F3010190B8
:101500000020E9F731973E2E3618B9C0153511F095
:10151000153731F4153511F4F1E0FF2A0AE00FC058
:10152000183519F0183709F0A0C000E1F3FE07C024
:1015300081149104A104B10411F020E4F22A19A647
:10154000EDA6E7FC02C03FEDF32269E2662E712CA6
:101550006C0E7D1E81149104A104B10421F44DA5EB
:10156000442309F47BC0802F9927AA27BB278EA785
:101570009FA7A8ABB9AB202E332490E0891690E04A
:10158000990691E0A90690E0B90648F0C501B401BA
:101590002EA53FA548A959A90E94E79117C0AFEF12
:1015A0008A169104A104B10449F040F0C401B101CC
:1015B0000E94C0919B014427552708C0882D602FA9
:1015C0000E94B491282F3327442755272AAB3BABE1
:1015D0004CAB5DAB0A3059F48AA9880F880F880F8D
:1015E0009AA9990F890F382D381B832F10C000310D
:1015F00039F48AA98295807F482D481B842F07C023
:101600008AA9880F880F880F582D581B852F90E0C6
:101610002EA53FA548A959A982169306A406B5068A
:1016200008F091E08AA89BA8ACA8BDA88A3010F465
:10163000805D04C0895A183509F48F7DD3018E93DB
:101640003D01992309F099CF083041F4F3FE06C01B
:10165000803321F080E3FD0182933F01CE010196AA
:10166000382E3618F8E23F0E0BC0112309F46CC077
:101670003E010894611C711C198351E0352E19A696
:10168000032D2DA4231827FC222489A5882311F0DB
:101690000F5F02C0F6FC0E5F020DEF2CFF24C701A6
:1016A00080739070892B49F48CA5801B682F2C9631
:1016B0008EAD9FAD2C970E94E58889A5882331F0D7
:1016C00041E050E0BE01675D7F4F0AC0E6FE0EC0FC
:1016D00080E38AA71BA742E050E0BE01665D7F4F12
:1016E0002C968EAD9FAD2C970E94B688C701807353
:1016F0009070809749F48CA5801B682F2C968EAD36
:101700009FAD2C970E94F688622D2C968EAD9FADD2
:101710002C970E94F688832D992787FD9095AC0120
:10172000B3012C968EAD9FAD2C970E94B688E4FE37
:1017300089CD2CA5201B2CA7622F2C968EAD9FAD9A
:101740002C970E94E5887ECDE2E1CB5C0C94409220
:10175000982F8091B40B883A50F48091B40BE82F05
:10176000FF27E556F54F93838F5F8093B40B089561
:10177000982F8091B40B883A58F48091B40BE82FDD
:10178000FF27E556F54F906893838F5F8093B40BE6
:101790000895982F80912305882321F0892F0E9496
:1017A000B88B0895892F0E94A88B0895883A10F469
:1017B0008093B40B089580E090E2EEE9FAE0919313
:1017C0008F5F883AE0F308954FB721E830E0F8944E
:1017D0008091C9008F778093C9008091C9008F7B69
:1017E0008093C9008091C9008F7D8093C9005A9A67
:1017F00052985B9A539A832F99278093CD00209318
:10180000CC008091C80082608093C80088E18093FA
:10181000C9008091CA008F778093CA008091CA0066
:101820008F7B8093CA008091CA008F7D8093CA000D
:101830008091CA008F7E8093CA008091CA00877F02
:101840008093CA008091C90084608093C900809110
:10185000CA0084608093CA008091CA00826080932D
:10186000CA008091C90081608093C9008091C8003E
:1018700087FF03C08091CE00F9CF8091C9008068B6
:101880008093C9004FBF3CE73093170A2DE72093A0
:10189000420A8EE88093180A1092340A1092330A92
:1018A00010921D0A80EE80931A0A30936F0A2093DB
:1018B0009A0A10927B0A10927A0A10927D0A10926C
:1018C0007C0A10927F0A10927E0A84EF91E0909336
:1018D000790A8093780A9093770A8093760A909396
:1018E000750A8093740A1092710A89E88093700ACD
:1018F0001092980A1092990A80E98093720A3093A4
:10190000470B2093720B1092490B8AE88093480B87
:1019100010924F0B10924E0B10924D0B1092510BD8
:101920001092520B1092530B1092540B1092560BB4
:101930001092570B1092580B1092590B10925D0B8E
:1019400010925C0B10925B0B10925A0B80EA809302
:101950004A0B3093430A20936E0A1092450A8DE891
:101960008093440A10926D0A80ED8093460A8BE7BB
:1019700080939B0A80E880939C0A10929D0A809134
:101980001D0A90E2EEE9FAE091938F5F883AE0F366
:101990008DE78093460B0895CF93C82F809136052D
:1019A000803879F48C2F0E947A7480932505809179
:1019B0002505882331F1C093B30B809125058F5FF6
:1019C00016C08F37F1F48091AC0B882329F48C2F4B
:1019D00080958F708093AC0B0E94837380939D0AD7
:1019E0008BE99AE090932705809326058DEA8093F2
:1019F00025058091C9008F7E8093C90082E0809385
:101A00002405C0933605CF910895309124053323E2
:101A100031F08091240581508093240508958091B0
:101A20002505882381F140912505909137054130A6
:101A300091F4292F309337058091C90080618093FC
:101A4000C90080912305882319F03093230510C025
:101A5000409323050DC0E0912605F0912705819163
:101A6000F0932705E0932605282F980F90933705CC
:101A70008091C80085FFFCCF2093CE008091250582
:101A800081508093250508952FB740E0F894E0E059
:101A9000F0E081E2809357009491E2E0F0E08093DF
:101AA00057003491E4E0F0E08093570084912FBF19
:101AB0009E3199F4363941F4893011F441E00DC07A
:101AC0008A3059F442E009C0373939F4863011F4CC
:101AD00043E003C0853009F444E0842F992708953A
:101AE0009FB7F8948091C900877F8093C900809147
:101AF000C9008F7E8093C9008091C9008F77809341
:101B0000C9008091C9008F7B8093C9008091C90072
:101B10008F7D8093C90052985A9A53985B9A9FBFC1
:101B200008951F93CF93DF93182F80912205882368
:101B300009F4A7C08091CF02181709F4A2C08091C0
:101B40002105882321F40E94448D8093210582ED94
:101B500091E0909339018093380189E791E19F9357
:101B60008F93C0E6D5E1DF93CF93E0913B05F091F1
:101B70003C0509950F900F900F900F90812F99279A
:101B8000AA27BB27FC01099778F5E554FF4F209160
:101B90003B0530913C050C945B9285E791E102C0D6
:101BA0008CE691E19F938F93DF93CF93F901099591
:101BB00027C087E691E1F6CF8FE591E1F3CF87E586
:101BC00091E19F938F93DF93CF93F901099588ED6E
:101BD00091E0909339018093380112C082E591E140
:101BE000E1CF86E891E1DECF8CE891E19F938F937E
:101BF000DF93CF93E0913B05F0913C05099510E010
:101C00000F900F900F900F9080912105843011F06C
